:100000000C94BB0A0C94E80A0C94E80A0C94E80AD5
:100010000C94E80A0C94E80A0C94E80A0C94E80A98
:100020000C94E80A0C94E80A0C94E80A0C94E80A88
:100030000C94E80A0C94E80A0C94E80A0C94E80A78
:100040000C94E80A0C9445130C94E80A0C94E80A02
:100050000C94E80A0C94E80A0C9424860C945A96A2
:100060000C94E80A0C94FE4E0C94E80A0C94E80AEE
:100070000C94E80A0C94E80A0C94E80A0C94E80A38
:100080000C94DF3A0C94E80A0C94E80A0C94E80A01
:100090000C94E80A0C94E80A0C94E80A0C949E91DB
:1000A0000C94E80A0C94E80A0C94B23A0C94E80A0E
:1000B0000C94E80A0C94E80A0C94E80A0C94853A2B
:1000C0000C94E80A0C94E80A0C94E80A0C94E80AE8
:1000D0000C94E80A0C94E80A0C94E80A0C94E80AD8
:1000E0000C94E80A084AD73B3BCE016E84BCBFFDA6
:1000F000C12F3D6C74319ABD56833DDA3D00C77FF8
:1001000011BED9E4BB4C3E916BAAAABE0000008090
:100110003F05A84CCDB2D44EB93836A9020C50B91F
:10012000918688083CA6AAAA2ABE000000803F4506
:10013000313A200045303A20005A3A2000593A20FE
:1001400000583A20004D53312C4D53322050696EE7
:10015000730A0024F404D9201BC40C5C0E9804C458
:10016000095F0265077101F405F900FB04B300485B
:10017000048700C10369005803550003034500BE0E
:10018000023A008402310053022A002902250004A9
:10019000022000E4011C00C8011900AF01170098FB
:1001A000011400840113007101100061011000515D
:1001B000010E0043010D0036010B002B010B002046
:1001C000010B00150109000C01090003010800FBE7
:1001D000000800F3000800EB000700E4000600DE62
:1001E000000600D8000600D2000600CC000500C7BB
:1001F000000500C2000500BD000400B9000400B500
:10020000000400B1000400AD000400A9000400A532
:10021000000300A20003009F0004009B000300985D
:100220000003009500020093000300900003008D7E
:100230000002008B00030088000200860002008498
:10024000000300810002007F0002007D0002007BAD
:1002500000020079000200770001007600020074BD
:1002600000020072000100710002006F0002006DC8
:100270000001006C0002006A0001006900020067D2
:1002800000010066000100650001006400020062D8
:1002900000010061000100600001005F0002005DDC
:1002A0000001005C0001005B0001005A00010059E0
:1002B00000010058000100570001005600010055E0
:1002C00000010054000100530000005300010052DF
:1002D00000010051000100500001004F0001004EDC
:1002E0000000004E0001004D0001004C0001004BD9
:1002F0000000004B0001004A0001004900010048D5
:1003000000000048000100470001004600000046D0
:1003100000010045000000450001004400010043C9
:1003200000000043000100420000004200010041C3
:1003300000000041000100400001003F0000003FBC
:100340000001003E0000003E0001003D0000003DB5
:100350000001003C0000003C0000003C0001003BAC
:100360000000003B0001003A0000003A00010039A3
:10037000000000390001003800000038000000389B
:100380000001003700000037000100360000003691
:100390000000003600010035000000350000003587
:1003A000000100340000003400000034000100337C
:1003B0000000003300000033000100320000003272
:1003C0000000003200010031000000310000003167
:1003D0000001003000000030000000300001002F5C
:1003E0000000002F0000002F0000002F0001002E51
:1003F0000000002E0000002E0001002D0000002D46
:100400000000002D0000002D0001002C0000002C39
:100410000000002C0000002C0001002B0000002B2D
:100420000000002B0000002B0001002A0000002A21
:100430000000002A0000002A000100290000002915
:100440000000002900000029000000290001002808
:1004500000000028000000280000002800000028FC
:1004600000010027000000270000002700000027EF
:1004700000000027000100260000002600000026E2
:1004800000000026000000260001002500000025D5
:1004900000000025000000250000002500000025C8
:1004A00000010024000000240000002400000024BB
:1004B00000000024000100230000002300000023AE
:1004C00000000023000000230000002300000023A0
:1004D0000001002200000022000000220000002293
:1004E0000000002200000022000100210000002185
:1004F0000000002100000021000000210000002178
:100500000000002100010020000000200000002069
:10051000000000200000002000000020000000205B
:10052000000000200001001F0000001F0000001F4D
:100530000000001F0000001F0000001F0000001F3F
:100540000001001E0000001E0000001E0000001E32
:1005500000000024F4D43050C38E20C2A240178281
:100560008B7011127A910D816CD90AA861E108C7CC
:10057000586607615143061E4B5D05C145A7041A25
:10058000411104093D9803713931034036DB02659E
:10059000339102D4305402802E1D02632CEE01757B
:1005A0002AC501B028A001102781018F2564012BE5
:1005B000244B01E0223401AC211F018D200D01806C
:1005C0001FFC00841EED00971DDF00B81CD200E662
:1005D0001BC600201BBC00641AB200B219A8000A96
:1005E00019A0006A189900D117910040178B00B527
:1005F00016840031167E00B31579003A157300C7D2
:10060000146F0058146A00EE136600881363002507
:10061000135E00C7125B006C12570015125400C124
:1006200011510070114F0021114B00D61049008D5F
:100630001047004610440002104200C00F400080E6
:100640000F3E00420F3C00060F3B00CB0E380093DC
:100650000E37005C0E3500270E3400F30D3200C15A
:100660000D3100900D3000600D2E00320D2D000573
:100670000D2C00D90C2B00AE0C2900850C29005C38
:100680000C2700350C27000E0C2600E80B2400C4B4
:100690000B2400A00B23007D0B23005A0B210039F3
:1006A0000B2100180B2000F80A1F00D90A1E00BBFE
:1006B0000A1E009D0A1D00800A1D00630A1C0047D7
:1006C0000A1B002C0A1B00110A1A00F7091A00DD88
:1006D000091900C4091900AB091900920917007B18
:1006E000091800630917004C091600360916002086
:1006F0000916000A091500F5081500E0081400CCD9
:10070000081400B8081400A4081400900813007D11
:100710000812006B08130058081200460812003433
:10072000081100230811001208110001081100F03F
:10073000071000E0071000D0071000C0071000B03D
:10074000070F00A107100091070E0083070F007428
:10075000070F0065070E0057070E0049070E003B04
:10076000070D002E070E0020070D0013070D0006D1
:10077000070D00F9060C00ED060D00E0060C00D494
:10078000060C00C8060C00BC060C00B0060C00A449
:10079000060B0099060C008D060B0082060B0077F5
:1007A000060B006C060B0061060A0057060B004C96
:1007B000060A0042060A0038060A002E060A00242D
:1007C000060A001A060A001006090007060A00FDBC
:1007D000050900F4050900EB050900E2050900D947
:1007E000050900D0050900C7050900BE050900B5C7
:1007F000050800AD050800A50509009C0508009442
:100800000508008C050800840508007C05080074B4
:100810000508006C050700650508005D0507005622
:100820000508004E05070047050700400508003889
:10083000050700310507002A050700230507001CEE
:10084000050600160507000F05070008050600024B
:10085000050700FB040600F5040700EE040600E8A7
:10086000040600E2040700DB040600D5040600CFFE
:10087000040600C9040600C3040600BD040600B750
:10088000040600B1040500AC040600A6040600A09E
:100890000405009B04060095040500900406008AE8
:1008A00004050085040500800406007A040500752F
:1008B000040500700405006B040500660405006172
:1008C0000405005C04050057040500520405004DB2
:1008D00004050048040500430405003E0404003AF2
:1008E00004050035040500300404002C040500272D
:1008F000040400230405001E0404001A0404001666
:10090000040500110404000D04040009040500049A
:1009100004040000040400FC030400F8030400F4D1
:10092000030400F0030400EC030400E8030400E403
:10093000030400E0030400DC030400D8030400D433
:10094000030400D0030400CC030400C8030300C563
:100950000303006563686F3A00205A3A0020593A51
:100960000020583A00656E6473746F707320686974
:10097000743A20006563686F3A0020746F6F206CD2
:100980006F6E6720657874727573696F6E20707210
:100990006576656E7465640020636F6C64206578AD
:1009A00074727573696F6E2070726576656E7465AA
:1009B00064000A0020000A00207A3A200020793AD8
:1009C000200020783A20006563686F3A0048617221
:1009D00064636F6465642044656661756C7420535C
:1009E000657474696E6773204C6F6164656400534D
:1009F000746F7265642073657474696E67732072B6
:100A000065747269657665640020440020490020A1
:100A100020204D33303120500050494420736574FC
:100A200074696E67733A00205A0020590020204DE7
:100A3000323036205800486F6D65206F66667365EA
:100A40007420286D6D293A00204500205A00205856
:100A50000020420020540020204D32303520530029
:100A6000416476616E636564207661726961626C6F
:100A700065733A20533D4D696E2066656564726109
:100A8000746520286D6D2F73292C20543D4D696E9F
:100A90002074726176656C20666565647261746548
:100AA00020286D6D2F73292C20423D6D696E696D74
:100AB000756D207365676D656E742074696D652052
:100AC000286D73292C20583D6D6178696D756D20F6
:100AD0005859206A65726B20286D6D2F73292C2060
:100AE000205A3D6D6178696D756D205A206A657276
:100AF0006B20286D6D2F73292C2020453D6D61786A
:100B0000696D756D2045206A65726B20286D6D2FAB
:100B100073290020540020204D32303420530041EE
:100B20006363656C65726174696F6E3A20533D61F1
:100B30006363656C65726174696F6E2C20543D72DD
:100B400065747261637420616363656C657261745E
:100B5000696F6E00204500205A0020590020204D6A
:100B60003230312058004D6178696D756D204163D8
:100B700063656C65726174696F6E20286D6D2F738B
:100B800032293A00204500205A0020590020204DEB
:100B90003230332058004D6178696D756D2066657F
:100BA0006564726174657320286D6D2F73293A0036
:100BB000204500205A0020590020204D393220586D
:100BC0000053746570732070657220756E69743A95
:100BD0000053657474696E67732053746F72656433
:100BE000006563686F3A004572726F723A00507226
:100BF000696E7465722073746F70706564206475BB
:100C00006520746F206572726F72732E204669784A
:100C100020746865206572726F7220616E64207541
:100C20007365204D39393920746F20726573746192
:100C300072742E202854656D7065726174757265CA
:100C40002069732072657365742E20536574206962
:100C50007420616674657220726573746172746960
:100C60006E6729005072696E7465722068616C74D9
:100C700065642E206B696C6C28292063616C6C653F
:100C80006421006F6B00526573656E643A20002228
:100C900000556E6B6E6F776E20636F6D6D616E6465
:100CA0003A2022005A204F6666736574203A20006D
:100CB0007A5F6D61783A20007A5F6D696E3A200044
:100CC0005A204F6666736574005A204F66667365D6
:100CD00074206F6B007A5F6D61783A20007A5F6DE7
:100CE000696E3A2000795F6D61783A2000795F6D16
:100CF000696E3A2000785F6D61783A2000785F6D08
:100D0000696E3A2000205A3A0020593A0020436F79
:100D1000756E7420583A200020453A00205A3A0057
:100D200020593A00583A004649524D574152455FC2
:100D30004E414D453A4D61726C696E2056313B20F3
:100D4000537072696E7465722F6772626C206D6188
:100D50007368757020666F722067656E362046492D
:100D6000524D574152455F55524C3A6874747073F6
:100D70003A2F2F6769746875622E636F6D2F457205
:100D8000696B5A616C6D2F4D61726C696E2F2050CA
:100D9000524F544F434F4C5F56455253494F4E3A72
:100DA000312E30204D414348494E455F54595045FE
:100DB0003A4D656E64656C20455854525544455211
:100DC0005F434F554E543A3120555549443A3030DF
:100DD0003030303030302D303030302D3030303019
:100DE0002D303030302D3030303030303030303009
:100DF00030300A0020423A0020453A00543A0020A0
:100E0000573A0020453A00543A002042403A002028
:100E1000403A00202F003A00205400202F002042AA
:100E20003A00202F006F6B20543A002569206D692D
:100E30006E2C20256920736563000A00205A3A2031
:100E40000020593A200020583A20004265640050A2
:100E5000726F62696E6720646F6E65210020643A6C
:100E6000200020623A200045716E20636F6566663F
:100E7000696369656E74733A20613A2000486F6D4A
:100E80006520582F59206265666F7265205A00FFF1
:100E9000FF01000025430000394300001F4300000C
:100EA00000000000000000001F43000000000000E0
:100EB000000000000000000025430000394300004E
:100EC0001F430000A0400000A040000000400A00B6
:100ED000207A3A200020793A200020783A200042F7
:100EE0006564005072696E7465722073746F7070FF
:100EF00065642064756520746F206572726F72730B
:100F00002E2046697820746865206572726F7220A1
:100F1000616E6420757365204D39393920746F20F6
:100F2000726573746172742E202854656D706572D9
:100F300061747572652069732072657365742E2003
:100F400053657420697420616674657220726573DC
:100F500074617274696E6729006F6B004E6F204C6C
:100F6000696E65204E756D626572207769746820C0
:100F7000636865636B73756D2C204C617374204CD2
:100F8000696E653A20004E6F20436865636B737528
:100F90006D2077697468206C696E65206E756D626E
:100FA00065722C204C617374204C696E653A200088
:100FB000636865636B73756D206D69736D617463D0
:100FC000682C204C617374204C696E653A20004C8B
:100FD000696E65204E756D626572206973206E6F53
:100FE00074204C617374204C696E65204E756D627F
:100FF00065722B312C204C617374204C696E653AFC
:1010000020004D313130002020506C616E6E6572D1
:1010100042756666657242797465733A20002046AF
:10102000726565204D656D6F72793A20004D61796A
:10103000203132203230313500436F6D70696C657C
:10104000643A200028416C657068204F626A6563CD
:10105000747320496E632C204D696E692D323031D6
:101060003551312900207C20417574686F723A2017
:10107000004D617920313220323031352031303A23
:1010800030303A343300204C617374205570646101
:101090007465643A2000312E302E30004D61726C40
:1010A000696E0020536F66747761726520526573B4
:1010B000657400205761746368646F6720526573BC
:1010C0006574002042726F776E206F7574205265D0
:1010D000736574002045787465726E616C2052658A
:1010E00073657400506F7765725570007374617228
:1010F00074002200656E717565696E67202200229A
:1011000000656E717565696E672022004572726FA9
:10111000723A0054656D706572617475726520680D
:1011200065617465642062656420737769746368BF
:101130006564206F66662E204D415854454D502001
:10114000747269676765726564202121003A2045E1
:101150007874727564657220737769746368656406
:10116000206F66662E204D494E54454D50207472B6
:10117000696767657265642021003A20457874725A
:1011800075646572207377697463686564206F663F
:10119000662E204D415854454D5020747269676742
:1011A00065726564202100202D20496E76616C698E
:1011B00064206578747275646572206E756D626501
:1011C000722021001000AD0330016A0150022B0192
:1011D00070030A019004F500B005E500D006D800C0
:1011E000F007CE001009C500300ABE00500BB70052
:1011F000700CB100900DAB00B00EA600D00FA20095
:10120000F0109D00101299003013950050149200B8
:1012100070158E0090168B00B0178700D0188400D0
:10122000F0198100101B7E00301C7B00501D7900DE
:10123000701E7600901F7300B0207000D0216E00E9
:10124000F0226B00102469003025660050266300F0
:101250007027610090285E00B0295C00D02A5900F8
:10126000F02B5600102D5400302E5100502F4E0000
:1012700070304B0090314800B0324500D03342000E
:10128000F0343E0010363B00303737005038330022
:1012900070392E00903A2900B03B2300D03C1B004F
:1012A000F03D1100103F0100F03F00005049442084
:1012B0004175746F74756E652066696E69736865D3
:1012C00064212050757420746865204B702C204B6D
:1012D0006920616E64204B6420636F6E7374616E6D
:1012E000747320696E746F20436F6E6669677572E0
:1012F0006174696F6E2E6800504944204175746FA7
:1013000074756E65206661696C6564212074696D11
:10131000656F75740020403A006F6B20543A006F7F
:101320006B20423A00504944204175746F74756EC9
:1013300065206661696C6564212054656D70657215
:10134000617475726520746F6F206869676800202A
:101350004B643A2000204B693A2000204B703A2021
:101360000020436C6173696320504944200020547D
:10137000753A2000204B753A2000206D61783A20A4
:1013800000206D696E3A200020643A2000206269D6
:1013900061733A20001000C90210012C01400122A3
:1013A0000170011801B0010E01F00104015002FAB0
:1013B00000B002F0003003E600D003DC009004D25D
:1013C000007005C800A006BE000008B400B009AA5D
:1013D00000D00BA000600E960060118C00001582FA
:1013E0000020197800C01D6E00A0226400B0275AAA
:1013F00000902C500000314600E0343C00103832A0
:1014000000903A2800603C1E00A03D1400803E0A77
:1014100000203F000000002100240027002A002DAA
:10142000003000330001010000040107010A01003F
:10143000002200250028002B002E0031003400027D
:10144000010000050108010B010000200023002617
:101450000029002C002F00320000010000030106CB
:10146000010901050505050705080808080202022B
:10147000020A0A080804040404010101010101012F
:10148000010303030303030303040707070C0C0C06
:101490000C0C0C0C0C0202020206060606060606DE
:1014A000060B0B0B0B0B0B0B0B010210202008087B
:1014B00010204010204080020102010804020101B6
:1014C000020408102040808040201008040201809F
:1014D00004020180402010080402010804020101F6
:1014E00002040810204080010204081020408000FF
:1014F00000090A02080B0C0D070603040100000096
:1015000000000000000000000000000000000000DB
:10151000000000000000000000000011100F00009B
:1015200000000000000000000000000000000000BB
:101530000000000000494E46494E4954594E414E64
:10154000CDCCCC3D0AD7233C17B7D13877CC2B3242
:101550009595E6241FB14F0A000020410000C842C3
:1015600000401C4620BCBE4CCA1B0E5AAEC59D7422
:10157000924F9B5A0D9111241FBECFEFD1E2DEBFD7
:10158000CDBF00E00CBF14E0A0E0B2E0E2E3FAE37C
:1015900001E00BBF02C007900D92AA3AB107D9F73C
:1015A0001BBE1EE0AAEAB4E001C01D92A23EB10734
:1015B000E1F715E1C6E7D5E104C02297FE010E94DC
:1015C000D19CC037D107C9F70E94B2970C94179DE0
:1015D0000C940000A0E0B0E0E0EFFAE00C94E69C90
:1015E000EC015B016115710519F0FB0191838083AA
:1015F000F9908F2D90E00E94D59C892BC9F7FDE2D0
:10160000FF1621F4F990EE24E39405C02BE2F216C4
:1016100009F4F990EE248E0101501040C80165E3F1
:1016200075E143E050E062D2892BF9F48E010E5F40
:101630001F4FC80168E375E145E050E057D2892BA0
:1016400019F48E01095F1F4FA114B10419F0F501BF
:1016500011830083E0FC04C070E090E080E813C0D8
:1016600070E090E080E86FEF07C1C8016DE375E1BD
:1016700043E050E03BD2892B69F4A114B10429F472
:1016800070E090E080EC6FE7F7C02296F501D1831F
:10169000C083F6CF8824992440E050E060E070E0F9
:1016A000EF2DE053EA30A0F5F2E0EF2A8E2D90E026
:1016B0009C0128703070E2FE06C0232B79F5089457
:1016C000811C911C2BC0232B19F0089481089108D0
:1016D000DB01CA0112E0880F991FAA1FBB1F1A95D0
:1016E000D1F7480F591F6A1F7B1F440F551F661FF4
:1016F000771F4E0F511D611D711D483929E9520791
:1017000029E9620729E1720748F084E0E82A06C067
:10171000EE3F31F4E3FC39C098E0E92AF990C0CFFC
:10172000E53311F0E53189F529912D3219F4E0E125
:10173000EE2A05C02B3219F081E090E003C0299118
:1017400082E090E0E22FE053EA3018F0C81BD90B9A
:101750001CC020E030E0FCE020383F075CF4C90109
:10176000880F991F880F991F280F391F220F331FC9
:101770002E0F311DE991E053EA3068F3E4FE03C017
:10178000309521953F4F820E931ECE2CDD24E1FE35
:1017900007C0A114B10421F02197F501D183C083C2
:1017A000CB01BA010E943A997B018C01F3E0CF2270
:1017B000DD2423E0C216D10421F417FB109517F99C
:1017C000109557016801C801B70120E030E040E002
:1017D00050E00E949A98882309F44AC097FE0DC0F1
:1017E00024E5E22E25E1F22E9094819491089394C1
:1017F000C0E2D0E000E010E012C09CE6E92E95E1E6
:10180000F92EF6CFF7012591359145915491C601F6
:10181000B5010E947A9B5B016C018C1A9D0A8C16A3
:101820009D0684F7D595C7950F5F1F4F06301105AC
:1018300029F08CEF9FEFE80EF91EF1CFC501D6011C
:101840007C018D018C2D880F8D2D881F8F3F51F0CD
:10185000C601B50120E030E040E050E00E949A98D7
:10186000882331F482E290E09093E10E8093E00EC1
:101870007E2D9F2D802F612F272F392F482F562FF8
:10188000B901CA01CDB7DEB7ECE00C94029D2F92EE
:101890003F925F926F927F928F929F92AF92BF9290
:1018A000CF92DF92EF92FF920F931F93CF93DF932C
:1018B0008C011B01EA016115710519F0FB0191838F
:1018C0008083209749F0CE010297839728F020E08B
:1018D00030E040E050E0F6C0F801A1908F018A2D81
:1018E00090E00E94D59C892BB9F7FDE2AF1631F448
:1018F000F801A1908F015524539407C0FBE2AF1665
:1019000019F4F801A1908F015524209719F0C031E6
:10191000D105C1F4F0E3AF1679F4F801808188377E
:1019200011F0883549F4F801A1800E5F1F4FF2E0F5
:101930005F2AC0E1D0E006C0209721F480E3A8161A
:10194000E9F427C0C830D10531F1C930D10524F4FC
:10195000C230D10531F50CC0CA30D10589F0C03193
:10196000D105F9F4C12CD12CE12CB8E0FB2E28C014
:10197000C12CD12CE12CA0E4FA2E22C0CAE0D0E088
:10198000FCECCF2EFCECDF2EFCECEF2EFCE0FF2E6F
:1019900017C0C8E0D0E0C12CD12CE12CE0E1FE2E34
:1019A0000FC09E01442737FD4095542F60E070E042
:1019B00080E090E80E94929CC901DA016C017D01EF
:1019C00020E030E040E050E060E03E01882477FC19
:1019D0008094982C70EDB72EBA0CE9E0EB1570F4FA
:1019E0008A2D81548A3118F499ECB92E06C08A2DBB
:1019F00081568A3150F589EAB82EBA0C8B2D90E0C9
:101A00008C179D0714F56F3FE1F0C216D306E4066C
:101A1000F506B0F0CA01B901A40193010E944C9CE3
:101A20009B01AC012B0D311D411D511D2130F0E0FA
:101A30003F07F0E04F07F0E85F0710F461E001C0F6
:101A40006FEFF801A1908F01C5CF2114310481F00F
:101A5000662331F001501040F1011183008308C06A
:101A600051FE1AC002501040F1011183008314C0CE
:101A700067FF12C050FC05C02FEF3FEF4FEF5FE74D
:101A800004C020E030E040E050E882E290E0909333
:101A9000E10E8093E00E16C050FE08C050954095B0
:101AA000309521953F4F4F4F5F4F0CC057FF0AC0F5
:101AB00082E290E09093E10E8093E00E2FEF3FEFF3
:101AC0004FEF5FE7B901CA01DF91CF911F910F91ED
:101AD000FF90EF90DF90CF90BF90AF909F908F904E
:101AE0007F906F905F903F902F900895FB01DC01F5
:101AF0004150504088F08D9181341CF08B350CF4AE
:101B0000805E659161341CF06B350CF4605E861B61
:101B1000611171F3990B0895881BFCCFFB0155915E
:101B20005523A9F0BF01DC014D9145174111E1F7A3
:101B300059F4CD010590002049F04D914015411117
:101B4000C9F3FB014111EFCF81E090E001970895C7
:101B5000FC018191861721F08823D9F799270895F0
:101B60003197CF010895FB01DC018D91019080191F
:101B70000110D9F3990B0895FB01DC01415050404D
:101B800030F08D910190801919F40020B9F7881B6D
:101B9000990B0895AEE0B0E0E0EDFDE00C94EE9C12
:101BA0000E891F898EE08C831A8309838FEF9FE74C
:101BB0009E838D839E01265E3F4FCE010196688DE8
:101BC000798DA9010AD02F813885020F131FF801E2
:101BD00010822E96E4E00C940A9DABE0B0E0E3EFB7
:101BE000FDE00C94E09C3C012B015A01FC011782A2
:101BF0001682838181FD03C06FEF7FEFB9C19AE048
:101C0000892E1E010894211C311CF3012381F2014D
:101C100023FD859123FF81912F01882309F4A5C11C
:101C2000853239F423FD859123FF81912F0185327F
:101C300021F490E0B301B7D1E8CF982FFF24EE2430
:101C40009924FFE1FF15D0F09B3269F09C3228F413
:101C5000903259F0933291F40EC09D3249F0903396
:101C600069F441E024C052E0F52A84E0F82A28C053
:101C700098E0F92A25C0E0E1FE2A22C0F7FC29C03D
:101C8000892F80538A3070F4F6FE05C0989C902C02
:101C90001124980E15C0E89CE02C1124E80EF0E207
:101CA000FF2A0EC09E3229F4F6FC5FC140E4F42AFC
:101CB00007C09C3619F450E8F52A02C0983649F45A
:101CC000F20123FD959123FF91912F01992309F0B2
:101CD000B8CF892F8554833018F08052833038F480
:101CE00044E050E0A40EB51E5FE359830FC0933665
:101CF00031F0933779F0933509F052C01FC0F501E8
:101D00008081898342E050E0A40EB51E610101E0AC
:101D100010E011C0F501C080D180F6FC03C06FEF68
:101D20007FEF02C0692D70E042E050E0A40EB51EC6
:101D3000C6012ED18C015FE7F52213C0F501C080EA
:101D4000D180F6FC03C06FEF7FEF02C0692D70E019
:101D500042E050E0A40EB51EC6010FD18C0150E840
:101D6000F52AF3FE06C018C080E290E0B3011BD153
:101D7000EA948E2D90E008171907B0F30DC0F60114
:101D8000F7FC8591F7FE81916F0190E0B3010BD1D3
:101D9000E110EA94015010400115110581F7E2C0ED
:101DA000943611F0993661F5F7FE08C0F5012081EF
:101DB00031814281538184E090E00AC0F501808145
:101DC00091819C01442737FD4095542F82E090E09B
:101DD000A80EB91E9FE6F92257FF09C050954095FD
:101DE000309521953F4F4F4F5F4FE0E8FE2ACA01E3
:101DF000B901A1012AE030E002D1D82ED2183FC0AB
:101E0000953729F41F2D1F7E2AE030E01DC01F2DBD
:101E1000197F9F3661F0903720F4983509F0A5C0FE
:101E20000FC0903739F0983709F09FC004C028E000
:101E300030E00AC0106114FD146020E130E004C0FD
:101E400014FD166020E132E017FF08C0F501608143
:101E500071818281938144E050E008C0F501808166
:101E60009181BC0180E090E042E050E0A40EB51EFC
:101E7000A101C5D0D82ED2188FE7F82EF122F6FE98
:101E80000BC05EEFF522D91438F4F4FE07C0F2FC63
:101E900005C08FEEF82202C01D2D01C0192DF4FEE1
:101EA0000DC0FE01ED0DF11D8081803319F499EE16
:101EB000F92208C01F5FF2FE05C003C08F2D86788F
:101EC00009F01F5F0F2DF3FC13C0F0FE0EC01E15AE
:101ED00010F09D2C0AC09D2C9E0C911A1E2D05C041
:101EE00080E290E0B3015FD01F5F1E15C8F304C00D
:101EF0001E1510F4E11A01C0EE2404FF0EC080E3A9
:101F000090E0B30150D002FF1BC001FD03C088E781
:101F100090E00EC088E590E00BC0802F867881F0BD
:101F200001FF02C08BE201C080E2F7FC8DE290E08D
:101F3000B30139D005C080E390E0B30134D09A9466
:101F4000D914C8F3DA94F101ED0DF11D808190E010
:101F5000B30129D0DD20B1F705C080E290E0B301E4
:101F600022D0EA94EE20C9F750CEF3016681778142
:101F7000CB012B96E2E10C94FC9CFC010590615096
:101F800070400110D8F7809590958E0F9F1F08958F
:101F9000FC016150704001900110D8F78095909538
:101FA0008E0F9F1F08950F931F93CF93DF938C0184
:101FB000EB018B8181FF1BC082FF0DC02E813F8111
:101FC0008C819D812817390764F4E881F981019398
:101FD000F983E88306C0E885F985802F1995892B58
:101FE00031F48E819F8101969F838E8302C00FEF13
:101FF0001FEFC801DF91CF911F910F910895FA0152
:10200000AA27283051F1203181F1E8946F936E7F37
:102010006E5F7F4F8F4F9F4FAF4FB1E03ED0B4E028
:102020003CD0670F781F891F9A1FA11D680F791F69
:102030008A1F911DA11D6A0F711D811D911DA11D7A
:1020400020D009F468943F912AE0269F112430198A
:10205000305D3193DEF6CF010895462F4770405D25
:102060004193B3E00FD0C9F7F6CF462F4F70405DD4
:102070004A3318F0495D31FD4052419302D0A9F72F
:10208000EACFB4E0A6959795879577956795BA9529
:10209000C9F700976105710508959B01AC010A2EEF
:1020A00006945795479537952795BA95C9F7620FC6
:1020B000731F841F951FA01D08951092E0041092B5
:1020C000E7041092EE040895809387030895EFE6E5
:1020D000F0E080818260808308951F93FC011FB728
:1020E000F89480819181A281B3818093B804909308
:1020F000B904A093BA04B093BB04FB018081918121
:10210000A281B3818093BC049093BD04A093BE04CC
:10211000B093BF04FA0180819181A281B381809341
:10212000C0049093C104A093C204B093C304F90106
:1021300080819181A281B3818093C4049093C5046E
:10214000A093C604B093C7041FBF1F910895FC015C
:102150002FB7F89480819181A281B3818093C404C8
:102160009093C504A093C604B093C7042FBF0895ED
:10217000E82F8FB7F894F0E0EE0FFF1FEE0FFF1F70
:10218000E854FB4F20813181428153818FBFB901D7
:10219000CA010895CF93DF932FB7F894C82FD0E0EA
:1021A000CC0FDD1FCC0FDD1FFE01E854FB4F60811B
:1021B0007181828193812FBF0E943C99CB5EDA4F5F
:1021C000288139814A815B810E94A198DF91CF915A
:1021D0000895E5E4F1E0949108C08091C00085FF86
:1021E000FCCF9093C600319694919923B1F7E1E426
:1021F000F1E0949108C08091C00085FFFCCF9093DE
:10220000C600319694919923B1F788E20E94189400
:10221000BC0184E99BE04AE050E00E947A5089E2E8
:102220000E941894BC0184E99BE04AE050E00E94BF
:102230007A508091C00085FFFCCF8AE08093C60071
:10224000EDE3F1E0949108C08091C00085FFFCCFE0
:102250009093C600319694919923B1F785E40E943A
:102260001894BC0184E99BE04AE050E00E947A5057
:1022700087E20E941894BC0184E99BE04AE050E0A8
:102280000E947A508091C00085FFFCCF8AE0809345
:10229000C600E9E3F1E0949108C08091C00085FF99
:1022A000FCCF9093C600319694919923B1F784E4C2
:1022B0000E941894BC0184E99BE04AE050E00E942F
:1022C0007A5083E40E941894BC0184E99BE04AE0C0
:1022D00050E00E947A508091C00085FFFCCF8AE0D8
:1022E0008093C600E4E3F1E0949108C08091C000BF
:1022F00085FFFCCF9093C600319694919923B1F756
:1023000081E40E941894BC0184E99BE04AE050E01B
:102310000E947A5082E40E941894BC0184E99BE0F8
:102320004AE050E00E947A508091C00085FFFCCFC7
:102330008AE08093C600EFE2F1E0949108C08091BA
:10234000C00085FFFCCF9093C600319694919923ED
:10235000B1F78FE30E941894BC0184E99BE04AE046
:1023600050E00E947A5080E40E941894BC0184E9F5
:102370009BE04AE050E00E947A508091C00085FFC7
:10238000FCCF8AE08093C60008950F931F93182F07
:10239000042F67FD19C0823081F0833028F4882330
:1023A00041F0813089F407C0833049F0843061F412
:1023B00008C088E207C085E405C084E403C081E466
:1023C00001C08FE30E94E69307FD1AC0123081F02E
:1023D000133028F4112341F0113091F407C0133069
:1023E00049F0143069F408C089E207C087E205C0EB
:1023F00083E403C082E401C080E4602F0E94E6937E
:102400001F910F910895643089F0653028F4613090
:1024100041F0623099F407C0683051F0603171F4D6
:102420000AC060E001C061E040E004C060E001C0BB
:1024300061E041E0AACF61E041E0A7CF0895CF93EA
:10244000DF938FE361E00E94339380E461E00E94B8
:10245000339388E261E00E94339389E261E00E9455
:10246000339385E461E00E94339387E261E00E9448
:10247000339384E461E00E94339383E461E00E943B
:10248000339381E461E00E94339382E461E00E942F
:102490003393C0E0D0E0FE01EA5DFB4F8C2F6081FA
:1024A000B2DF2196C530D105B1F7DF91CF91089504
:1024B0009B01882399F4B901882777FD8095982F8F
:1024C0002FEF30E040E050E00E944C9C20ED37E0E0
:1024D00040E050E00E94B49C8CE214C08130A9F42A
:1024E000B901882777FD8095982F2FEF30E040E0E5
:1024F00050E00E944C9C20ED37E040E050E00E940C
:10250000B49C8DE2B9010C947C958230A9F4B90198
:10251000882777FD8095982F2FEF30E040E050E03E
:102520000E944C9C20ED37E040E050E00E94B49CBB
:102530008EE2B9010C947C9508958CE261E00E94D2
:1025400033938DE261E00E9433938EE261E00E945A
:10255000339360917B0370917C0380E0A9DF6091ED
:102560007D0370917E0381E0A3DF60917F03709112
:10257000800382E09DDFE1E2F1E08081887F81607D
:1025800080830895DADF5BDFEAE0F1E0808182603A
:10259000808380818160808380818460808380816A
:1025A000806480838081806880830F9A179A0E9A56
:1025B000169A0D9A159A0C9A149A0B9A139A2698B1
:1025C0002E9A25982D9A24982C9A3F98479A0A98E3
:1025D000129A0998119A389A4098179A1092C30B38
:1025E000399A4198169A1092C40B3A9A4298159AC1
:1025F0001092C50B3B9A4398149A3C9A4498A1E8D0
:10260000B0E08C918F7E8C938C9188608C93E0E805
:10261000F0E080818D7F808380818E7F80838081C8
:102620008F73808380818F7C80838C91887F826090
:102630008C9380E090E490938900809388001092BE
:10264000850010928400EFE6F0E080818260808354
:1026500081E080938703789408959091820A809115
:10266000830A981729F00E949F890E94DE66F5CFA1
:102670000895F3DF179A1092C30B169A1092C40BA9
:10268000159A1092C50B149A08951F920F920FB6C7
:102690000F920BB60F921124AF92BF92CF92DF929E
:1026A000EF92FF920F931F932F933F934F935F935C
:1026B0006F937F938F939F93AF93BF93CF93DF934A
:1026C000EF93FF938091AA049091AB04892B09F0BA
:1026D00099C19091820A8091830A981719F4E0E0D9
:1026E000F0E014C08091830A90E021E530E0829F01
:1026F000F001839FF00D929FF00D1124EE58FA4FD8
:10270000E05BFF4F81E08083E055F040F093AB0445
:10271000E093AA04309709F46FC1E05BFF4F81E0BA
:1027200080831092F9041092FA041092FB04109224
:10273000FC04E091AA04F091AB0460AD71AD2CE90A
:102740006134720718F060E47CE904C03EE4613251
:10275000730730F0769567957695679584E007C0A6
:1027600047E26131740730F07695679582E0809397
:10277000F20407C08093F2046032710510F460E245
:1027800070E06052704058E060307507E8F0472F05
:1027900050E0440F551F440F551F4D5A5E4F9A018C
:1027A0002E5F3F4FF901859194919C01AA27639F69
:1027B000C001629F810D9A1F06948A1F9A1F1124DF
:1027C000FA01459154911EC0CB01969587958C7F57
:1027D0008D5A9A4FFC0145915491FC0132962591F6
:1027E0003491862F90E087709070FC012E9FC0017D
:1027F0002F9F900D3E9F900D112403E09695879595
:102800000A95E1F7481B590B44365105A8F4E0E05E
:10281000F2E007C08091C00085FFFCCF3196909315
:10282000C60090819923B1F784E99BE04AE050E02B
:102830000E94A15044E650E05093FE044093FD04F2
:102840008091F204992787FD9095909300058093DD
:10285000FF04E091AA04F091AB0464AD75AD7093F0
:10286000F8046093F704FCE961347F0718F060E432
:102870007CE904C02EE46132720730F076956795EA
:102880007695679584E007C037E26131730730F0D1
:102890007695679582E08093F20408C081E080938A
:1028A000F2046032710510F460E270E06052704032
:1028B00048E060307407E8F0472F50E0440F551FA0
:1028C000440F551F4D5A5E4F9A012E5F3F4FF9013D
:1028D000859194919C01AA27639FC001629F810DFD
:1028E0009A1F06948A1F9A1F1124FA014591549148
:1028F0001EC0CB01969587958C7F8D5A9A4FFC010F
:1029000045915491FC01329625913491862F90E0A7
:1029100087709070FC012E9FC0012F9F900D3E9FED
:10292000900D1124E3E096958795EA95E1F7481B11
:10293000590B44365105A8F4E0E0F2E007C080915D
:10294000C00085FFFCCF31969093C60090819923FB
:10295000B1F784E99BE04AE050E00E94A15044E6D0
:1029600050E0CA01A0E0B0E08093F3049093F40437
:10297000A093F504B093F604509389004093880027
:10298000E091AA04F091AB0480899189A289B3896E
:10299000B695A79597958795B095A09590958195B3
:1029A0009F4FAF4FBF4F8093C8049093C904A0932B
:1029B000CA04B093CB048093CC049093CD04A0932D
:1029C000CE04B093CF048093D0049093D104A0930D
:1029D000D204B093D3048093D4049093D504A093ED
:1029E000D604B093D7041092D8041092D904109250
:1029F000DA041092DB0406C080ED97E09093890022
:102A000080938800E091AA04F091AB04309709F418
:102A100018C680A18093DC0480FF0AC08FB7F894A9
:102A200090910B019D7F90930B018FBF8FEF09C099
:102A30008FB7F89490910B01926090930B018FBF28
:102A400081E0809383038091DC0481FF0AC08FB70B
:102A5000F89490910B01916090930B018FBF8FEFD1
:102A600009C08FB7F89490910B019E7F90930B0152
:102A70008FBF81E0809384038091DC0420918703E1
:102A800080FF56C0222309F4A8C01E994AC0809135
:102A9000DD04882309F441C0E091AA04F091AB045D
:102AA00080819181A281B381181619061A061B062E
:102AB00054F52091DE043091DF04809181039091E0
:102AC000820382179307F8F48091B8049091B904B7
:102AD000A091BA04B091BB048093AC049093AD0470
:102AE000A093AE04B093AF0481E08093E0048089AA
:102AF0009189A289B3898093D8049093D904A09333
:102B0000DA04B093DB048091DE049091DF04019637
:102B10009093DF048093DE0460C081E08093DD0445
:102B20005CC01092DD041092DF041092DE0455C0E8
:102B3000222309F452C037994AC08091E1048823C6
:102B400009F441C0E091AA04F091AB048081918125
:102B5000A281B381181619061A061B0654F5209196
:102B6000E2043091E3048091810390918203821703
:102B70009307F8F48091B8049091B904A091BA0435
:102B8000B091BB048093AC049093AD04A093AE04C9
:102B9000B093AF0481E08093E00480899189A28999
:102BA000B3898093D8049093D904A093DA04B093A6
:102BB000DB048091E2049091E30401969093E30496
:102BC0008093E2040AC081E08093E10406C0109281
:102BD000E1041092E3041092E2048091DC0420915D
:102BE000870381FF56C0222309F4A8C01D994AC05B
:102BF0008091E404882309F441C0E091AA04F09193
:102C0000AB0484819581A681B781181619061A062E
:102C10001B0654F52091E5043091E6048091810370
:102C20009091820382179307F8F48091BC049091ED
:102C3000BD04A091BE04B091BF048093B0049093F2
:102C4000B104A093B204B093B30481E08093E7048D
:102C500080899189A289B3898093D8049093D904FB
:102C6000A093DA04B093DB048091E5049091E6042C
:102C700001969093E6048093E50460C081E0809320
:102C8000E4045CC01092E4041092E6041092E5049F
:102C900055C0222309F452C002994AC08091E80429
:102CA000882309F441C0E091AA04F091AB04848127
:102CB0009581A681B781181619061A061B0654F5C8
:102CC0002091E9043091EA0480918103909182037C
:102CD00082179307F8F48091BC049091BD04A091F1
:102CE000BE04B091BF048093B0049093B104A0934C
:102CF000B204B093B30481E08093E70480899189A2
:102D0000A289B3898093D8049093D904A093DA045C
:102D1000B093DB048091E9049091EA0401969093CA
:102D2000EA048093E9040AC081E08093E80406C0C5
:102D30001092E8041092EA041092E9048091DC04F5
:102D40002091870382FF61C08FB7F89490910B01A7
:102D50009B7F90930B018FBF8FEF8093850322237E
:102D600009F4B1C01C994AC08091EB04882309F48E
:102D700041C0E091AA04F091AB0480859185A285C1
:102D8000B385181619061A061B0654F52091EC0493
:102D90003091ED0480918103909182038217930713
:102DA000F8F48091C0049091C104A091C204B09144
:102DB000C3048093B4049093B504A093B604B09375
:102DC000B70481E08093EE0480899189A289B38958
:102DD0008093D8049093D904A093DA04B093DB04D1
:102DE0008091EC049091ED0401969093ED04809312
:102DF000EC0469C081E08093EB0465C01092EB04A1
:102E00001092ED041092EC045EC09FB7F89480918C
:102E10000B01846080930B019FBF41E040938503C9
:102E2000222309F450C0019948C08091EF048823FF
:102E300009F440C0E091AA04F091AB04808591852B
:102E4000A285B385181619061A061B064CF52091A3
:102E5000F0043091F10480918103909182038217F4
:102E60009307F0F48091C0049091C104A091C20432
:102E7000B091C3048093B4049093B504A093B604B6
:102E8000B093B7044093EE0480899189A289B389F5
:102E90008093D8049093D904A093DA04B093DB0410
:102EA0008091F0049091F10401969093F104809345
:102EB000F00409C04093EF0406C01092EF04109292
:102EC000F1041092F0048091DC0483FF0AC08FB7F4
:102ED000F89490910B01906490930B018FBF8FEF4A
:102EE00009C08FB7F89490910B019F7B90930B01D1
:102EF0008FBF81E08093860360E07EC18091C00037
:102F000087FF19C04091C600E091900BF091910BA2
:102F100031969F012F77307031978091920B90916D
:102F2000930B2817390739F0E05FF44F4083309353
:102F3000910B2093900BE091AA04F091AB042081B7
:102F40003181428153818091C8049091C904A0913C
:102F5000CA04B091CB04280F391F4A1F5B1F20936E
:102F6000C8043093C9044093CA045093CB0412168A
:102F70001306140615066CF5409A80899189A2897A
:102F8000B389281B390B4A0B5B0B2093C804309381
:102F9000C9044093CA045093CB042091B8043091E3
:102FA000B9044091BA045091BB04809183039927DE
:102FB00087FD9095A92FB92F820F931FA41FB51FCE
:102FC0008093B8049093B904A093BA04B093BB045F
:102FD0004098E091AA04F091AB04248135814681A8
:102FE00057818091CC049091CD04A091CE04B091F2
:102FF000CF04280F391F4A1F5B1F2093CC04309346
:10300000CD044093CE045093CF0412161306140639
:1030100015066CF5419A80899189A289B389281B8C
:10302000390B4A0B5B0B2093CC043093CD044093B7
:10303000CE045093CF042091BC043091BD04409144
:10304000BE045091BF0480918403992787FD909519
:10305000A92FB92F820F931FA41FB51F8093BC0403
:103060009093BD04A093BE04B093BF044198E09137
:10307000AA04F091AB042085318542855385809167
:10308000D0049091D104A091D204B091D304280F20
:10309000391F4A1F5B1F2093D0043093D104409303
:1030A000D2045093D30412161306140615066CF5B9
:1030B000429A80899189A289B389281B390B4A0BCE
:1030C0005B0B2093D0043093D1044093D2045093EF
:1030D000D3042091C0043091C1044091C2045091A6
:1030E000C30480918503992787FD9095A92FB92F57
:1030F000820F931FA41FB51F8093C0049093C10437
:10310000A093C204B093C3044298E091AA04F09142
:10311000AB0424853585468557858091D4049091EC
:10312000D504A091D604B091D704280F391F4A1FA7
:103130005B1F2093D4043093D5044093D60450935E
:10314000D70412161306140615066CF5439A8089E7
:103150009189A289B389281B390B4A0B5B0B2093F9
:10316000D4043093D5044093D6045093D7042091CF
:10317000C4043091C5044091C6045091C7048091A5
:103180008603992787FD9095A92FB92F820F931F4A
:10319000A41FB51F8093C4049093C504A093C604D4
:1031A000B093C70443988091D8049091D904A0911A
:1031B000DA04B091DB040196A11DB11D8093D804FF
:1031C0009093D904A093DA04B093DB042091D8043F
:1031D0003091D9044091DA045091DB04E091AA04C3
:1031E000F091AB0480899189A289B38928173907A6
:1031F0004A075B0730F46F5F8091F20468170CF4A4
:103200007DCE2091D8043091D9044091DA045091B8
:10321000DB04E091AA04F091AB0484899589A68926
:10322000B78982179307A407B50708F4E3C0E090B5
:10323000F304F090F4040091F5041091F604A48CCA
:10324000B58CC68CD78CA8019701C601B501AA27F9
:10325000279FB12D389FE001489FD00D479FC00D9B
:10326000D11D289FB00DC11DDA1F379FB00DC11DA4
:10327000DA1F469FB00DC11DDA1F369FB10DCA1F60
:10328000DA1FB695CA1FDA1F112484AD95AD8C0FD5
:103290009D1F9093F8048093F70420AD31AD42ADAB
:1032A00053ADA0E0B0E0281739074A075B0720F4C8
:1032B0003093F8042093F7046091F7047091F804B8
:1032C0008CE96134780718F060E47CE904C09EE47E
:1032D0006132790730F0769567957695679584E049
:1032E00007C0E7E261317E0730F07695679582E0AE
:1032F0008093F20408C081E08093F204603271058B
:1033000010F460E270E060527040F8E060307F07D7
:10331000E8F0472F50E0440F551F440F551F4D5AFA
:103320005E4F9A012E5F3F4FF901859194919C0168
:10333000AA27639FC001629F810D9A1F06948A1F6E
:103340009A1F1124FA01459154911EC0CB01969504
:1033500087958C7F8D5A9A4FFC0145915491FC01C1
:10336000329625913491862F90E087709070FC0101
:103370002E9FC0012F9F900D3E9F900D112403E0C2
:10338000969587950A95E1F7481B590B44365105E8
:10339000A8F4E0E0F2E007C08091C00085FFFCCF18
:1033A00031969093C60090819923B1F784E99BE010
:1033B0004AE050E00E94A15044E650E0509389005A
:1033C000409388009A0140E050E08091F30490918E
:1033D000F404A091F504B091F604820F931FA41F8A
:1033E000B51F8093F3049093F404A093F504B09375
:1033F000F60402C12091D8043091D9044091DA0436
:103400005091DB04808D918DA28DB38D821793072F
:10341000A407B50708F0E4C06091F9047091FA04BC
:103420008091FB049091FC04248D358D468D578D41
:10343000AA27639FB12D749FE001849FD00D839FC5
:10344000C00DD11D649FB00DC11DDA1F739FB00D5B
:10345000C11DDA1F829FB00DC11DDA1F729FB10D11
:10346000CA1FDA1FB695CA1FDA1F11248091F7040C
:103470009091F8048C179D0738F4E05CFF4F608151
:103480007181E054F04003C0BC016C1B7D0BE05C1B
:10349000FF4F2081318142815381CB01A0E0B0E018
:1034A00082179307A407B50708F4B901FCE9613452
:1034B0007F0718F060E47CE904C02EE461327207F3
:1034C00030F0769567957695679584E007C037E28A
:1034D0006131730730F07695679582E08093F2044E
:1034E00008C081E08093F2046032710510F460E25C
:1034F00070E06052704048E060307407E8F0472F99
:1035000050E0440F551F440F551F4D5A5E4F9A010E
:103510002E5F3F4FF901859194919C01AA27639FEB
:10352000C001629F810D9A1F06948A1F9A1F112461
:10353000FA01459154911EC0CB01969587958C7FD9
:103540008D5A9A4FFC0145915491FC013296259178
:103550003491862F90E087709070FC012E9FC001FF
:103560002F9F900D3E9F900D1124E3E09695879537
:10357000EA95E1F7481B590B44365105A8F4E0E001
:10358000F2E007C08091C00085FFFCCF3196909398
:10359000C60090819923B1F784E99BE04AE050E0AE
:1035A0000E94A15044E650E0509389004093880067
:1035B0009A0140E050E08091F9049091FA04A091C2
:1035C000FB04B091FC04820F931FA41FB51F8093CE
:1035D000F9049093FA04A093FB04B093FC040CC08C
:1035E0008091FD049091FE0490938900809388005F
:1035F0008091FF048093F2042091D8043091D90483
:103600004091DA045091DB04E091AA04F091AB04FC
:1036100080899189A289B389281739074A075B07EE
:1036200080F01092AB041092AA049091820A8091CB
:10363000830A981731F08091830A8F5F8F7080938F
:10364000830AFF91EF91DF91CF91BF91AF919F914D
:103650008F917F916F915F914F913F912F911F912A
:103660000F91FF90EF90DF90CF90BF90AF900F90B1
:103670000BBE0F900FBE0F901F9018958091E00425
:10368000882349F48091E704882329F48091EE048B
:10369000882309F490C0E3E5F9E0949108C0809193
:1036A000C00085FFFCCF9093C6003196949199237A
:1036B000B1F7E5E6F9E0949108C08091C00085FF7C
:1036C000FCCF9093C600319694919923B1F78091E5
:1036D000E0048823D1F06091AC047091AD04809136
:1036E000AE049091AF040E943C9920911505309151
:1036F000160540911705509118050E94A198AB013D
:10370000BC0181E699E00E94D35D8091E7048823A3
:10371000D1F06091B0047091B1048091B2049091A5
:10372000B3040E943C992091190530911A054091EB
:103730001B0550911C050E94A198AB01BC018DE5B1
:1037400099E00E94D35D8091EE048823D1F06091CE
:10375000B4047091B5048091B6049091B7040E94AE
:103760003C9920911D0530911E0540911F055091F7
:1037700020050E94A198AB01BC0189E599E00E9457
:10378000D35DE4E1F2E007C08091C00085FFFCCF8B
:1037900031969093C60090819923B1F78091C00033
:1037A00085FFFCCF8AE08093C6001092E00410925F
:1037B000E7041092EE0408953F924F925F926F9249
:1037C0007F928F929F92AF92BF92CF92DF92EF92B1
:1037D000FF920F931F93CF93DF93809171058823FE
:1037E00009F4F6C08090B0039090B103A090B203AA
:1037F000B090B3036091A70D7091A80D882777FD55
:103800008095982F0E943C9920E030E040E050E401
:103810000E94C197A50194010E949A9887FDD8C083
:103820003090830A0F2EF0E04F2EF0E05F2EF0E094
:103830006F2EF0E07F2EF02DC1E5D0E058C0232D93
:1038400030E02C9FF0012D9FF00D3C9FF00D1124D6
:10385000EE58FA4F80819181A281B3810097A10532
:10386000B10581F484819581A681B7810097A10576
:10387000B10541F480859185A285B3850097A105A6
:10388000B10591F12C9F60012D9FD00C3C9FD00C75
:10389000112482E795E0C80ED91EF601648575856E
:1038A000868597850E943C997B018C01F601608991
:1038B0007189828993890E943A999B01AC01C80160
:1038C000B7010E94A198F60122A133A144A155A1FC
:1038D0000E947A9B7B018C01A30192010E94A89A0D
:1038E000181614F4270138013394FFE03F22809129
:1038F000820A381609F0A3CFC301B2012091B403A4
:103900003091B5034091B6035091B7030E947A9B62
:103910009B01AC01C501B4010E94C1977B018C01E0
:10392000A50194010E949A9887FD02C047015801A1
:103930001091AC030091AD03F090AE03E090AF03A3
:10394000C501B401212F302F4F2D5E2D0E94A89A62
:10395000181634F4812F902FAF2DBE2D4C015D0130
:1039600040909C0A50909D0A60909E0A70909F0A19
:10397000C301B201A50194010E94A89A1816C4F4CB
:10398000C501B40120E037ED43EA5CE30E947A9B75
:103990007B018C01C301B20128E431EE4AE75FE309
:1039A0000E947A9BA80197010E94C1974B015C017C
:1039B00080929C0A90929D0AA0929E0AB0929F0AC1
:1039C000C501B4010E9409997093A80D6093A70DD9
:1039D000DF91CF911F910F91FF90EF90DF90CF90EB
:1039E000BF90AF909F908F907F906F905F904F901F
:1039F0003F9008956093B8037093B9038093BA031E
:103A00009093BB0308950F931F93CF93DF93C0E070
:103A1000D0E08E010F5A1A4FFE01EB5DFA4F608124
:103A20007181828193810E943A99FE01EB5EFA4F87
:103A300020813181428153810E947A9B0E940E999C
:103A4000F80160837183828393832496C031D1050A
:103A500001F7DF91CF911F910F910895FC016081D3
:103A600071818281938120912105309122054091BD
:103A70002305509124050E947A9B0E944A9B6093E3
:103A80006D0570936E0580936F05909370058DE6BC
:103A900095E00C94A710AF92BF92CF92DF92EF9275
:103AA000FF920F931F93DF93CF93CDB7DEB72C9781
:103AB0000FB6F894DEBF0FBECDBF69837A838B83C8
:103AC0009C832D833E834F835887E986FA860B8734
:103AD0001C8756018DB79EB78A970FB6F8949EBF84
:103AE0000FBE8DBFEDB7FEB731969F0148E853E09A
:103AF00084E2DA010D90AD01D9010D929D01815052
:103B0000C1F7CE01019695A384A3CE01059697A394
:103B100086A3CE01099691A780A70E947531EDB7C3
:103B2000FEB7BA960FB6F894FEBF0FBEEDBF69811F
:103B30007A818B819C8120911505309116054091E9
:103B40001705509118050E947A9B0E944A9B31E606
:103B5000C32E35E0D32E6093610570936205809388
:103B60006305909364056D817E818F819885209196
:103B7000190530911A0540911B0550911C050E94B2
:103B80007A9B0E944A9B24E0E22EF12CEC0CFD1C57
:103B900060936505D70111967C93119712968C93CB
:103BA000129713969C9369857A858B859C852091C5
:103BB0001D0530911E0540911F05509120050E9462
:103BC0007A9B0E944A9B8601085F1F4F609369059C
:103BD000F801718382839383D5016D917D918D91DD
:103BE0009C9120912105309122054091230550910F
:103BF00024050E947A9B0E944A9BF6013C966093A2
:103C00006D05718382839383C601B701A8019F016B
:103C10000E946D1080E090E0A0E0B0E08093840A04
:103C20009093850AA093860AB093870A8093880AA6
:103C30009093890AA0938A0AB0938B0A80938C0A86
:103C400090938D0AA0938E0AB0938F0A8093900A66
:103C50009093910AA093920AB093930A8093940A46
:103C60009093950AA093960AB093970A2C960FB654
:103C7000F894DEBF0FBECDBFCF91DF911F910F91A2
:103C8000FF90EF90DF90CF90BF90AF9008952F926C
:103C90003F924F925F926F927F928F929F92AF92DC
:103CA000BF92CF92DF92EF92FF920F931F93DF9319
:103CB000CF93CDB7DEB7A4970FB6F894DEBF0FBE93
:103CC000CDBF1C0180E00E94CA102B013C0181E0A5
:103CD0000E94CA104B015C0182E00E94CA106B0175
:103CE0007C01C101B301A201950184010E946E30E3
:103CF0008DB79EB784970FB6F8949EBF0FBE8DBF49
:103D0000ADB7BEB71196E8E8F3E084E201900D92FA
:103D10008150E1F78E010F5F1F4FC8010E941732DB
:103D20008DB79EB784960FB6F8949EBF0FBE8DBF19
:103D300084970FB6F8949EBF0FBE8DBFADB7BEB7C8
:103D40001196F80184E201900D928150E1F7C101D2
:103D50000E9488308DB79EB784960FB6F8949EBFA8
:103D60000FBE8DBFC101A4960FB6F894DEBF0FBE83
:103D7000CDBFCF91DF911F910F91FF90EF90DF901A
:103D8000CF90BF90AF909F908F907F906F905F90FB
:103D90004F903F902F9008958F929F92AF92BF9235
:103DA000CF92DF92EF92FF920F931F93CF93DF9307
:103DB000EC016B01009709F45CC08FA9882309F01E
:103DC00058C0EEA0FFA008A519A5FB01B6A0A7A0AA
:103DD00090A481A4C801B7012B2D3A2D492D582D4F
:103DE0000E949A9888230CF044C0C801B701A8012A
:103DF00097010E947A9B7B018C016AA97BA98CA9FF
:103E00009DA9905820E030E040E050EC0E947A9B61
:103E10002EA53FA548A959A90E947A9B9B01AC01F8
:103E2000C801B7010E94C1970E94E79B7B018C01EA
:103E30006B2D7A2D892D982D9701A8010E949A98B3
:103E4000882324F4EB2CFA2C092D182D6B2D7A2DB8
:103E5000892D982D9701A8010E949A98882349F0EE
:103E6000C701D801F60186A397A3A0A7B1A781E057
:103E700086ABDF91CF911F910F91FF90EF90DF9074
:103E8000CF90BF90AF909F908F900895EF92FF9248
:103E90000F931F93CF93DF93F090830A00E010E01D
:103EA00020E030E041E5E42E11C0FE9CE001112449
:103EB000CE58DA4FC901B801AE016EDF8F2D8F5F8A
:103EC000803109F480E0F82E98018E018091820AF9
:103ED000F81659F7C901B80140E050E05DDFDF9105
:103EE000CF911F910F91FF90EF900895AF92BF92E5
:103EF000CF92DF92EF92FF920F931F93CF93DF93B6
:103F0000EB018A016115710509F466C0411551057F
:103F100009F462C0DAA4CBA4BCA4ADA46EA17FA1B5
:103F200088A599A52D2D3C2D4B2D5A2D0E949A9890
:103F3000882309F451C08FA9882309F043C0F801F0
:103F4000E6A0F7A000A511A56D2D7C2D8B2D9A2D37
:103F5000A80197010E94A89A1816A4F5C801B701F4
:103F6000A80197010E947A9B7B018C016AA97BA919
:103F70008CA99DA9905820E030E040E050EC0E94D0
:103F80007A9B2EA53FA548A959A90E947A9B9B011F
:103F9000AC01C801B7010E94C1970E94E79B7B0159
:103FA0008C016D2D7C2D8B2D9A2D9701A8010E94DF
:103FB0009A98882324F4ED2CFC2C0B2D1A2DC70184
:103FC000D80104C08D2D9C2DAB2DBA2D8EA39FA39F
:103FD000A8A7B9A781E08EABDF91CF911F910F9178
:103FE000FF90EF90DF90CF90BF90AF900895CF9269
:103FF000DF92EF92FF920F93DF93CF930F920F9286
:10400000CDB7DEB78091820A8FB7F894F090830A1B
:104010008FBF8091820A90E040968F1991098F702E
:1040200090700497FCF00091820A03500F70CC242A
:10403000DD2440E050E061E5E62E12C0802F002331
:1040400009F480E1082F01500E9DC00111248E5803
:104050009A4F9A838983B60149DFA601C980DA8025
:104060000F1561F70F900F90CF91DF910F91FF9097
:10407000EF90DF90CF900895DF92EF92FF920F9331
:104080001F936091CC0B9091830A8091820A9817BC
:10409000B9F04091830A242F30E081E590E0289F19
:1040A000F001299FF00D389FF00D1124E654FA4FCE
:1040B000608102C04F5F4F708091820A4817D1F72C
:1040C000D62E662331F1E090980AF090990A00917B
:1040D0009A0A10919B0AE114F1040105110579F483
:1040E0000E94A2966C597F4F8F4F9F4F6093980A02
:1040F0007093990A80939A0A90939B0A07C00E9432
:10410000A2966E157F058007910758F4DD24DA9496
:1041100008C01092980A1092990A10929A0A109266
:104120009B0A88E06D2D70E00E947C9588E06D2DE3
:1041300070E00E947C9540DB1F910F91FF90EF9003
:10414000DF9008951092820A1092830A80E1E1E6DE
:10415000F5E0DF011D928A95E9F780E090E0A0E0AC
:10416000B0E08093880A9093890AA0938A0AB0935A
:104170008B0A80938C0A90938D0AA0938E0AB09339
:104180008F0A8093900A9093910AA093920AB09319
:10419000930A8093940A9093950AA093960AB093F9
:1041A000970A8093840A9093850AA093860AB09315
:1041B000870A08952F923F924F925F926F927F925B
:1041C0008F929F92AF92BF92CF92DF92EF92FF9227
:1041D0000F931F93DF93CF93CDB7DEB766970FB6DC
:1041E000F894DEBF0FBECDBF9E8B8D8B6A017B0125
:1041F00048015901DC01D8966D917D918D919C917A
:10420000DB970E943A99698B7A8B8B8B9C8BA701E9
:1042100096010E947A9B0E9487980E940E996D8356
:104220007E838F83988769897A898B899C89A50188
:1042300094010E947A9B0E9487980E940E9969833C
:104240007A838B839C832D813E814F8158852837CB
:1042500031054105510540F448E750E060E070E069
:104260004D835E836F83788769817A818B819C819E
:10427000683771058105910540F488E790E0A0E07A
:10428000B0E089839A83AB83BC83AD89BE89AC5B84
:10429000BF4FAD90BD90CD90DC901397A454B0402B
:1042A000BE8BAD8B6D817E818F8198850E943A99FE
:1042B0006D877E878F87988BC601B5010E943C99D8
:1042C0001B012C0120E030E040E050E00E949A9871
:1042D000882321F4E0E070E060E028C069897A89F1
:1042E0008B899C899B01AC010E947A9B7B018C018C
:1042F0006D857E858F8598899B01AC010E947A9B94
:104300009B01AC01C801B7010E94C0977B018C01E1
:10431000C201B101A20191010E94C1979B01AC01B0
:10432000C801B7010E94A198E62F692F2E2F372FC1
:10433000482F562FB901CA010E9487980E940999F7
:104340003B014C0169817A818B819C810E943A9961
:1043500069877A878B879C8766277727CB016A19BD
:104360007B098C099D090E943C995B016C0120E04E
:1043700030E040E050E00E949A98882321F4E0E089
:1043800070E060E028C069857A858B859C859B01FB
:10439000AC010E947A9B7B018C0169897A898B89A7
:1043A0009C899B01AC010E947A9B9B01AC01C801D6
:1043B000B7010E94C0977B018C01C601B501A6011F
:1043C00095010E94C1979B01AC01C801B7010E94F1
:1043D000A198E62F692F2E2F372F482F562FB9017E
:1043E000CA010E947799ED89FE89A088B188C288A8
:1043F000D38886017501E618F708080919090E9493
:104400000999A8019701261B370B480B590B57FF39
:1044100071C0C201B10120E030E040E050E00E94F4
:104420009A98882321F4E0E070E060E044C0C20183
:10443000B101A20191010E94C1977B018C01C601CB
:10444000B5010E943A999B01AC01C801B7010E94D5
:104450007A9B7B018C016D857E858F8598899B0178
:10446000AC010E947A9B9B01AC01C801B7010E947C
:10447000C0977B018C0169857A858B859C859B0122
:10448000AC010E947A9B9B01AC01C801B7010E945C
:10449000C1977B018C01C201B10120E030E040E80E
:1044A00050E40E947A9B9B01AC01C801B7010E94B5
:1044B000A198E62F692F2E2F372F482F562FB9019D
:1044C000CA010E9487980E940999AC01CB01DA01C8
:1044D0003C014D0197FE03C06624772443016A1412
:1044E0007B048C049D0410F03501460120E030E08F
:1044F00040E050E09FB7F8946D897E89605B7F4F04
:10450000DB018C91A055B040BE8BAD8B882321F58B
:10451000FD01648A758A868A978A260D371D481D93
:10452000591D58962D933D934D935C935B972D8128
:104530003E814F815885DC962D933D934D935C933E
:10454000DF97A05CBF4F29813A814B815C812D931D
:104550003D934D935C9313979FBF66960FB6F89467
:10456000DEBF0FBECDBFCF91DF911F910F91FF90A6
:10457000EF90DF90CF90BF90AF909F908F907F9003
:104580006F905F904F903F902F9008954F925F9261
:104590007F928F929F92AF92BF92CF92DF92EF92D3
:1045A000FF920F931F93CF93DF937090830AC0E025
:1045B000D0E071E5472E512C45C02097A9F18EA976
:1045C000882361F4849CF001859CF00D949CF00D8F
:1045D0001124EE58FA4F86A9882331F1EAA0FBA0F6
:1045E0000CA11DA16EA17FA188A599A5A801970185
:1045F0000E94A1985B016C01849CF001859CF00DE8
:10460000949CF00D1124EE58FA4F66A177A180A575
:1046100091A5A80197010E94A1988B019C01CE0150
:10462000B601A501C7DD1EAA739480E1781609F4CE
:104630007724849CE001859CD00D949CD00D11249E
:10464000CE58DA4F872C992487FC90948091820A67
:1046500090E08816990609F0B0CF2097E9F0EAA01B
:10466000FBA00CA11DA16EA17FA188A599A5A80101
:1046700097010E94A1985B016C016DEC7CEC8CE4CD
:104680009DE3A80197010E94A1988B019C01CE0196
:10469000B601A5018FDD1EAADF91CF911F910F9169
:1046A000FF90EF90DF90CF90BF90AF909F908F9052
:1046B0007F905F904F9008959ADCE8DB67CF2F9250
:1046C0003F924F925F926F927F928F929F92AF92A2
:1046D000BF92CF92DF92EF92FF920F931F93DF93DF
:1046E000CF93CDB7DEB7CA5AD0400FB6F894DEBF2D
:1046F0000FBECDBF69A37AA38BA39CA32DA33EA31A
:104700004FA358A7E9A6FAA60BA71CA78601C9556F
:10471000DF4F8882C75AD040C855DF4F9882C85AA9
:10472000D040C755DF4FA882C95AD040C655DF4F89
:10473000B882CA5AD0408091820A8F5F803109F4D2
:1047400080E0282F332727FD30953CAF2BAF04C0E6
:104750000E949F890E94DE668091830A90E04BADA3
:104760005CAD84179507A1F36DB77EB76A527040B0
:104770000FB6F8947EBF0FBE6DBFEDB7FEB7319692
:104780009F0148E853E084E2DA010D90AD01D901C0
:104790000D929D018150C1F7CE01819695A384A30E
:1047A000CE01859697A386A3CE01899691A780A76F
:1047B0000E9475312091150530911605409117051D
:1047C00050911805CF57DF4F288339834A835B8385
:1047D000C158D0404DB75EB7465D5F4F0FB6F894F5
:1047E0005EBF0FBE4DBFCF57DF4F688179818A8191
:1047F0009B81C158D04029A13AA14BA15CA10E9444
:104800007A9B0E944A9BCF56DF4F6883C159D040A4
:10481000CE56DF4F7883C259D040CD56DF4F8883C4
:10482000C359D040CC56DF4F9883C459D0406091D3
:10483000190570911A0580911B0590911C05C358AC
:10484000DF4F688379838A839B83CD57D0402DA126
:104850003EA14FA158A50E947A9B0E944A9BCB562D
:10486000DF4F6883C559D040CA56DF4F7883C65999
:10487000D040C956DF4F8883C759D040C856DF4F54
:104880009883C859D04080911D0590911E05A09134
:104890001F05B0912005ED968CAF9DAFAEAFBFAFB9
:1048A000ED97BC01CD0129A53AA54BA55CA50E94B9
:1048B0007A9B0E944A9BC756DF4F6883C959D040F4
:1048C000C656DF4F7883CA59D040C556DF4F88831C
:1048D000CB59D040C456DF4F9883CC59D04020915B
:1048E0002105309122054091230550912405E99638
:1048F0002CAF3DAF4EAF5FAFE997CA01B901D80108
:104900002D913D914D915C910E947A9B0E944A9B12
:10491000C356DF4F6883CD59D040C256DF4F7883EE
:10492000CE59D040C156DF4F8883CF59D040C056B2
:10493000DF4F9883C05AD04080916D0590916E05ED
:10494000A0916F05B0917005C356DF4F2881398162
:104950004A815B81CD59D040281739074A075B0748
:1049600009F4B8C0E091CA0BF0E0EE0FFF1FEE0FA4
:10497000FF1FE355F24F6081718182819381209105
:10498000B8033091B9034091BA035091BB030E9420
:104990009A9888230CF033C0C356DF4F4881598161
:1049A0006A817B81CD59D04040936D0550936E054F
:1049B00060936F0570937005E4E7F9E0949108C087
:1049C0008091C00085FFFCCF9093C60031969491F2
:1049D0009923B1F7E8E9F9E0949108C08091C0000B
:1049E00085FFFCCF9093C600319694919923B1F73F
:1049F0008091C00085FFFCCF8AE08093C600809143
:104A00006D0590916E05A0916F05B0917005C3562C
:104A1000DF4F288139814A815B81CD59D040281BE5
:104A2000390B4A0B5B0BCA01B90157FF07C09095C0
:104A30008095709561957F4F8F4F9F4F0E943C9955
:104A40007B018C01E9966CAD7DAD8EAD9FADE99794
:104A500020E030E04FEA53E40E947A9B9B01AC01D6
:104A6000C801B7010E94A89A18160CF033C0C356AB
:104A7000DF4F488159816A817B81CD59D040409375
:104A80006D0550936E0560936F0570937005E4E7B4
:104A9000F9E0949108C08091C00085FFFCCF90930D
:104AA000C600319694919923B1F7EAE7F9E0949121
:104AB00008C08091C00085FFFCCF9093C60031965E
:104AC00094919923B1F78091C00085FFFCCF8AE0D3
:104AD0008093C6008091820A682F70E0E5967FAFD0
:104AE0006EAFE59781E590E0689FF001699FF00D5A
:104AF000789FF00D1124EE58FA4FE05BFF4F1082C3
:104B0000E055F0408091610590916205A0916305A8
:104B1000B0916405E3968CAF9DAFAEAFBFAFE397A6
:104B2000CF56DF4F288139814A815B81C159D040FE
:104B3000281B390B4A0B5B0BAF962CAF3DAF4EAF2A
:104B40005FAFAF97208331834283538357FF0DC0FC
:104B5000DA01C901B095A095909581959F4FAF4F0F
:104B6000BF4F80839183A283B383409165055091A9
:104B700066056091670570916805AB964CAF5DAFB7
:104B80006EAF7FAFAB97CB56DF4F88819981AA81FB
:104B9000BB81C559D040841B950BA60BB70BA796BC
:104BA0008CAF9DAFAEAFBFAFA79781E590E0E59624
:104BB000AEADBFADE597A89FF001A99FF00DB89FDE
:104BC000F00D1124EE58FA4FA7962CAD3DAD4EAD29
:104BD0005FADA797248335834683578357FF0DC066
:104BE000DA01C901B095A095909581959F4FAF4F7F
:104BF000BF4F84839583A683B78340916905509105
:104C00006A0560916B0570916C05A3964CAF5DAF22
:104C10006EAF7FAFA397C756DF4F88819981AA8176
:104C2000BB81C959D040841B950BA60BB70B6F965F
:104C30008CAF9DAFAEAFBFAF6F9781E590E0E596CB
:104C4000AEADBFADE597A89FF001A99FF00DB89F4D
:104C5000F00D1124EE58FA4F6F962CAD3DAD4EADD0
:104C60005FAD6F97208731874287538757FF0DC00D
:104C7000DA01C901B095A095909581959F4FAF4FEE
:104C8000BF4F80879187A287B38740916D05509170
:104C90006E0560916F05709170054DAB5EAB6FABAB
:104CA00078AFC356DF4F88819981AA81BB81CD59E6
:104CB000D040841B950BA60BB70B89AB9AABABAB63
:104CC000BCABE091CA0BF0E0EE0FFF1FEE0FFF1F31
:104CD000EE52FC4F20813181428153816B962CAF83
:104CE0003DAF4EAF5FAF6B974091CE035091CF0376
:104CF00067965FAF4EAF6797BC01CD0197FF07C0C6
:104D000090958095709561957F4F8F4F9F4F0E9432
:104D10003C996B962CAD3DAD4EAD5FAD6B970E944F
:104D20007A9B0E9409996796AEADBFAD67979D01CA
:104D3000442737FD4095542F0E944C9C24E630E0D8
:104D400040E050E00E94B49C81E590E0E5966EADB5
:104D50007FADE597689FF001699FF00D789FF00D9A
:104D60001124EE58FA4FDF011C96248711963C93CC
:104D7000119712964C93129713965C934080518032
:104D800062807380A480B580C680D780E084F1847F
:104D900002851385C901DA018E159F05A007B107A9
:104DA00014F4D801C7018A159B05AC05BD0514F4A0
:104DB000D601C5019C01AD0184159505A605B70571
:104DC00014F4A301920181E590E0E596AEADBFAD8C
:104DD000E597A89FB001A99F700DB89F700D112491
:104DE0006E587A4FFB01208B318B428B538B2630D0
:104DF00031054105510510F40C945430E85BFF4F28
:104E00008091CC0B9091CD0BAA2797FDA095BA2F3E
:104E100080839183A283B383FB01E45BFF4F809186
:104E2000CE0B9091CF0BAA2797FDA095BA2F808328
:104E30009183A283B383DB0190961C92CF56DF4F00
:104E4000288139814A815B81C159D040E3968CAD7C
:104E50009DADAEADBFADE397281739074A075B0795
:104E600024F481E0DB0190968C93CB56DF4F2881B0
:104E700039814A815B81C559D040AB966CAD7DAD1F
:104E80008EAD9FADAB97261737074807590794F4A7
:104E900081E590E0E596AEADBFADE597A89FF00146
:104EA000A99FF00DB89FF00D1124EE58FA4F80A184
:104EB000826080A3C756DF4F288139814A815B8198
:104EC000C959D040A3966CAD7DAD8EAD9FADA39773
:104ED000261737074807590794F481E590E0E596CF
:104EE000AEADBFADE597A89FF001A99FF00DB89FAB
:104EF000F00D1124EE58FA4F80A1846080A3C356B0
:104F0000DF4F288139814A815B81CD59D0406DA91D
:104F10007EA98FA998AD261737074807590794F43B
:104F200081E590E0E596AEADBFADE597A89FF001B5
:104F3000A99FF00DB89FF00D1124EE58FA4F80A1F3
:104F4000886080A381E590E0E5962EAD3FADE597C2
:104F5000289FF001299FF00D389FF00D1124EE5885
:104F6000FA4FC054DF4FA881B981C05CD0408C910A
:104F700081A3408151816281738165964CAF5DAFA1
:104F80006EAF7FAF6597411551056105710509F059
:104F9000179881E590E0E5966EAD7FADE597689F47
:104FA000F001699FF00D789FF00D1124EE58FA4F33
:104FB00064807580868097806114710481049104F7
:104FC00009F0169881E590E0E596AEADBFADE597A6
:104FD000A89FF001A99FF00DB89FF00D1124EE5885
:104FE000FA4FA084B184C284D384A114B104C10453
:104FF000D10409F0159881E590E0E5962EAD3FAD1E
:10500000E597289FF001299FF00D389FF00D11249E
:10501000EE58FA4F84859585A685B7850097A1053A
:10502000B10551F014982090350530903605409028
:1050300037055090380508C020904D0530904E053A
:1050400040904F0550905005C955DF4F6881C75AB1
:10505000D040C855DF4F7881C85AD040C755DF4F80
:105060008881C95AD040C655DF4F9881CA5AD0406E
:10507000A20191010E949A9887FD16C0C955DF4F81
:105080008881C75AD040C855DF4F9881C85AD04050
:10509000C755DF4FA881C95AD040C655DF4FB881E8
:1050A000CA5AD0401C012D01AF966CAD7DAD8EADBE
:1050B0009FADAF970E943C99CF57DF4F2881398130
:1050C0004A815B81C158D0400E94A198C357DF4FED
:1050D0006883CD58D040C257DF4F7883CE58D04038
:1050E000C157DF4F8883CF58D040C057DF4F9883D8
:1050F000C059D040AC01CB01DA0189839A83AB83DC
:10510000BC83A7966CAD7DAD8EAD9FADA7970E9479
:105110003C99C358DF4F288139814A815B81CD5743
:10512000D0400E94A198C757DF4F6883C958D0402C
:10513000C657DF4F7883CA58D040C557DF4F8883A2
:10514000CB58D040C457DF4F9883CC58D040AC01E7
:10515000CB01DA018D839E83AF83B8876F966CADE8
:105160007DAD8EAD9FAD6F970E943C99ED962CADB5
:105170003DAD4EAD5FADED970E94A198CB57DF4F8F
:105180006883C558D040CA57DF4F7883C658D0408F
:10519000C957DF4F8883C758D040C857DF4F98831F
:1051A000C858D040AC01CB01DA0189879A87AB8718
:1051B000BC8769A97AA98BA99CA90E943C99E99608
:1051C0002CAD3DAD4EAD5FADE9970E94A1986B96B9
:1051D0002CAD3DAD4EAD5FAD6B970E947A9B7B01D0
:1051E0008C0167964EAD5FAD6797BA01882777FD52
:1051F0008095982F0E943C999B01AC01C801B70192
:105200000E947A9B20E030E048EC52E40E94A19892
:105210009B01AC016D877E878F87988B65966CADFF
:105220007DAD8EAD9FAD65976630710581059105A9
:105230001CF576E06716710481049104ECF486E0B5
:10524000A816B104C104D104BCF481E590E0E59650
:10525000AEADBFADE597A89FF001A99FF00DB89F37
:10526000F00D1124EE58FA4FDA01C901BF7786A775
:1052700097A7A0ABB1AB6DC0C357DF4F2881CD5806
:10528000D040C257DF4F3881CE58D040C157DF4F92
:105290004881CF58D040C057DF4F5881C059D040C7
:1052A000B901CA010E94319C3B014C01C757DF4F35
:1052B0002881C958D040C657DF4F3881CA58D040DE
:1052C000C557DF4F4881CB58D040C457DF4F588176
:1052D000CC58D040B901CA010E94319C5B016C01DD
:1052E000CB57DF4F2881C558D040CA57DF4F388190
:1052F000C658D040C957DF4F4881C758D040C8571B
:10530000DF4F5881C858D040B901CA010E94319C72
:105310007B018C01C401B301A60195010E94C197D4
:10532000A80197010E94C1970E94E79B21E530E008
:10533000E5964EAD5FADE597429FF001439FF00DBE
:10534000529FF00D1124EE58FA4F66A777A780AB55
:1053500091AB81E590E0E5966EAD7FADE597689FF6
:10536000F001699FF00D789FF00D1124EE58FA4F6F
:1053700086A597A5A0A9B1A961968CAF9DAFAEAF48
:10538000BFAF619760E070E080E89FE361962CAD6D
:105390003DAD4EAD5FAD61970E94A1989B01AC0100
:1053A000C201B1010E947A9B2B013C018091820ACB
:1053B0009091830AA82FB0E05096A91BB109AF7055
:1053C000B070BAAFA9AFA230B1050CF451C05D0105
:1053D000CC24B7FCC094DC2CC601B5010E943C99DA
:1053E00020E030E040E051E40E949A9888230CF0DD
:1053F0003FC060E074E284E799E4A30192010E9457
:10540000A1980E944A9B7B018C01609101057091DB
:1054100002058091030590910405E616F70608073A
:10542000190730F56E197F09800B910B660F771FF6
:10543000881F991FA60195010E94929CCA01B9017B
:105440000E943A990E944A9B9B01AC012E0D3F1D80
:10545000401F511FCA01B9010E943A999B01AC013A
:1054600060E074E284E799E40E94A1982B013C017A
:1054700081E590E0E596EEADFFADE597E89F800110
:10548000E99F100DF89F100D11240E581A4F6196C8
:105490006CAD7DAD8EAD9FAD6197A30192010E9471
:1054A0007A9BD80192966D937D938D939C9395975B
:1054B00050966D917D918D919C9153970E943A9950
:1054C000A30192010E947A9B0E9487980E940E99E4
:1054D000F80160AF71AF82AF93AFCF55DF4F188245
:1054E000C15AD040CE55DF4F1882C25AD04020E872
:1054F000222E9FE3392E88249924E1E0F0E0EC0F7E
:10550000FD1FE80DF91DC301B201208131814281E7
:1055100053810E947A9BE1E1F0E0EC0FFD1FE80D62
:10552000F91D60837183828393835B016C01E8942E
:10553000D7F8F401EB5FFA4FE080F180028113812C
:10554000C601B501A80197010E94A89A1816CCF4CB
:10555000C801B701A60195010E94A1986B017C01C9
:10556000CF55DF4F6881C15AD040CE55DF4F78818B
:10557000C25AD040C101A70196010E949A9888237F
:105580006CF4CF55DF4F8881C15AD040CE55DF4FE4
:105590009881C25AD040D1016C017D0124E030E0F5
:1055A000820E931E30E18316910471F0D701C6017B
:1055B000CF55DF4FC882C15AD040CE55DF4F9883B8
:1055C000C25AD0401D0199CFC701B60120E030E09A
:1055D00040E85FE30E949A9888230CF04CC08E014B
:1055E0000F5E1F4F81E2A82EB12CAC0EBD1ED8015C
:1055F0006D917D918D919C91A70196010E947A9B5E
:10560000F80161937193819391938F01EA15FB05E2
:1056100071F781E590E0E5962EAD3FADE597289FC7
:105620008001299F100D389F100D11240E581A4F1C
:10563000D80192966D917D918D919C919597A7013E
:1056400096010E947A9BF80162A373A384A395A399
:1056500060AD71AD82AD93AD0E943A99A7019601FC
:105660000E947A9B0E940E99D801D8966D937D93E3
:105670008D939C93DB9781E590E0E596EEADFFADD1
:10568000E597E89F8001E99F100DF89F100D112408
:105690000E581A4FD80150966D917D918D919C9125
:1056A00053970E943A99F80126A537A540A951A918
:1056B0000E94A1981B012C01F80180819181A28197
:1056C000B3810097A105B10549F584819581A68133
:1056D000B7810097A105B10509F580859185A2855F
:1056E000B3850097A105B105C9F4C201B1012091AC
:1056F0003D0530913E0540913F05509140050E9487
:105700007A9B0E9487980C5B1F4F0E940E99D801CC
:105710006D937D938D939C93139771C1C201B101D9
:105720002091390530913A0540913B0550913C0557
:105730000E947A9B0E9487980E940E9921E530E092
:10574000E596EEADFFADE597E29F6001E39FD00CDB
:10575000F29FD00C112422E735E0C20ED31EB4E430
:105760006B2E712C6C0C7D1CD3016D937D938D93EE
:105770009C9313978090510590905205A0905305EB
:10578000B09054050E943A997B018C01F60160812A
:105790007181828193810E943C999B01AC01C80177
:1057A000B7010E947A9B7B018C01D60150966D91C6
:1057B0007D918D919C9153970E943A999B01AC01E8
:1057C000C801B7010E94A1987B018C01C501B401F9
:1057D0000E943A999B01AC01C801B7010E94A89AA6
:1057E00018162CF4F30180829182A282B3828090F9
:1057F000550590905605A0905705B090580581E545
:1058000090E0E5962EAD3FADE597289F6001299F7A
:10581000D00C389FD00C112442E755E0C40ED51EA1
:10582000A4E46A2E712C6C0C7D1CD3016D917D91CA
:105830008D919C910E943A997B018C01F6016481C3
:105840007581868197810E943C999B01AC01C801BA
:10585000B7010E947A9B7B018C01D60150966D9115
:105860007D918D919C9153970E943A999B01AC0137
:10587000C801B7010E94A1987B018C01C501B40148
:105880000E943A999B01AC01C801B7010E94A89AF5
:1058900018162CF4F30180829182A282B382809048
:1058A0005D0590905E05A0905F05B090600581E574
:1058B00090E0E5962EAD3FADE597289F6001299FCA
:1058C000D00C389FD00C112442E755E0C40ED51EF1
:1058D000F4E46F2E712C6C0C7D1CD3016D917D91C5
:1058E0008D919C910E943A997B018C01F60164850F
:1058F0007585868597850E943C999B01AC01C801FE
:10590000B7010E947A9B7B018C01D60150966D9164
:105910007D918D919C9153970E943A999B01AC0186
:10592000C801B7010E94A1987B018C01C501B40197
:105930000E943A999B01AC01C801B7010E94A89A44
:1059400018162CF4F30180829182A282B382809097
:10595000590590905A05A0905B05B0905C0581E5D3
:1059600090E0E5962EAD3FADE597289F6001299F19
:10597000D00C389FD00C112442E755E0C40ED51E40
:10598000E4E46E2E712C6C0C7D1CD3016D917D9125
:105990008D919C910E943A997B018C01F601608562
:1059A0007185828593850E943C999B01AC01C80159
:1059B000B7010E947A9B7B018C01D60150966D91B4
:1059C0007D918D919C9153970E943A999B01AC01D6
:1059D000C801B7010E94A1987B018C01C501B401E7
:1059E0000E943A999B01AC01C801B7010E94A89A94
:1059F00018162CF4F30180829182A282B38281E591
:105A000090E0E5962EAD3FADE597289F6001299F78
:105A1000D00C389FD00C112442E755E0C40ED51E9F
:105A2000F601EC5BFF4F60817181828193810E945E
:105A30003A997B018C01A20191010E94A198D601A3
:105A4000D2966D937D938D939C93D597C801B701A2
:105A50002DEB37E346E051E40E947A9B0E940999BE
:105A6000F601648F758F868F978F609041057090D7
:105A700042058090430590904405C401B30120E0A5
:105A800030E040E05FE30E947A9B5B016C01298D6E
:105A90003A8D4B8D5C8D2D962CAF3DAF4EAF5FAFE9
:105AA0002D974091450550914605609147057091AD
:105AB000480529964CAF5DAF6EAF7FAF2997CB01FC
:105AC000BA0120E030E040E05FE30E947A9B7B0176
:105AD0008C012D966CAD7DAD8EAD9FAD2D979F77D2
:105AE000A80197010E94A89A181644F4C601B501AE
:105AF000A80197010E949A98882314F486017501E1
:105B00006D8D7E8D8F8D98A125966CAF7DAF8EAFFC
:105B10009FAF25978091490590914A05A0914B052B
:105B2000B0914C0521968CAF9DAFAEAFBFAF219722
:105B3000BC01CD0120E030E040E05FE30E947A9BB1
:105B40001B012C0125966CAD7DAD8EAD9FAD2597CB
:105B50009F77A20191010E94A89A181644F4C801E7
:105B6000B701A20191010E949A98882314F41701A9
:105B7000280181E590E0E596AEADBFADE597A89F21
:105B8000F001A99FF00DB89FF00D1124EE58FA4FC7
:105B900022A133A144A155A12DA73EA74FA758ABE1
:105BA000C201B1010E949A9887FD04C02DA43EA4B1
:105BB0004FA458A849AD5AAD423051050CF411C15B
:105BC0005091840ACD55DF4F5883C35AD04060911D
:105BD000850ACC55DF4F6883C45AD0407091860A3D
:105BE000CB55DF4F7883C55AD0408091870ACA557C
:105BF000DF4F8883C65AD040652FCC55DF4F788160
:105C0000C45AD040CB55DF4F8881C55AD040CA55C1
:105C1000DF4F9881C65AD04027E137EB41ED58E37A
:105C20000E94A89A18160CF0DCC069897A898B89C1
:105C30009C892091880A3091890A40918A0A509162
:105C40008B0A0E94C0979B01AC010E947A9B7B014A
:105C50008C016D897E898F89988D20918C0A309175
:105C60008D0A40918E0A50918F0A0E94C0979B0125
:105C7000AC010E947A9B9B01AC01C801B7010E9454
:105C8000C1970E94E79B7B018C01A40193010E94B4
:105C9000A89A18165CF00F2EF0E06F2EF0E07F2E21
:105CA000F0E88F2EFFE39F2EF02D08C0C401B30152
:105CB000A80197010E94A1983B014C012D966CAD63
:105CC0007DAD8EAD9FAD2D972091900A3091910AB8
:105CD0004091920A5091930A0E94C0977B018C01D7
:105CE000E89417F9C801B70129962CAD3DAD4EAD2A
:105CF0005FAD29970E94A89A1816A4F429966CAD56
:105D00007DAD8EAD9FAD2997A80197010E94A19806
:105D10005B016C01C401B301A60195010E949A9830
:105D2000882314F46401530125966CAD7DAD8EADCE
:105D30009FAD25972091940A3091950A4091960A3B
:105D40005091970A0E94C0977B018C01E89417F943
:105D5000C801B70121962CAD3DAD4EAD5FAD219789
:105D60000E94A89A1816A4F421966CAD7DAD8EAD54
:105D70009FAD2197A80197010E94A1987B018C01FA
:105D8000C601B501A80197010E949A98882314F4CE
:105D9000860175016DA57EA58FA598A9A80197011B
:105DA0000E947A9B7B018C01CD55DF4F6881C35ADD
:105DB000D040CC55DF4F7881C45AD040CB55DF4F0F
:105DC0008881C55AD040CA55DF4F9881C65AD04005
:105DD000A80197010E949A9887FD19C0D801C701B0
:105DE00002C0D201C101CD55DF4F8883C35AD040D4
:105DF000CC55DF4F9883C45AD040CB55DF4FA88392
:105E0000C55AD040CA55DF4FB883C65AD04081E545
:105E100090E0E596AEADBFADE597A89F8001A99F44
:105E2000100DB89F100D11240E581A4FCD55DF4F8D
:105E30008881C35AD040CC55DF4F9881C45AD04096
:105E4000CB55DF4FA881C55AD040CA55DF4FB88126
:105E5000C65AD040F80182A793A7A4A7B5A762A904
:105E600073A984A995A9905820E030E040E050EC57
:105E70000E947A9BD8019E962D913D914D915C9107
:105E8000D1970E947A9B2BE037ED43E25BE30E94BF
:105E9000C1970E94E79BF62EE72ED82EC92ECD552E
:105EA000DF4F6881C35AD040CC55DF4F7881C45A48
:105EB000D040CB55DF4F8881C55AD040CA55DF4FFF
:105EC0009881C65AD0402F2D3E2D4D2D5C2D0E941D
:105ED0009A9887FD14C0CD55DF4FF882C35AD04041
:105EE000CC55DF4FE882C45AD040CB55DF4FD88223
:105EF000C55AD040CA55DF4FC882C65AD04081E546
:105F000090E0E596EEADFFADE597E89F8001E99F53
:105F1000100DF89F100D11240E581A4FCD55DF4F5C
:105F20008881C35AD040CC55DF4F9881C45AD040A5
:105F3000CB55DF4FA881C55AD040CA55DF4FB88135
:105F4000C65AD040F80186A397A3A0A7B1A762A123
:105F500073A184A195A12F2D3E2D4D2D5C2D0E9466
:105F60009A9818162CF081E0D801D7968C9302C02D
:105F7000F80117AA81E590E0E5962EAD3FADE597D3
:105F8000289FF001299FF00D389FF00D1124EE5845
:105F9000FA4F81E086ABA8E8BAE0FE01719680E195
:105FA00001900D928150E1F781E590E0E5964EADCC
:105FB0005FADE597489F6001499FD00C589FD00C7A
:105FC000112462E775E0C60ED71ED6019296ED90B9
:105FD000FD900D911C919597E092840AF092850AAC
:105FE0000093860A1093870A96966D917D918D9104
:105FF0009C919997A80197010E94A1984B015C017F
:10600000C201B101A80197010E94A1988B019C01D6
:10601000C601B501A4010E94DA20BBADB093820A8B
:10602000C356DF4F288139814A815B81CD59D040E9
:1060300020936D0530936E0540936F055093700566
:10604000C756DF4F488159816A817B81C959D04049
:106050004093690550936A0560936B0570936C05D6
:10606000CB56DF4F688179818A819B81C559D040A9
:106070006093650570936605809367059093680546
:10608000CF56DF4F88819981AA81BB81C159D04009
:106090008093610590936205A0936305B0936405B6
:1060A0000E945C230E946710C655DF4F0FB6F8941C
:1060B000DEBF0FBECDBFCF91DF911F910F91FF903B
:1060C000EF90DF90CF90BF90AF909F908F907F9098
:1060D0006F905F904F903F902F900895CF92DF92F6
:1060E000EF92FF920F931F93FC01408351836283D1
:1060F00073830483158326833783C086D186E28623
:10610000F3861F910F91FF90EF90DF90CF9008954D
:106110002F923F924F925F926F927F928F929F92B7
:10612000AF92BF92CF92DF92EF92FF920F931F93A5
:10613000DF93CF93CDB7DEB72A970FB6F894DEBFC3
:106140000FBECDBF9A878987DC012D903D904D9081
:106150005C90139714968D919D910D90BC91A02DFC
:106160008D839E83AF83B887A985BA8518968D9154
:106170009D910D90BC91A02D89839A83AB83BC83A4
:10618000C201B1012CA13DA14EA15FA10E947A9B49
:106190007B018C016D817E818F81988528A939A929
:1061A0004AA95BA90E947A9B9B01AC01C801B70177
:1061B0000E94C1977B018C0169817A818B819C81CE
:1061C0002CAD3DAD4EAD5FAD0E947A9B9B01AC0105
:1061D000C801B7010E94C1973B014C01C201B10146
:1061E00028A539A54AA55BA50E947A9B7B018C0155
:1061F0006D817E818F8198852CA93DA94EA95FA9CB
:106200000E947A9B9B01AC01C801B7010E94C19713
:106210007B018C0169817A818B819C8124962CADD4
:106220003DAD4EAD5FAD24970E947A9B9B01AC01C2
:10623000C801B7010E94C1975B016C01C201B101A5
:1062400028A139A14AA15BA10E947A9B7B018C0104
:106250006D817E818F8198852CA53DA54EA55FA57A
:106260000E947A9B9B01AC01C801B7010E94C197B3
:106270007B018C0169817A818B819C8128AD39AD4C
:106280004AAD5BAD0E947A9B9B01AC01C801B7018E
:106290000E94C197E985FA85608371838283938325
:1062A000C301D40184839583A683B783C501D60136
:1062B00080879187A287B3872A960FB6F894DEBFAE
:1062C0000FBECDBFCF91DF911F910F91FF90EF9047
:1062D000DF90CF90BF90AF909F908F907F906F9006
:1062E0005F904F903F902F900895EF92FF920F9301
:1062F0001F93DF93CF93CDB7DEB72C970FB6F894EB
:10630000DEBF0FBECDBFECADFDAD80819181A2811E
:10631000B381EEADFFADE080F18002811381EAAD83
:10632000FBAD208131814281538129833A834B83A4
:106330005C838D839E83AF83B887E986FA860B875B
:106340001C878DB79EB784970FB6F8949EBF0FBE7B
:106350008DBFADB7BEB71196FE01769684E201906F
:106360000D928150E1F7CE010196D2DE89819A81AA
:10637000AB81BC81EAADFBAD80839183A283B38303
:106380008D819E81AF81B885ECADFDAD8083918319
:10639000A283B38389859A85AB85BC85EEADFFADBD
:1063A00080839183A283B3838DB79EB784960FB603
:1063B000F8949EBF0FBE8DBF2C960FB6F894DEBF2B
:1063C0000FBECDBFCF91DF911F910F91FF90EF9046
:1063D0000895FC0120E030E040E85FE32083318352
:1063E0004283538380E090E0A0E0B0E08483958313
:1063F000A683B78380879187A287B3878487958791
:10640000A687B787208B318B428B538B848B958BE0
:10641000A68BB78B808F918FA28FB38F848F958F30
:10642000A68FB78F20A331A342A353A308952F9221
:106430003F924F925F926F927F928F929F92AF9214
:10644000BF92CF92DF92EF92FF920F931F93DF9351
:10645000CF93CDB7DEB72C970FB6F894DEBF0FBE43
:10646000CDBFFC012EA53FA548A959A9EAACFBACBC
:106470000CAD1DADAEA0BFA0C8A4D9A46AA87BA8CE
:106480008CA89DA822962CAC3DAC4EAC5FAC22975C
:106490008AA59BA5ACA5BDA589879A87AB87BC8734
:1064A0008EA99FA9A8ADB9AD8D839E83AF83B88710
:1064B00026968CAD9DADAEADBFAD269789839A83F0
:1064C000AB83BC838AA19BA1ACA1BDA18083918336
:1064D000A283B3832483358346835783E086F18682
:1064E00002871387A486B586C686D786608A718A96
:1064F000828A938A248A358A468A578A89859A8528
:10650000AB85BC85808F918FA28FB38F8D819E814B
:10651000AF81B885848F958FA68FB78F89819A8137
:10652000AB81BC8180A391A3A2A3B3A3CF012C967E
:106530000FB6F894DEBF0FBECDBFCF91DF911F9194
:106540000F91FF90EF90DF90CF90BF90AF909F9012
:106550008F907F906F905F904F903F902F90089515
:10656000CF93DF93EC01FB0107C08091C00085FF52
:10657000FCCF31969093C60090819923B1F7E2EC5D
:10658000F9E0949108C08091C00085FFFCCF909302
:10659000C600319694919923B1F7488159816A8157
:1065A0007B8184E99BE022E030E00E944D51EDEBDD
:1065B000F9E0949108C08091C00085FFFCCF9093D2
:1065C000C600319694919923B1F74C815D816E811B
:1065D0007F8184E99BE022E030E00E944D51E8EBAE
:1065E000F9E0949108C08091C00085FFFCCF9093A2
:1065F000C600319694919923B1F7488559856A85EB
:106600007B8584E99BE022E030E00E944D51E6EB7F
:10661000F9E0949108C08091C00085FFFCCF909371
:10662000C600319694919923B1F7DF91CF910895E7
:106630006F927F928F929F92AF92BF92CF92DF9292
:10664000EF92FF920F931F93FC01208131814281D1
:106650005381E480F580068117816084718482848F
:106660009384CA01B9010E947A9B5B016C01C80145
:10667000B701A80197010E947A9B9B01AC01C6015A
:10668000B5010E94C1977B018C01C401B301A40133
:1066900093010E947A9B9B01AC01C801B7010E9443
:1066A000C1970E94E79B1F910F91FF90EF90DF90A1
:1066B000CF90BF90AF909F908F907F906F900895F4
:1066C000CF92DF92EF92FF920F931F938C01B0DF76
:1066D0006B017C01F8016081718182819381A70146
:1066E00096010E94A198F80160837183828393834D
:1066F0006481758186819781A70196010E94A19886
:10670000F8016483758386839783608571858285AC
:106710009385A70196010E94A198F801608771876F
:10672000828793871F910F91FF90EF90DF90CF901A
:106730000895CF92DF92EF92FF920F931F938C01F7
:10674000FB012481358146815781C084D184E28454
:10675000F38480819181A281B381F8018083918348
:10676000A283B3832483358346835783C086D1862F
:10677000E286F386C801A4DFC8011F910F91FF9044
:10678000EF90DF90CF9008952F923F924F925F92BB
:106790006F927F928F929F92AF92BF92CF92DF9231
:1067A000EF92FF920F931F93DF93CF93CDB7DEB796
:1067B000C655D0400FB6F894DEBF0FBECDBF67966A
:1067C0009FAF8EAF6797CDAEDEAEEFAEFE01E05C61
:1067D000FF4FF082E1E46E2E712C6C0E7D1ED30112
:1067E0000C93FE01EE5BFF4F1083FE01ED5BFF4F4C
:1067F0002083FE01EC5BFF4F308395E4892E912CC2
:106800008C0E9D1EF4014083FE01EA5BFF4F508316
:10681000FE01E95BFF4F6083FE01E85BFF4F708381
:106820008E01035C1F4FCE010196B80182DFD801B3
:106830006D917D918D919C919058F40120813181D1
:10684000428153810E94A1980F2EF0E0AF2EF0E01C
:10685000BF2EF0E8CF2EFFE3DF2EF02DA98EBA8EEB
:10686000CB8EDC8E0F2EF0E0EF2EF0E0FF2EF0E06E
:106870000F2FF0E01F2FF02DED8EFE8E0F8F18A33F
:10688000AC01CB01DA0189A39AA3ABA3BCA3CE01CF
:106890000D96BE01675E7F4F4CDFD3016D917D91F8
:1068A0008D919C919058F4012081318142815381D6
:1068B0000E94A198E9AAFAAA0BAB1CABADAABEAA8A
:1068C000CFAAD8AEAC01CB01DA0189AF9AAFABAF9A
:1068D000BCAFCE018596BE016F5C7F4F2ADF298950
:1068E0003A894B895C89ED88FE880F89188DADA0A7
:1068F000BEA0CFA0D8A469A47AA48BA49CA42DA4E4
:106900003EA44FA458A889819A81AB81BC81659629
:106910008CAF9DAFAEAFBFAF65978D819E81AF81CC
:10692000B88561968CAF9DAFAEAFBFAF61978985DB
:106930009A85AB85BC852D968CAF9DAFAEAFBFAFB2
:106940002D978D859E85AF85B8896796EEADFFAD95
:10695000679780839183A283B3832483358346839F
:106960005783E086F18602871387A486B586C6869C
:10697000D786608A718A828A938A248A358A468A6F
:10698000578A65968CAD9DADAEADBFAD6597808FD6
:10699000918FA28FB38F61968CAD9DADAEADBFAD23
:1069A0006197848F958FA68FB78F2D968CAD9DADF7
:1069B000AEADBFAD2D9780A391A3A2A3B3A3CF018A
:1069C000CA5ADF4F0FB6F894DEBF0FBECDBFCF91CE
:1069D000DF911F910F91FF90EF90DF90CF90BF90CC
:1069E000AF909F908F907F906F905F904F903F906F
:1069F0002F9008952F923F924F925F926F927F92C5
:106A00008F929F92AF92BF92CF92DF92EF92FF92BE
:106A10000F931F93DF93CF93CDB7DEB7CD55D04003
:106A20000FB6F894DEBF0FBECDBF2F969FAF8EAFCF
:106A30002F9761967FAF6EAF61972A0162962FAF55
:106A4000629763960FAF63976496EFAE649768960C
:106A5000ACAEBDAECEAEDFAE6897E22EFF24EE0C3C
:106A6000FF1CEE0CFF1C9A012E0D3F1D2D963FAF13
:106A70002EAF2D97D9016D907D908D909C90FC014B
:106A8000EE0DFF1DC401B30120813181428153818C
:106A90000E94C19769AF7AAF8BAF9CAF10E0000F37
:106AA000111F000F111FF201E00FF11F2B96FFAF16
:106AB000EEAF2B97A080B180C280D3802F96EEAD31
:106AC000FFAD2F97E00FF11FC601B5012081318185
:106AD000428153810E94C1976DAB7EAB8FAB98AF63
:106AE00064962FAD6497E22FF0E0EE0FFF1FEE0FDC
:106AF000FF1F2F96AEADBFAD2F97AE0FBF1F2D91CD
:106B00003D914D915C9129962CAF3DAF4EAF5FAF5B
:106B1000299761964EAD5FAD6197E40FF51F6081D7
:106B200071818281938129962CAD3DAD4EAD5FADD3
:106B300029970E94C09769AB7AAB8BAB9CAB6196EF
:106B4000AEADBFAD61971C968D919D910D90BC919E
:106B5000A02D25968CAF9DAFAEAFBFAF25972F96DA
:106B6000AEADBFAD2F971C962D913D914D915C918F
:106B70001F9721962CAF3DAF4EAF5FAF2197A40179
:106B8000930150582DA73EA74FA758ABD601C5017A
:106B9000B05889A79AA7ABA7BCA76196AEADBFAD09
:106BA0006197EA0EFB1EF7016081718182819381FA
:106BB00029AD3AAD4BAD5CAD0E94C0973B014C0195
:106BC00061962EAD3FAD6197020F131FD8016D91F5
:106BD0007D918D919C912DA93EA94FA958AD0E9400
:106BE000C0975B016C016DA57EA58FA598A9A60134
:106BF00095010E947A9B7B018C0169A57AA58BA5E2
:106C00009CA5A40193010E947A9B9B01AC01C80141
:106C1000B7010E94C0971B012C016DA57EA58FA511
:106C200098A9A40193010E947A9B7B018C0169A51C
:106C30007AA58BA59CA5A60195010E947A9B9B0134
:106C4000AC01C801B7010E94C1979B01AC01C20110
:106C5000B1010E9434985B016C0120E030E040E01B
:106C600050E00E949A98882354F4C601B5012BED98
:106C70003FE049EC50E40E94C1975B016C01E8964B
:106C80008FADE897882351F0C601B5012BED3FE0A9
:106C900049EC50E40E94C0975B016C01C601B5014C
:106CA000E7962CAD3DAD4EAD5FADE7970E947A9B68
:106CB00029A93AA94BA95CA95F770E94B59A7B01E3
:106CC0008C012FE632E143E85AE30E949A9887FD4F
:106CD00010C2C801B7010E9477990E940E9978A747
:106CE0006FA3672B21F4E1E0F0E0F8A7EFA32FA159
:106CF00038A5B90180E090E00E943A997B018C01AF
:106D0000C601B501A80197010E94A1986BA37CA3BD
:106D10008DA39EA369A97AA98BA99CA9A801970113
:106D20000E94A1986F8F78A389A39AA325966CAD32
:106D30007DAD8EAD9FAD259721962CAD3DAD4EAD71
:106D40005FAD21970E94C097A80197010E94A1986A
:106D50006B8F7C8F8D8F9E8F6BA17CA18DA19EA14F
:106D600020E030E040E05FEB0E947A9B2BA13CA149
:106D70004DA15EA10E947A9B20E030E040E85FE3F5
:106D80000E94C1976F8B788F898F9A8F64963FADE1
:106D90006497E32FF0E0EE0FFF1FEE0FFF1F9E0141
:106DA0002F5F3F4FE20FF31F29968CAD9DADAEAD27
:106DB000BFAD299780839183A283B3832F96AEAD15
:106DC000BFAD2F971C964D915D916D917C911F9752
:106DD0004D875E876F87788B41E050E05A8B498BF7
:106DE000662462969FAD6297892F90E0880F991F65
:106DF000880F991FD901A80FB91F6A96BFAFAEAF10
:106E00006A9763963FAD6397232F30E0220F331FBD
:106E1000220F331F4C0F5D1F420F531F6C965FAF45
:106E20004EAF6C976E96FFAFEEAF6E9727C158E1ED
:106E300056150CF446C06DA57EA58FA598A92BA16B
:106E40003CA14DA15EA10E947A9B7B018C0169A5AA
:106E50007AA58BA59CA52F89388D498D5A8D0E94C6
:106E60007A9B9B01AC01C801B7010E94C1977B01CD
:106E70008C016DA57EA58FA598A92F89388D498D88
:106E80005A8D0E947A9B5B016C0169A57AA58BA53E
:106E90009CA52BA13CA14DA15EA10E947A9B9B01C8
:106EA000AC01C601B5010E94C0976DA77EA78FA750
:106EB00098AB6394C701D80189A79AA7ABA7BCA7D1
:106EC00065C0A989BA89BD0180E090E00E943A9925
:106ED0002BA13CA14DA15EA10E947A9B7B018C015C
:106EE000C8010E949E986B8B7C8B8D8B9E8BB7010B
:106EF000C8010E94DD9B3B014C012D96EEADFFAD1C
:106F00002D97E080F1800281138117FB109517F90E
:106F100010952B96AEADBFAD2B972D903D904D901B
:106F20005C90C801B7012B893C894D895E890E941C
:106F30007A9B5B016C01C201B101A40193010E9423
:106F40007A9B9B01AC01C601B5010E94C1976DA758
:106F50007EA78FA798ABC801B701A40193010E9437
:106F60007A9B7B018C01C201B1012B893C894D893F
:106F70005E890E947A9B9B01AC01C801B7010E9407
:106F8000C09769A77AA78BA79CA7662469AD7AAD3D
:106F90008BAD9CAD2DA53EA54FA558A90E94C197CC
:106FA0006A96EEADFFAD6A976083718382839383A7
:106FB0006DA97EA98FA998AD29A53AA54BA55CA579
:106FC0000E94C1976C96AEADBFAD6C976D937D93EB
:106FD0008D939C9313976E96EEADFFAD6E97608187
:106FE0007181828193812F8D38A149A15AA10E947C
:106FF000C1976E96AEADBFAD6E976D937D938D9339
:107000009C9313976D857E858F8598892B8D3C8DFC
:107010004D8D5E8D0E94C1976D877E878F87988B7F
:10702000CE0101960E94575A0F920F9269817A8180
:107030008B819C812D813E814F815885E984FA8422
:107040000B851C85A8E7B0E0AC0FBD1FEDB7FEB700
:10705000B283A183EDE0CE2ED12CCC0EDD1E68963E
:107060008CAC9DACAEACBFAC68970E945F23E98945
:10707000FA893196FA8BE98B0F900F9029893A891A
:107080004FA158A52417350708F4D1CE0F920F92BF
:107090006196AEADBFAD61976D917D918D919C91E3
:1070A000139714962D913D914D915C9117971896D9
:1070B000ED90FD900D911C911B971C966196BFAFB2
:1070C000AEAF6197FE01E858FF4FADB7BEB712965D
:1070D000FC93EE9311976196CEACDFAC6197689606
:1070E0008CAC9DACAEACBFAC68970E945F230F9098
:1070F0000F90C35ADF4F0FB6F894DEBF0FBECDBF5F
:10710000CF91DF911F910F91FF90EF90DF90CF9083
:10711000BF90AF909F908F907F906F905F904F90B7
:107120003F902F900895FC018091A00A843290F442
:1071300080838F5F8093A00A815090E0FC01EE0F66
:10714000FF1FE80FF91FEF55F54F88EB9BE0928387
:10715000818308958FEF80830895FC01208124327C
:10716000B8F58181992787FD909548E850E0481B44
:10717000590B440F551F440F551F6417750784F0B2
:107180008281992787FD909548E552E0481B590B6D
:10719000440F551F440F551F641775070CF4AB01BE
:1071A00042505040CA01AA2797FDA095BA2F880FD8
:1071B000991FAA1FBB1F4FB7F89430E0F901EE0FDB
:1071C000FF1FE20FF31FEF55F54F928381834FBFEF
:1071D0000895FC0180818F3F19F420E030E016C053
:1071E00090E0FC01EE0FFF1FE80FF91FEF55F54F80
:1071F0002181328183E0220F331F8A95E1F7B4E0C9
:1072000036952795BA95E1F72E5F3F4FC90108954E
:10721000AF92BF92CF92DF92EF92FF920F931F93A4
:107220008C01D7DF00D00F920196AA2797FDA09579
:10723000BA2FF8016181772767FD709528E830E063
:10724000261B370B220F331F220F331F442737FD16
:107250004095542F6281772767FD7095E8E5EE2E03
:10726000E2E0FE2EE61AF70AEE0CFF1CEE0CFF1C05
:107270000027F7FC0095102F64EBA62EB12CC12C33
:10728000D12CEDB7FEB7A182B282C382D482BC01F9
:10729000CD01AA24BB2465010E946B970F900F902B
:1072A0000F900F90CB011F910F91FF90EF90DF9007
:1072B000CF90BF90AF900895AF92BF92CF92DF92E0
:1072C000EF92FF920F931F93CF93DF93EC019B01FB
:1072D00082E0603278070CF048C077FF03C020E0FE
:1072E00030E005C0653B710514F024EB30E000D0C0
:1072F0000F92B901882777FD8095982F2981332730
:1073000027FD3095E8E8AE2EB12CA21AB30AAA0CDC
:10731000BB1CAA0CBB1CCC24B7FCC094DC2CEA819F
:10732000FF27E7FDF09528E532E02E1B3F0B220FEB
:10733000331F220F331F442737FD4095542FEDB7DD
:10734000FEB7218332834383548320E030E040E062
:1073500050E004EBE02EF12C012D112D0E946B97D3
:107360009B010F900F900F900F90CE01B901F5DEA9
:10737000DF91CF911F910F91FF90EF90DF90CF9011
:10738000BF90AF900895EF92FF920F931F93CF930A
:10739000DF938B017A01EC01DC01A35FB44F8C9188
:1073A00087FF04C0FB011182108237C0AE01440F79
:1073B000551F4C0F5D1F440F551F440F551F2C9137
:1073C000332727FD3095240F351F8091A00A90E0C8
:1073D0002817390714F58C91992787FD9095840F0C
:1073E000951FFC01EE0FFF1FE80FF91FEF55F54F3A
:1073F000808186FF12C08C91992787FD9095840F1C
:10740000951FFC01EE0FFF1FE80FF91FEF55F54F19
:1074100080818F7360E00E94E693DE01A35FB44F2A
:107420008C918F5F8C93AE01440F551F4C0F5D1FE5
:10743000440F551F440F551F2C91332727FD3095BE
:10744000240F351F8091A00A90E0281739070CF00F
:107450004DC08C918C300CF049C0F80120813181F5
:107460008C91992787FD9095840F951FFC01EE0F55
:10747000FF1FE80FF91FEF55F54F81819281280F0B
:10748000391FF701318320838C91992787FD9095CF
:10749000840F951FFC01EE0FFF1FE80FF91FEF553A
:1074A000F54F808186FF2AC08C91992787FD9095A2
:1074B000840F951FFC01EE0FFF1FE80FF91FEF551A
:1074C000F54F80818F7361E00E94E69317C080E4DE
:1074D0009CE904C0F801808191810496F7019183B1
:1074E0008083C35FD44F8FEF888308C0F801808109
:1074F0009181049680549C4950F3ECCFDF91CF9159
:107500001F910F91FF90EF9008951F920F920FB669
:107510000F920BB60F9211242F933F934F935F93CB
:107520006F937F938F939F93AF93BF93EF93FF934B
:1075300080E090E064E271E048E251E024DFFF91F6
:10754000EF91BF91AF919F918F917F916F915F91DB
:107550004F913F912F910F900BBE0F900FBE0F9048
:107560001F9018951F920F920FB60F920BB60F92A5
:1075700011242F933F934F935F936F937F938F9338
:107580009F93AF93BF93EF93FF9382E090E064EA01
:1075900070E048EA50E0F7DEFF91EF91BF91AF91C4
:1075A0009F918F917F916F915F914F913F912F911B
:1075B0000F900BBE0F900FBE0F901F9018951F924B
:1075C0000F920FB60F920BB60F9211242F933F9389
:1075D0004F935F936F937F938F939F93AF93BF93DB
:1075E000EF93FF9381E090E064E970E048E950E0B8
:1075F000CADEFF91EF91BF91AF919F918F917F91E3
:107600006F915F914F913F912F910F900BBE0F9013
:107610000FBE0F901F9018952F923F924F925F923E
:107620006F927F928F929F92AF92BF92CF92DF9292
:10763000EF92FF920F931F93DF93CF9300D000D070
:10764000CDB7DEB71C017C836B836A01FA01E08051
:10765000F18002811381C801B70120E030E040E0F1
:1076600050E00E94A89A87FF04C017FB109517F9F5
:107670001095C101880F991F880F991F9A838983DC
:1076800026016624772443C0F401A080B180C28023
:10769000D380C601B50120E030E040E050E00E9418
:1076A000A89A88231CF0A601950103C0A6019501A4
:1076B0005058C801B7010E949A9888239CF4C601CB
:1076C000B50120E030E040E050E00E94A89A882315
:1076D0001CF08601750106C08601750117FB109527
:1076E00017F910958D819E8101969E838D83E4E02C
:1076F000F0E08E0E9F1E8D819E818215930524F2EF
:107700000894611C711CE981FA814E0E5F1E8B8109
:107710009C816816790624F442011E821D82EBCFFB
:10772000B701C80126960FB6F894DEBF0FBECDBFD5
:10773000CF91DF911F910F91FF90EF90DF90CF904D
:10774000BF90AF909F908F907F906F905F904F9081
:107750003F902F9008952F923F924F925F926F9299
:107760007F928F929F92AF92BF92CF92DF92EF92D1
:10777000FF920F931F93DF93CF93CDB7DEB72A9776
:107780000FB6F894DEBF0FBECDBF98878F834A0136
:107790005B013901181619060CF063C1CB01BA015F
:1077A00020E030E040E050E00E949A98882309F4FD
:1077B00058C10130110529F421E0C216D10419F491
:1077C00060C017FD03C020E030E00DC081E090E014
:1077D0004F815885841B950B089F9001099F300DA0
:1077E000189F300D1124D7FC03C060E070E00DC07D
:1077F00081E090E0EF81F8858E1B9F0BC89EB00161
:10780000C99E700DD89E700D1124CC0CDD1CCC0CC3
:10781000DD1C1B01220C331C220C331C2E0C3F1CC4
:107820002801440C551C440C551C7901EE0CFF1C1E
:10783000EE0CFF1CE60CF71C00E010E0C501B401E3
:10784000F70120813181428153810E947A9B9B0103
:10785000AC01F10160817181828193810E94C197A5
:10786000F10160837183828393830F5F1F4F2C0C20
:107870003D1CE40CF51C2F81388502171307F4F228
:10788000F0C00F8118850370107067012301222456
:1078900033241CC0C501B401F20121913191419101
:1078A00051912F010E947A9B9B01AC01F6016081EE
:1078B0007181828193810E94C197F60161937193D6
:1078C000819391936F010894211C311C201631067D
:1078D0000CF3C801880F991F880F991F1701280EF4
:1078E000391E9301280F391F3E832D830F5F1F4FD1
:1078F000C801880F991F880F991F2701480E591E2C
:10790000A301480F591F5C834B830F5F1F4FC801B2
:10791000880F991F880F991F6701C80ED91EF301A0
:10792000E80FF91FFA83E9830F5F1F4FC801880F23
:10793000991F880F991F035010409701280F391F76
:107940003A8729877301E80EF91E85C0C501B40185
:10795000ED81FE8120813181428153810E947A9B99
:107960009B01AC01F10160817181828193810E9450
:10797000C197F1016083718382839383C501B40150
:10798000EB81FC8120813181428153810E947A9B6D
:107990009B01AC01F20160817181828193810E941F
:1079A000C197F2016083718382839383C501B4011F
:1079B000E981FA8120813181428153810E947A9B41
:1079C0009B01AC01F60160817181828193810E94EB
:1079D000C197F6016083718382839383C501B401EB
:1079E000F70120813181428153810E947A9B9B0162
:1079F000AC01E985FA8560817181828193810E9461
:107A0000C197E985FA8560837183828393830C5FD4
:107A10001F4F20E130E0220E331E4D815E81405F1A
:107A20005F4F5E834D83420E531E8B819C81409637
:107A30009C838B83C20ED31EE981FA817096FA83F0
:107A4000E98329853A85205F3F4F3A87298740E1BE
:107A500050E0E40EF51E8F819885081719070CF485
:107A600075CF2A960FB6F894DEBF0FBECDBFCF916B
:107A7000DF911F910F91FF90EF90DF90CF90BF901B
:107A8000AF909F908F907F906F905F904F903F90BE
:107A90002F9008952F923F924F925F926F927F9214
:107AA0008F929F92AF92BF92CF92DF92EF92FF920E
:107AB0000F931F93DF93CF93CDB7DEB72E970FB6FB
:107AC000F894DEBF0FBECDBF9E878D874B01390175
:107AD000F801181619065CF00F2EF0E0CF2EF0E03A
:107AE000DF2EF0E0EF2EF0E0FF2EF02D93C14130BD
:107AF000510521F40130110519F469C057FD03C087
:107B000060E070E00DC081E090E02D853E85821B35
:107B1000930B489FB001499F700D589F700D112421
:107B2000F7FD03C020E030E00DC081E090E0AD85BE
:107B3000BE858A1B9B0BE89F9001E99F300DF89F43
:107B4000300D11242A01440C551C440C551C8B018A
:107B5000000F111F000F111F080D191D4F01880C78
:107B6000991C880C991C1901220C331C220C331C03
:107B7000260C371CAA24BB240F2EF0E0CF2EF0E0F9
:107B8000DF2EF0E0EF2EF0E0FF2EF02DF801608107
:107B9000718182819381D1012D913D914D915C91B3
:107BA0000E947A9B9B01AC01C701B6010E94C1975C
:107BB0006B017C010894A11CB11C040D151D280C3F
:107BC000391CED85FE85AE16BF0604F323C18D85F5
:107BD0009E8565E070E00E947F9C8C01AA24BB24F6
:107BE0000F2EF0E0CF2EF0E0DF2EF0E0EF2EF0E0F1
:107BF000FF2EF02D442455241FC0F401E40DF51D83
:107C0000D301A40DB51D60817181828193812D9175
:107C10003D914D915C910E947A9B9B01AC01C70103
:107C2000B6010E94C1976B017C010894A11CB11C94
:107C300024E030E0420E531EA016B106F4F2C80153
:107C4000880F991F880F991FD401A80FB91FBC87EF
:107C5000AB87F301E80FF91FFA87E9870F5F1F4F22
:107C6000C801880F991F880F991F9401280F391F89
:107C700038872F83D301A80FB91FBE83AD830F5F51
:107C80001F4FC801880F991F880F991FF401E80F33
:107C9000F91FFC83EB839301280F391F3A83298353
:107CA0000F5F1F4FC801880F991F880F991F14017C
:107CB000280E391E2301480E591E0F5F1F4FC801A1
:107CC000880F991F880F991F04501040880E991E25
:107CD0005301A80EB91E380197C0AB85BC856D91C4
:107CE0007D918D919C91E985FA8520813181428138
:107CF00053810E947A9B9B01AC01C701B6010E948F
:107D0000C1977B018C01AF81B8856D917D918D917B
:107D10009C91ED81FE8120813181428153810E94BD
:107D20007A9B9B01AC01C801B7010E94C1977B01FE
:107D30008C01AB81BC816D917D918D919C91E9818C
:107D4000FA8120813181428153810E947A9B9B017B
:107D5000AC01C801B7010E94C1977B018C01D10120
:107D60006D917D918D919C91F201208131814281B3
:107D700053810E947A9B9B01AC01C801B7010E940C
:107D8000C1977B018C01D4016D917D918D919C9166
:107D9000F50120813181428153810E947A9B9B01B0
:107DA000AC01C801B7010E94C1976B017C0125E0BD
:107DB00030E0620E731E8B859C8544969C878B8772
:107DC000A985BA855496BA87A987EF81F8857496F4
:107DD000F887EF832D813E812C5E3F4F3E832D83BC
:107DE0008B819C8144969C838B83A981BA81549614
:107DF000BA83A983E4E1F0E02E0E3F1E4E0E5F1E13
:107E00008E0E9F1EAE0EBF1E2D853E85621673061A
:107E10000CF463CFB601C7012E960FB6F894DEBFFF
:107E20000FBECDBFCF91DF911F910F91FF90EF90CB
:107E3000DF90CF90BF90AF909F908F907F906F908A
:107E40005F904F903F902F9008952F923F924F92C6
:107E50005F926F927F928F929F92AF92BF92CF92DA
:107E6000DF92EF92FF920F931F93DF93CF93CDB7E3
:107E7000DEB7EC970FB6F894DEBF0FBECDBF9CA760
:107E80008BA77EA76DA758AB4FA73AAB29AB1CAB0E
:107E90000BAB37017601BEAAADAA98AE8FAA689641
:107EA000EEADFFAD689700E010E0CF01815F984D27
:107EB0008F519E4410F001E010E0CF0160E177E2C5
:107EC0000E947F9C9AAF89AF892B21F061E070E01E
:107ED0007AAF69AF1AA619A6CF0168EE73E00E94C7
:107EE0007F9C8D599F4F873C910520F081E090E069
:107EF0009AA789A718A61FA2CF0164E670E00E9486
:107F00007F9C0996439720F0A1E0B0E0B8A7AFA30B
:107F1000CF016AE070E00E947F9C9CAF8BAF892B01
:107F200021F0E1E0F0E0FCAFEBAF8FA598A901975D
:107F300029A93AA93A8329838217930714F49A83CB
:107F4000898369817A81672B09F068C0012B51F020
:107F5000F30180819181A281B381F70180839183B4
:107F6000A283B38329AD3AAD232B59F0F30180816D
:107F70009181A281B381EDA9FEA980839183A2831F
:107F8000B3832BAD3CAD232B69F0F301808191814C
:107F9000A281B3816696EEADFFAD66978083918333
:107FA000A283B38329A53AA5232B21F1ABA5BCA5B8
:107FB000ED90FD900D911C91C801B70120E030E0DB
:107FC00040E050E00E949A98882329F4E1E0F0E034
:107FD000FEA3EDA311C0D3016D917D918D919C9174
:107FE000A80197010E94A198EFA9F8AD6083718361
:107FF000828393831EA21DA22FA138A5232B09F4EF
:10800000F9C380E090E0A0E0B0E06496EEADFFAD93
:10801000649780839183A283B383ECC30115110518
:10802000E9F061E070E040E050E013C09701240FF8
:10803000351FF301E40FF51F80819181A281B38187
:10804000F90180839183A283B3836F5F7F4F4C5F7D
:108050005F4F2FA538A92617370744F769AD7AADCA
:10806000672BF1F061E070E040E050E014C02DA912
:108070003EA9240F351FF301E40FF51F8081918184
:10808000A281B381F90180839183A283B3836F5F5F
:108090007F4F4C5F5F4F2FA538A9261737073CF756
:1080A000012B09F4C7C021E030E069817A81261BE9
:1080B000370BA901440F551F440F551F509541958B
:1080C0005F4F8BA99CA9840F951F9C8B8B8BADA5B3
:1080D000BEA5A095B095AA0FBB1FAA0FBB1FBA8B58
:1080E000A98B615070408DA59EA50196689F2001C7
:1080F000699F500C789F500C1124440C551C440C63
:10810000551CEBA5FCA54E0E5F1EAFA5B8A9119698
:10811000B8ABAFA7E981FA81AE1BBF0BB88BAF87B5
:10812000AFA5B8A91197B8ABAFA7880F991F880F53
:10813000991FEE27FF27E81BF90BFE87ED878DA51A
:108140009EA5689F3001699F700C789F700C112468
:10815000621A730A660C771C660C771CABA5BCA56B
:108160006A0E7B1E1701240E351EE1E0F0E0FAA333
:10817000E9A358C0AB89BC89ED90FD900D911C918D
:10818000C801B70120E030E040E050E00E949A983A
:10819000882361F1F20180809180A280B380D201B6
:1081A000ED92FD920D931C9313978F859889B301DF
:1081B00041E050E0910101E010E06CDC9058F201E8
:1081C00020813181428153810E94A198AB01BC0181
:1081D0008F85988993017101E1E0CE2ED12CBBDA15
:1081E000D2018D929D92AD92BC921397E9A1FAA112
:1081F0003196FAA3E9A32B893C89245030403C8B6B
:108200002B8B69897A89460E571E8F85988901962E
:10821000988B8F87AD85BE856A0E7B1EECEFFFEFD6
:108220002E0E3F1E29A13AA169817A816217730738
:108230000CF0A0CF89AD9AAD892B09F489C0ADA50A
:10824000BEA51196BEA7ADA7AA0FBB1FAA0FBB1F45
:10825000BE8BAD8BEDA5FEA53197FEA7EDA72BA498
:108260003CA44FA458A8CF0180959095880F991FE2
:10827000880F991F22273327281B390B3C832B8318
:10828000310161E070E07CA36BA3188E1F8A58C097
:10829000EBA9FCA98F89988DE80FF91FE080F18088
:1082A00002811381C801B70120E030E040E050E0D6
:1082B0000E949A98882369F1D1018D909D90AD908C
:1082C000BC90F101E082F18202831383EDA8FEA845
:1082D0002F89388DE20EF31EC201B30141E050E058
:1082E000970101E010E0D6DB9058D1012D913D912E
:1082F0004D915C910E94A198AB01BC01C201930118
:10830000E1E0CE2ED12C27DAF10180829182A28287
:10831000B3822BA13CA12F5F3F4F3CA32BA36F89BE
:10832000788D6C5F7F4F788F6F8B8D899E89280E3B
:10833000391E089441085108AB81BC816A0E7B1E2E
:10834000EBA1FCA129813A812E173F070CF0A0CFA9
:1083500069A57AA5672BF9F061E070E040E050E094
:1083600015C02FA938AD240F351FEDA9FEA9E40FC4
:10837000F51F80819181A281B381F901808391836E
:10838000A283B3836F5F7F4F4C5F5F4F29A93AA9E8
:108390002617370734F76BAD7CAD672B09F161E029
:1083A00070E040E050E017C066962EAD3FAD669796
:1083B000240F351FEDA9FEA9E40FF51F80819181DF
:1083C000A281B381F90180839183A283B3836F5F1C
:1083D0007F4F4C5F5F4F29A93AA92617370724F72B
:1083E0006FA178A5672B41F189A99AA9AFA5B8A972
:1083F0008A179B070CF59C01880F991F880F991FFE
:108400004DA95EA9480F591F6496EEADFFAD649764
:10841000E80FF91F0AC0DA01ED90FD900D911D9152
:10842000AD01E192F192019311932F5F3F4F6FA540
:1084300078A9621773077CF78BAD9CAD892B11F17E
:10844000A9A9BAA9EFA5F8A9AE17BF07DCF4CD0119
:10845000FD01EE0FFF1FEE0FFF1F66962EAD3FAD25
:108460006697E20FF31F20E030E040E050E004C0E8
:10847000219331934193519301966FA578A9681781
:108480007907B4F78FA198A5892BA9F06496EEAD72
:10849000FFAD649781E090E020E030E040E050E004
:1084A00005C021933193419351930196A9A9BAA98B
:1084B000A817B907B4F7E9A5FAA5EF2B09F49EC0F0
:1084C00069A87AA8089461087108660C771C660C84
:1084D000771C2FA938AD620E731E8DA59EA5880F3F
:1084E000991F880F991F66277727681B790B7A8F4A
:1084F000698F89A99AA90197ADA5BEA58A9F400158
:108500008B9F900C9A9F900C1124880C991C880CBE
:10851000991CEBA5FCA58E0E9F1EA095B095AA0FE9
:10852000BB1FAA0FBB1FBE83AD832DA53EA52F5F2A
:108530003F4F829F5001839FB00C929FB00C11243B
:10854000215030403EA72DA7AA0CBB1CAA0CBB1C77
:10855000AE0EBF1E29A83AA8F1E04F2E512C48C0FC
:10856000C9A8DAA8C418D508D501ED90FD900D91E1
:108570001C91C801B70120E030E040E050E00E94CB
:108580009A98882319F43EA22DA23AC0F301608183
:10859000718182819381A80197010E94A198D301E2
:1085A0006D937D938D939C931397B1E02B163104BB
:1085B00069F0AB01BC017058C601940101E010E004
:1085C000EFA8F8ACE1E0CE2ED12CC5D80894411C20
:1085D000511CECEFFFEF6E0E7F1E0894210831084E
:1085E000298D3A8D820E931E6D817E81A60EB71E57
:1085F00089A99AA9841595050CF0B2CF1EA21DA2D7
:10860000AFA1B8A5AB2B09F466C041E050E0E98109
:10861000FA814E1B5F0B9A01220F331F220F331F6B
:10862000309521953F4F6BA97CA9620F731F78A3EA
:108630006F8F8DA59EA580959095880F991F880FA7
:10864000991F9E8F8D8FBF01615070408DA59EA593
:108650000196689F3001699F700C789F700C1124FF
:10866000660C771C660C771CABA5BCA56A0E7B1E3E
:108670008FA498A80894811C911C8E1A9F0A880FB9
:10868000991F880F991FEE27FF27E81BF90BFC8F16
:10869000EB8F8DA59EA5689F5001699FB00C789FB8
:1086A000B00C1124A41AB50AAA0CBB1CAA0CBB1C42
:1086B000AA0EBB1E66962EAC3FAC6697220E331EEA
:1086C00064964EAC5FAC6497420E531EA1E0B0E0DE
:1086D000BC87AB8787C0EBADFCADEF2B09F095CF26
:1086E00089C0AF8DB8A1ED90FD900D911C91C8018E
:1086F000B70120E030E040E050E00E949A988823E3
:1087000009F454C0D3016D917D918D919C916F833B
:10871000788789879A87F301E082F1820283138345
:108720002FA138A5232BD1F0C401B50141E050E0C1
:10873000920101E010E0AED99058D3012D913D9106
:108740004D915C910E94A198AB01BC01C4019501BF
:108750007201F1E0CF2ED12C0E94AB3BEBADFCAD12
:10876000EF2BD1F0C401B50141E050E0910101E0EF
:1087700010E090D99058D3012D913D914D915C918D
:108780000E94A198AB01BC01C40195017101E1E017
:10879000CE2ED12C0E94AB3B6F81788589859A853E
:1087A000D3016D937D938D939C931397EB85FC85FB
:1087B0003196FC87EB872F8D38A12450304038A3A9
:1087C0002F8F6D8D7E8D660E771E0894811C911CF7
:1087D0008B8D9C8DA80EB91EACEFBFEF2A0E3B1EF1
:1087E0004A0E5B1EEB85FC8529813A812E173F07D7
:1087F0000CF077CF8DA19EA1EC960FB6F894DEBF5A
:108800000FBECDBFCF91DF911F910F91FF90EF90E1
:10881000DF90CF90BF90AF909F908F907F906F90A0
:108820005F904F903F902F9008952F923F924F92DC
:108830005F926F927F928F929F92AF92BF92CF92F0
:10884000DF92EF92FF920F931F93DF93CF9300D0AD
:108850000F92CDB7DEB79C838B833A83298338018F
:10886000260114010115110509F100D000D0EDB762
:10887000FEB73196ADB7BEB71296BC92AE921197C5
:10888000B382A2828EE690E0958384838B819C8163
:1088900098010A8D1B8D65014201D7DAEDB7FEB74D
:1088A00036960FB6F894FEBF0FBEEDBF6101F10121
:1088B00020E030E009C080819181909581959F4FA3
:1088C000819391932F5F3F4F89819A8128173907B0
:1088D00094F3F301EE0FFF1FEE0FFF1FE40DF51DE4
:1088E000830180E090E0A0E0B0E006C08193919326
:1088F000A193B1930F5F1F4F29813A81021713078C
:10890000ACF3720101E010E0F1E0AF2EB12C46C0F3
:10891000D6018D919C91119718161906ACF122275A
:108920003327281B390B2D933C932BC0F701408133
:10893000518162817381C501821B930B9C01880F59
:10894000991F880F991FF201E81BF90B6080718055
:1089500082809380D7016D927D928D929C92139725
:108960004083518362837383220F331FF101E21B23
:10897000F30B8081918122273327281B390B318308
:1089800020832017310791F60F5F1F4FE2E0F0E0E0
:10899000CE0EDF1E24E030E0E20EF31E89819A81C4
:1089A000801791070CF0B4CF0F900F900F900F909D
:1089B000CF91DF911F910F91FF90EF90DF90CF90BB
:1089C000BF90AF909F908F907F906F905F904F90EF
:1089D0003F902F9008952F923F924F925F926F9207
:1089E0007F928F929F92AF92BF92CF92DF92EF923F
:1089F000FF920F931F93DF93CF9300D00F92CDB7C9
:108A0000DEB79A8389833A014B01290118161906AA
:108A10000CF0EAC00130110509F0AFC065E070E06C
:108A20000E947F9C8C017901CC24DD2412C0F701C7
:108A30006081718182819381A40193010E947A9B5C
:108A4000F70161937193819391937F010894C11C05
:108A5000D11CC016D1065CF31801220C331C220C69
:108A6000331C240C351C58010894A11CB11CAA0C01
:108A7000BB1CAA0CBB1CA40CB51C42E0C42ED12C00
:108A8000C00ED11ECC0CDD1CCC0CDD1CC40CD51CC6
:108A900023E0E22EF12CE00EF11EEE0CFF1CEE0C9A
:108AA000FF1CE40CF51C98012C5F3F4F220F331F75
:108AB000220F331F240D351D3C832B8357C0F1013A
:108AC0006081718182819381A40193010E947A9BCC
:108AD000F1016083718382839383F50160817181E9
:108AE00082819381A40193010E947A9BF5016083A6
:108AF000718382839383F601608171818281938186
:108B0000A40193010E947A9BF601608371838283A2
:108B10009383F7016081718182819381A401930124
:108B20000E947A9BF7016083718382839383EB8138
:108B3000FC816081718182819381A40193010E94F3
:108B40007A9BEB81FC8160837183828393830B5FCB
:108B50001F4F24E130E0220E331EA20EB31EC20EC0
:108B6000D31EE20EF31E7496FC83EB8389819A81F7
:108B7000081719070CF4A3CF37C017FD03C060E036
:108B800070E00DC081E090E0E981FA818E1B9F0BBF
:108B9000089FB001099F700D189F700D1124780176
:108BA000EE0CFF1CEE0CFF1C6B01CC0CDD1CCC0C86
:108BB000DD1CC40CD51C00E010E0F6016081718161
:108BC00082819381A40193010E947A9BF6016083C4
:108BD0007183828393830F5F1F4FCE0CDF1C29812B
:108BE0003A81021713074CF30F900F900F900F90DC
:108BF000CF91DF911F910F91FF90EF90DF90CF9079
:108C0000BF90AF909F908F907F906F905F904F90AC
:108C10003F902F9008954F925F926F927F928F9224
:108C20009F92AF92BF92CF92DF92EF92FF920F93FB
:108C30001F93CF93DF932C014B01390118161906AE
:108C40000CF0F2C04130510509F09CC00130110513
:108C500009F09AC063E070E00E947F9CBC0184012F
:108C6000E901E0E0F0E014C0D8012D913D914D9173
:108C70005C911397C880D980EA80FB80CD92DD9209
:108C8000ED92FD928D012993399349935993319631
:108C9000E617F7074CF3CB01880F991F880F991F30
:108CA0005401A80EB91E6301C80ED91E6F5F7F4F15
:108CB000CB01880F991F880F991F7401E80EF91EC8
:108CC0008301080F191F6F5F7F4FCB01880F991F1A
:108CD000880F991F62507040E401C80FD91FF3013B
:108CE000E80FF91F4AC0D5012D913D914D915C913E
:108CF000D6016D907D908D909C90D5016D927D9266
:108D00008D929C921397D6012D933D934D935C9336
:108D10001397D7012D913D914D915C91D8016D90A4
:108D20007D908D909C90D7016D927D928D929C92BA
:108D30001397D8012D933D934D935C9313972881FE
:108D400039814A815B8180819181A281B38188834D
:108D50009983AA83BB8320833183428353836D5FCE
:108D60007F4F8CE090E0A80EB91EC80ED91EE80E09
:108D7000F91E045F1F4F2C963C96641575050CF484
:108D8000B2CF52C057FD03C020E030E00BC081E0FD
:108D900090E084199509489F9001499F300D589F94
:108DA000300D112417FD03C060E070E00BC081E0BE
:108DB00090E084199509089FB001099F700D189FD4
:108DC000700D11247A01EE0CFF1CEE0CFF1CE90162
:108DD000CC0FDD1FCC0FDD1FC80DD91D000F111FDB
:108DE000000F111FFB01EE0FFF1FEE0FFF1FE60D1F
:108DF000F71D60E070E0288139814A815B818081C4
:108E00009181A281B38188839983AA83BB832083C4
:108E10003183428353836F5F7F4FCE0DDF1DE00FA1
:108E2000F11F641575053CF3DF91CF911F910F91F0
:108E3000FF90EF90DF90CF90BF90AF909F908F907A
:108E40007F906F905F904F9008952F923F924F9236
:108E50005F926F927F928F929F92AF92BF92CF92CA
:108E6000DF92EF92FF920F931F93CF93DF937C01DA
:108E70005B014A016E9DC0016F9D900D7E9D900D1E
:108E80001124880F991F880F991F0E944794792EEB
:108E9000482F592F682E6701CC0CDD1CCC0CDD1C33
:108EA000E0E0F0E060E070E012C0D8012D903D906D
:108EB0004D905D908D0129923992499259922F5F80
:108EC0003F4F2E153F058CF331966C0D7D1DEA1535
:108ED000FB054CF48401060F171FEA01C60FD71FCC
:108EE00020E030E0EECFC301DF91CF911F910F91D1
:108EF000FF90EF90DF90CF90BF90AF909F908F90BA
:108F00007F906F905F904F903F902F9008952F9299
:108F10003F924F925F926F927F928F929F92AF9209
:108F2000BF92CF92DF92EF92FF920F931F93DF9346
:108F3000CF9300D00F92CDB7DEB71C01FB011816FE
:108F400019060CF0A8C0141615060CF0A4C081E098
:108F50002816310499F4E080F18002811381C80160
:108F6000B70120E030E040E050E00E94A89A87FF7F
:108F70009CC017FB109517F9109597C0DA01AA0F3E
:108F8000BB1FAA0FBB1FBA83A9832B011C821B82A4
:108F90000F2EF0E0EF2EF0E0FF2EF0E00F2FF0E0CC
:108FA0001F2FF02D0F2EF0E06F2EF0E07F2EF0E857
:108FB0008F2EFFE39F2EF02DF201A080B180C280A2
:108FC000D380C601B50120E030E040E050E00E94CF
:108FD0009A98882309F445C0C601B50120E030E025
:108FE00040E050E00E94A89A87FF04C0D7FAD094CE
:108FF000D7F8D094C801B701A60195010E949A98AC
:109000008823ECF4C801B701A60195010E94A1983C
:109010007B018C01C401B301A80197010E947A9BD6
:10902000A80197010E947A9B20E030E040E85FE3CE
:109030000E94C1973B014C018601750112C0C60117
:10904000B501A80197010E94A1989B01AC010E9463
:109050007A9B9B01AC01C401B3010E94C1973B0103
:109060004C018B819C8101969C838B83A981BA8161
:109070004A0E5B1E821593050CF49ECFC401B3010A
:109080000E94E79B9B01AC01C801B7010E947A9B3B
:109090007B018C010AC00F2EF0E0EF2EF0E0FF2ED6
:1090A000F0E00F2FF0E01F2FF02DB701C8010F9057
:1090B0000F900F900F90CF91DF911F910F91FF9024
:1090C000EF90DF90CF90BF90AF909F908F907F9068
:1090D0006F905F904F903F902F9008952F923F9206
:1090E0004F925F926F927F928F929F92AF92BF92B8
:1090F000CF92DF92EF92FF920F931F93DF93CF9364
:10910000CDB7DEB7C254D0400FB6F894DEBF0FBE65
:10911000CDBF98AB8FA77AAB69AB5CAB4BAB3EAB2B
:109120002DAB18AF0FABFAAEE9AEDCAECBAEAB28D1
:1091300031F431E0432E512C22243324E7C0E9AC32
:10914000FAACAFA4B8A821E0622E712C91E0492EB0
:10915000512CCC24CA94DC2C81E0882E912C52C056
:10916000D7018D919C91119797FF03C0CD92DC920E
:1091700003C0F7017182608218161906ACF56414F9
:109180007504F9F008944108510829A93AA9429EAA
:10919000B001439E700D529E700D11240894411C25
:1091A000511C660F771F660F771F4FA558A9640FD4
:1091B000751F8BA99CA941E050E0950101E010E0EA
:1091C0002ADDF201E819F909EE0FFF1F89AD9AAD0A
:1091D000E80FF91F80819181D7018D939C93718253
:1091E00060820894411C511C0894611C711CE2E0CF
:1091F000F0E0EE0EFF1E24E030E0A20EB31E089455
:10920000C108D1084DA95EA9461557050CF0A8CF95
:109210004A01089481089108880C991C89AD9AAD7F
:10922000880E991E89A99AA9880F991F880F991FDE
:10923000AA24BB24A81AB90A41505040A9A9BAA926
:109240004A9F70014B9FF00C5A9FF00C11244F5F06
:109250005F4F5EAB4DABEE0CFF1CEE0CFF1CEFA5A1
:10926000F8A9EE0EFF1E6A011A014CC0D4012D911F
:109270003C91119737FF3DC088279927821B930B9C
:109280008D939C93C214D30489F10894210831086A
:10929000E9A9FAA92E9EB0012F9E700D3E9E700D79
:1092A00011240894211C311C660F771F660F771F4D
:1092B0002FA538A9620F731F8BA99CA941E050E02C
:1092C000970101E010E0A7DCF1013197EE0FFF1FDD
:1092D00049AD5AADE40FF51F20813181D4018D9144
:1092E0009C911197918380832D933C93089421083E
:1092F00031080894C108D108EEEFFFEF8E0E9F1ED3
:10930000EA0CFB1C1C141D040CF4B0CF29A93AA9CB
:10931000220F331F220F331F3E872D8708944108E9
:10932000510849A95AA9449E8001459E100D549E9A
:10933000100D1124000F111F000F111F8FA598A9E8
:10934000080F191FA0E0B0E04A0E5B1E5201AA0CE4
:10935000BB1CAA0CBB1C0894411C511CEFA8F8AC08
:10936000EA0CFB1C32016701490190948194910839
:10937000939411C0B801680D791D8BA99CA941E097
:1093800050E0C5DDF60161937193819391936F0174
:109390000894611C711C2D853E85020F131F261435
:1093A000370444F7EBADFCADEA0DFB1D92010CC098
:1093B000D7014D915D916D917D917D0141935193C7
:1093C000619371932F5F3F4F221633068CF7EDA9FF
:1093D000FEA9FAA7E9A72BA93CA92E173F0714F469
:1093E0003AA729A74FA958AD5C8F4B8F89A99AA995
:1093F00080959095880F991F880F991FAA27BB27E2
:10940000A81BB90BB88FAF8BEFA5F8A9FA8BE98B26
:1094100029A93AA92F5F3F4F3AAB29AB220F331F3F
:10942000220F331F3E8B2D8B49A95AA94150504022
:109430005AAB49ABCF01AD85BE858A0F9B1F9CA35C
:109440008BA3EBADFCADFC8BEB8B4FA558A9420F6A
:10945000531F5A83498389AD9AAD988B8F87ABA9E7
:10946000BCA9BA8FA98FEFA5F8A9F887EF832BA124
:109470003CA13C832B83FE83ED8341E050E05CA75D
:109480004BA7AFC28BA59CA5841595050CF4A2C073
:10949000821593050CF09EC07C0123969FAF8EAF82
:1094A00023970B8D1C8D8824AA24CC24DD24D8017D
:1094B0006C9011967C90119712969C90129713962F
:1094C000BC90682D7A2DC6019301492D5B2D0E9419
:1094D0009A9888232CF42396FFAEEEAE239704C00F
:1094E000682C7A2C9C2CBD2C0894E11CF11C0C5F80
:1094F0001F4F2E143F042CF0862CA72CC92CDB2CDC
:10950000D6CF2396EEADFFAD23972BA53CA5E21752
:10951000F30709F45FC0319749A95AA9E49F900164
:10952000E59F300DF49F300D112431962396FFAF47
:10953000EEAF2397220F331F220F331F8FA598A959
:10954000280F391F8BA99CA96D817E8141E050E0D5
:1095500001E010E060DB21E030E02396AEADBFAD6E
:1095600023972A1B3B0BF901EE0FFF1FEE0FFF1F86
:10957000F095E195FF4F4FA958AD4E0F5F1FAB8D92
:10958000BC8DED90FD900D911C91DA01ED92FD9254
:109590000D931C9313974BAD5CADE40FF51FAB8996
:1095A000BC894D915D916D917C9140835183628323
:1095B0007383220F331FE9ADFAADE21BF30B208159
:1095C0003181AF85B8898D919C911197918380836A
:1095D0002D933C9320E030E040E050E0AB8DBC8D1B
:1095E0002D933D934D935C931397EBA5FCA52BA96D
:1095F0003CA9E217F30709F4ADC12E1B3F0B3EA7B0
:109600002DA7398D3FAF4A8D21964FAF21975F81AE
:109610005DAF88858EAF832F942F652F788541E0CD
:1096200050E075DC6DA37EA38FA398A720E030E007
:1096300040E050E00E949A98882309F48BC1A989E0
:10964000BA89ED90FD900D911C91C801B70120E001
:1096500030E040E050E00E949A988823E9F0C80189
:10966000B70120E030E040E050E00E949A9887FD8A
:1096700005C020E030E040E85FE304C020E030E0D7
:1096800040E85FEB6DA17EA18FA198A50E947A9B17
:109690006DA37EA38FA398A760E070E080E89FE3AE
:1096A0002DA13EA14FA158A50E94A198AB01BC01DC
:1096B0008FAD21969FAD21972DAD3EAD01E010E01D
:1096C0008AD9E989FA89608171818281938120E058
:1096D00030E040E85FE30E94C197A989BA896D93A1
:1096E0007D938D939C931397EBA5FCA53196FC87F6
:1096F000EB872B8D3C8D2C5F3F4F3AA329A34B89E1
:109700005C894C5F5F4F5E8F4D8F8B819C81239670
:109710009FAF8EAF2397A981BA81B8A3AF8FEBA17A
:10972000FCA1FA87E987F7C08FAD21969FAD2197FD
:109730006DAD7EAD41E050E022962FAD229723968D
:109740003FAD239701E010E00E944A3D9058A9895F
:10975000BA892D913D914D915C910E94A198AB01E8
:10976000BC018FAD21969FAD21972DAD3EAD2296C8
:10977000EFAC22972396FFAC2397E1E0CE2ED12CBD
:109780000E94AB3BEB85FC85E415F5050CF49AC013
:109790002E163F060CF496C0A9A1BAA16D907D903B
:1097A0008D909C90C401B30120E030E040E050E097
:1097B0000E949A98882309F485C0E985FA85E0809B
:1097C000F18002811381C801B70120E030E040E060
:1097D00050E00E94A89A87FF04C017FB109517F964
:1097E0001095C801B701A40193010E94A1989B01A3
:1097F000AC010E947A9B9B01AC0160E070E080E8C4
:109800009FE30E94C0975B016C0120E030E040E0E4
:1098100050E00E94A89A181654F00F2EF0E0AF2ED8
:10982000F0E0BF2EF0E0CF2EF0E0DF2EF02DC401EF
:10983000B301AD8DBE8D2D913D914D915C910E94F6
:10984000A1989B01AC010E947A9B7B018C01C6010F
:10985000B5012DEC3CEC4CE45DE30E947A9BA80141
:1098600097010E947A9B20E030E040E85FE30E948D
:10987000C19720E030E040E85FE30E949A98882397
:1098800069F0C601B5010E94E79B9B01AC01C401D0
:10989000B3010E947A9BE9A1FAA110C08DA59EA5F3
:1098A0006F8D78A141E050E032DBA9A1BAA16D93A0
:1098B0007D938D939C931397ED8DFE8D60837183C3
:1098C000828393832B853C852F5F3F4F3C872B877B
:1098D00023964EAD5FAD23978D859E85480F591F0A
:1098E00023965FAF4EAF2397A9A1BAA11496BAA34E
:1098F000A9A3EF8DF8A1E80FF91FF8A3EF8F2D8D25
:109900003E8D2C5F3F4F3E8F2D8F49855A85480FE6
:10991000591F5A8749878B859C85ADA9BEA9A81771
:10992000B9070CF001CFE989FA8980819181A28180
:10993000B381EB8DFC8D80839183A283B3838DA152
:109940009EA1AFA1B8A5B058E989FA898083918317
:10995000A283B3832BA53CA52F5F3F4F3CA72BA72A
:109960004B8D5C8D4C5F5F4F5C8F4B8F898D9A8DDB
:1099700001979A8F898FAF81B885EF89F88DAE0FE7
:10998000BF1FB887AF8329893A894D895E89240F23
:10999000351F3A8B298B8BA19CA1840F951F9CA30B
:1099A0008BA3AB89BC891496BC8BAB8BE981FA8104
:1099B000E40FF51FFA83E9832B813C814F89588D91
:1099C000240F351F3C832B838D819E81AD85BE8501
:1099D0008A0F9B1F9E838D83EF85F8893296F88BC3
:1099E000EF872BA53CA549A55AA5421753070CF0B4
:1099F00049CDCE5BDF4F0FB6F894DEBF0FBECDBFB3
:109A0000CF91DF911F910F91FF90EF90DF90CF905A
:109A1000BF90AF909F908F907F906F905F904F908E
:109A20003F902F9008952F923F924F925F926F92A6
:109A30007F928F929F92AF92BF92CF92DF92EF92DE
:109A4000FF920F931F93DF93CF93CDB7DEB72C9781
:109A50000FB6F894DEBF0FBECDBF9A8389837C8397
:109A60006B832A013901ED82FE820F831887DA8623
:109A7000C986F50180E090E003C011921192019631
:109A800086159705D4F3C301880F991F880F991F76
:109A90000E9447948B879C8789819A816B817C8106
:109AA000A201930184017501CB84DC84E1E0AE2E38
:109AB000B12C14DBE985FA8511821082130146145A
:109AC00057040CF412014B805C800894411C511C1B
:109AD000440C551C440C551C69807A8088249924B8
:109AE00040C0F301A080B180C280D380C601B5011F
:109AF00020E030E040E050E00E94A89A87FF04C0D8
:109B0000D7FAD094D7F8D094E981FA81E080F18037
:109B100002811381C801B70120E030E040E050E04D
:109B20000E94A89A87FF04C017FB109517F910959B
:109B3000640C751C6D817E818F819885A8019701C9
:109B40000E947A9B9B01AC01C601B5010E949A98C4
:109B500018167CF40894811C911CE985FA85918281
:109B60008082821493040CF4BCCF8B859C850E9468
:109B7000E4942C960FB6F894DEBF0FBECDBFCF9104
:109B8000DF911F910F91FF90EF90DF90CF90BF90EA
:109B9000AF909F908F907F906F905F904F903F908D
:109BA0002F9008952F923F924F925F926F927F92E3
:109BB0008F929F92AF92BF92CF92DF92EF92FF92DD
:109BC0000F931F93DF93CF93CDB7DEB728970FB6D0
:109BD000F894DEBF0FBECDBF9A8389833B012A0173
:109BE0001901DC82CB82BE82AD8298868F828CA1E5
:109BF0009DA1641775071CF42FEF3FEF36C01216B6
:109C000013061CF02EEF3FEF30C0181619061CF09B
:109C10002DEF3FEF2AC0019749F489819A81CB80CB
:109C2000DC80A8A0B9A08AA09BA0FDDE0F920F92B5
:109C3000EB81FC81008111818AA19BA1EDB7FEB768
:109C40009283818389819A81B301A2019101ED8080
:109C5000FE80CF80D884AE8CBF8C88A099A00E9453
:109C6000154420E030E00F900F90C90128960FB600
:109C7000F894DEBF0FBECDBFCF91DF911F910F9142
:109C8000FF90EF90DF90CF90BF90AF909F908F901C
:109C90007F906F905F904F903F902F9008952F92FC
:109CA0003F924F925F926F927F928F929F92AF926C
:109CB000BF92CF92DF92EF92FF920F931F93DF93A9
:109CC000CF93CDB7DEB72C970FB6F894DEBF0FBE9B
:109CD000CDBF4C016B837C835901B7D81C01C401F3
:109CE0006B817C81A1010E940C3B2B013C010B810B
:109CF0001C817801EE0CFF1CEE0CFF1CC7010E94BA
:109D000047948D839E83C801880F991F0E944794B2
:109D10008F839887C7010E94479489879A87C401D7
:109D2000880F991F880F991F0E9447948B879C87E3
:109D30008DB79EB708970FB6F8949EBF0FBE8DBF24
:109D4000CDB6DEB60894C11CD11C60E070E080E89E
:109D500095E2A30192010E94A1987B018C018B8561
:109D6000F60180839C8591838F818283988593837C
:109D7000898584839A85958381E090E097838683A3
:109D8000C101B401A4012B813C816E010894C11C66
:109D9000D11C8D809E8006DFEDB7FEB738960FB6DA
:109DA000F894FEBF0FBEEDBFC1010E94E4948F8105
:109DB00098850E94E49489859A850E94E4948B8515
:109DC0009C850E94E4948D819E812C960FB6F89418
:109DD000DEBF0FBECDBFCF91DF911F910F91FF90DE
:109DE000EF90DF90CF90BF90AF909F908F907F903B
:109DF0006F905F904F903F902F9008951F920F9219
:109E00000FB60F920BB60F9211242F933F934F93DF
:109E10008F939F93EF93FF934091C600E091900B37
:109E2000F091910B31969F012F773070319780918F
:109E3000920B9091930B2817390739F0E05FF44F9C
:109E400040833093910B2093900BFF91EF919F9162
:109E50008F914F913F912F910F900BBE0F900FBE9E
:109E60000F901F9018959A01AB01203081EE3807B2
:109E700080E0480780E0580749F182E08093C00005
:109E800060E079E08DE390E00E94B49C2150304086
:109E900040405040CA01B90122E030E040E050E0CB
:109EA0000E94B49C3093C5002093C4008091C100EF
:109EB00080618093C1008091C10088608093C1005F
:109EC0008091C10080688093C10008951092C00005
:109ED00020E130E0E7CF2091920B3091930B8091FD
:109EE000900B9091910B8217930719F42FEF3FEF8E
:109EF0000EC0F901E05FF44F80812F5F3F4F2F7755
:109F000030703093930B2093920B282F30E0C901CF
:109F100008958091920B9091930B9093910B809365
:109F2000900B089508952F923F924F925F926F92F7
:109F30007F928F929F92AF92BF92CF92DF92EF92D9
:109F4000FF920F931F93DF93CF93CDB7DEB7A09708
:109F50000FB6F894DEBF0FBECDBF1C016A017B01B6
:109F6000411551056105710541F440E350E060E0A1
:109F700070E020E030E08BD055C088249924540153
:109F8000422E55246624772401E010E00C0F1D1F9B
:109F9000080D191DC701B601A30192010E94929CF0
:109FA000F80160830894811C911CA11CB11CC7019D
:109FB000B601A30192010E94929CC901DA016C01D1
:109FC0007D01C114D104E104F104F1F681E0E82E31
:109FD000F12CEC0EFD1EE80CF91C3E010894611CEE
:109FE000711CD501C4010197A109B1096C01C81800
:109FF000D90815C0F601EE0DFF1D40814A3010F45E
:10A00000405D01C0495C552747FD5095652F752F70
:10A01000C10120E030E03BD00894E108F1086E1463
:10A020007F0441F7A0960FB6F894DEBF0FBECDBFF8
:10A03000CF91DF911F910F91FF90EF90DF90CF9024
:10A04000BF90AF909F908F907F906F905F904F9058
:10A050003F902F9008952115310539F48091C0006B
:10A0600085FFFCCF4093C60008955DCFEF92FF922D
:10A070000F931F939A01E62EFF2400E010E0B80131
:10A08000A701E9DF1F910F91FF90EF900895EF92E4
:10A09000FF920F931F93CF93DF93EC017A018B0113
:10A0A0002115310539F48091C00085FFFCCFE09285
:10A0B000C60019C02A303105A9F477FF0FC04DE260
:10A0C00050E060E070E020E030E0E1DF10950095C6
:10A0D000F094E094E11CF11C011D111DCE01B801AA
:10A0E000A7012AE020DFDF91CF911F910F91FF9010
:10A0F000EF900895EF92FF920F931F937B019A01C7
:10A100000027F7FC0095102FB801A701C0DF1F91B1
:10A110000F91FF90EF9008950F931F938C014DE0E6
:10A1200050E060E070E020E030E0B1DFC8014AE0DC
:10A1300050E060E070E020E030E0A9DF1F910F9177
:10A140000895CF92DF92EF92FF920F931F938C01AD
:10A150009A016B01EE24FF24B701A6017CDFC80140
:10A16000DBDF1F910F91FF90EF90DF90CF9008956C
:10A170009F92AF92BF92CF92DF92EF92FF920F9396
:10A180001F93CF93DF93EC017A018B01922ECB01C9
:10A19000BA0120E030E040E050E00E949A98882325
:10A1A00064F4CE014DE250E060E070E020E030E089
:10A1B0006EDF17FB109517F9109520E030E040E0B6
:10A1C0005FE3AA240BC0CA01B90120E030E040E2FD
:10A1D00051E40E94A1989B01AC01A394A91498F3A7
:10A1E000C801B7010E94C1977B018C010E940E99A2
:10A1F0005B016C010E943A999B01AC01C801B70157
:10A200000E94C0977B018C01CE01B601A5012AE016
:10A2100030E021DF992099F1E5E1F2E007C080917B
:10A22000C00085FFFCCF31969093C60090819923A2
:10A23000B1F725C0C801B70120E030E040E251E4A9
:10A240000E947A9B7B018C010E9409995B016C0141
:10A25000CC24B7FCC094DC2CCE01B601A5012AE0C9
:10A2600030E015DFC601B5010E943C999B01AC01AD
:10A27000C801B7010E94C0977B018C019A94992074
:10A28000C9F6DF91CF911F910F91FF90EF90DF9072
:10A29000CF90BF90AF909F9008956ACF0895DF93BD
:10A2A000CF93CDB7DEB766970FB6F894DEBF0FBE7B
:10A2B000CDBF8091170290911802A0911902B09120
:10A2C0001A028F87988BA98BBA8BFE013F9644E6C2
:10A2D00050E08081F999FECF1FBA52BD41BD80BDCB
:10A2E0000FB6F894FA9AF99A0FBE4F5F5F4F48364F
:10A2F000510511F03196EDCFE5E1F5E08081F99956
:10A30000FECF1FBA52BD41BD80BD0FB6F894FA9A78
:10A31000F99A0FBE4F5F5F4F4837510511F03196E4
:10A32000EDCFE5E0F5E08081F999FECF1FBA52BD8F
:10A3300041BD80BD0FB6F894FA9AF99A0FBE4F5FEF
:10A340005F4F4838510511F03196EDCFE5E2F5E069
:10A350008081F999FECF1FBA52BD41BD80BD0FB6B5
:10A36000F894FA9AF99A0FBE4F5F5F4F483951053A
:10A3700011F03196EDCFE9E3F5E08081F999FECF58
:10A380001FBA52BD41BD80BD0FB6F894FA9AF99A32
:10A390000FBE4F5F5F4F4C39510511F03196EDCF35
:10A3A000EDE3F5E08081F999FECF1FBA52BD41BDC2
:10A3B00080BD0FB6F894FA9AF99A0FBE4F5F5F4FBF
:10A3C000403A510511F03196EDCFE5E3F5E080819B
:10A3D000F999FECF1FBA52BD41BD80BD0FB6F894AA
:10A3E000FA9AF99A0FBE4F5F5F4F443A510511F048
:10A3F0003196EDCFEDE4F5E08081F999FECF1FBAFB
:10A4000052BD41BD80BD0FB6F894FA9AF99A0FBEBD
:10A410004F5F5F4F483A510511F03196EDCFE1E0C3
:10A42000F5E08081F999FECF1FBA52BD41BD80BDD4
:10A430000FB6F894FA9AF99A0FBE4F5F5F4F4C3AF5
:10A44000510511F03196EDCFE1E4F5E08081F99905
:10A45000FECF1FBA52BD41BD80BD0FB6F894FA9A27
:10A46000F99A0FBE4F5F5F4F403B510511F0319697
:10A47000EDCFE5E4F5E08081F999FECF1FBA52BD3A
:10A4800041BD80BD0FB6F894FA9AF99A0FBE4F5F9E
:10A490005F4F443B510511F03196EDCFE9E4F5E013
:10A4A0008081F999FECF1FBA52BD41BD80BD0FB664
:10A4B000F894FA9AF99A0FBE4F5F5F4F483B5105E7
:10A4C00011F03196EDCFEBEAFBE08081F999FECFF8
:10A4D0001FBA52BD41BD80BD0FB6F894FA9AF99AE1
:10A4E0000FBE4F5F5F4F443C510511F03196EDCFE9
:10A4F00084EB90E09A83898386E490E09C838B834D
:10A500002FEF30E03E832D8380EF90E098878F839C
:10A5100084E690E09A8789873C872B87FE013196F5
:10A520008081F999FECF1FBA52BD41BD80BD0FB6E3
:10A53000F894FA9AF99A0FBE4F5F5F4F463C510567
:10A5400071F7FE0133968081F999FECF1FBA52BD93
:10A5500041BD80BD0FB6F894FA9AF99A0FBE4F5FCD
:10A560005F4F483C510511F03196EDCFFE01359615
:10A570008081F999FECF1FBA52BD41BD80BD0FB693
:10A58000F894FA9AF99A0FBE4F5F5F4F4A3C510513
:10A5900011F03196EDCFFE0137968081F999FECF0B
:10A5A0001FBA52BD41BD80BD0FB6F894FA9AF99A10
:10A5B0000FBE4F5F5F4F4C3C510511F03196EDCF10
:10A5C000FE0139968081F999FECF1FBA52BD41BD77
:10A5D00080BD0FB6F894FA9AF99A0FBE4F5F5F4F9D
:10A5E0004E3C510511F03196EDCFFE013B96808136
:10A5F000F999FECF1FBA52BD41BD80BD0FB6F89488
:10A60000FA9AF99A0FBE4F5F5F4F403D510511F026
:10A610003196EDCFE6ECFBE08081F999FECF1FBAD1
:10A6200052BD41BD80BD0FB6F894FA9AF99A0FBE9B
:10A630004F5F5F4F443D510511F03196EDCFEEEF86
:10A64000F3E08081F999FECF1FBA52BD41BD80BDB4
:10A650000FB6F894FA9AF99A0FBE4F5F5F4F483DD4
:10A66000510511F03196EDCFE2E0F4E08081F999E7
:10A67000FECF1FBA52BD41BD80BD0FB6F894FA9A05
:10A68000F99A0FBE4F5F5F4F4C3D510511F0319667
:10A69000EDCFE6E0F4E08081F999FECF1FBA52BD1C
:10A6A00041BD80BD0FB6F894FA9AF99A0FBE4F5F7C
:10A6B0005F4F403E510511F03196EDCF80E290E0C2
:10A6C0009E878D87FE013D968081F999FECF1FBA46
:10A6D00052BD41BD80BD0FB6F894FA9AF99A0FBEEB
:10A6E000413E510521F0319641EE50E0EDCF809191
:10A6F0001B0290911C02A0911D02B0911E028B8B37
:10A700009C8BAD8BBE8BFE01739684E690E020811E
:10A71000F999FECF1FBA92BD81BD20BD0FB6F89446
:10A72000FA9AF99A0FBE8736910519F0019631967B
:10A73000EECFE7ECF9E0949108C08091C00085FF6E
:10A74000FCCF9093C600319694919923B1F7E1ED37
:10A75000FBE0949108C08091C00085FFFCCF9093EE
:10A76000C600319694919923B1F78091C00085FF7E
:10A77000FCCF8AE08093C60066960FB6F894DEBFE1
:10A780000FBECDBFCF91DF910895DF93CF93CDB7AB
:10A79000DEB7E0970FB6F894DEBF0FBECDBFDE0187
:10A7A0001196EBE4F4E080E101900D928150E1F725
:10A7B000DE015196EBE3F4E080E101900D928150CF
:10A7C000E1F7DE019196EBE2F4E080E101900D9279
:10A7D0008150E1F789819A81AB81BC818093150515
:10A7E00090931605A0931705B093180589899A8947
:10A7F000AB89BC898093050590930605A093070556
:10A80000B093080589A19AA1ABA1BCA180932505AD
:10A8100090932605A0932705B09328058D819E81EE
:10A82000AF81B8858093190590931A05A0931B05F5
:10A83000B0931C058D899E89AF89B88D80930905D9
:10A8400090930A05A0930B05B0930C058DA19EA1D2
:10A85000AFA1B8A58093290590932A05A0932B0555
:10A86000B0932C0589859A85AB85BC8580931D05A1
:10A8700090931E05A0931F05B0932005898D9A8D96
:10A88000AB8DBC8D80930D0590930E05A0930F05A5
:10A89000B093100589A59AA5ABA5BCA580932D05FD
:10A8A00090932E05A0932F05B09330058D859E853E
:10A8B000AF85B8898093210590932205A093230545
:10A8C000B09324058D8D9E8DAF8DB8A18093110519
:10A8D00090931205A0931305B09314058DA59EA522
:10A8E000AFA5B8A98093310590933205A0933305A5
:10A8F000B09334050E94031D80E090E0AAEFB4E419
:10A900008093390590933A05A0933B05B0933C059D
:10A9100080E090E8ABE3B5E480933D0590933E057D
:10A92000A0933F05B093400520E030E040E050E0C8
:10A9300020933505309336054093370550933805FD
:10A9400080E29EE4A0E0B0E08093010590930205D0
:10A95000A0930305B093040520934D0530934E0555
:10A9600040934F055093500580E090E0A0E4B1E49F
:10A970008093410590934205A0934305B09344050D
:10A980008DEC9CECACECBEE38093450590934605C2
:10A99000A0934705B093480580E090E0A0E2B1E4C1
:10A9A0008093490590934A05A0934B05B0934C05BD
:10A9B0002093B30B3093B40B4093B50B5093B60B6D
:10A9C0002093AF0B3093B00B4093B10B5093B20B6D
:10A9D0002093AB0B3093AC0B4093AD0B5093AE0B6D
:10A9E0008DE39AE0A7EBBFE38093C60B9093C70B70
:10A9F000A093C80BB093C90B8CEE91E5A6EEB1E421
:10AA00008093FE039093FF03A0930004B09301048E
:10AA100061EE7AE784EF9FE30E9468856093020409
:10AA20007093030480930404909305046FE175E030
:10AA300089ED92E40E947485609306047093070484
:10AA400080930804909309040E94628480E090E05F
:10AA5000A0E8BFE380930A0490930B04A0930C0436
:10AA6000B0930D04E7ECF9E0949108C08091C00028
:10AA700085FFFCCF9093C600319694919923B1F74E
:10AA8000EDECF9E0949108C08091C00085FFFCCF07
:10AA90009093C600319694919923B1F78091C000AC
:10AAA00085FFFCCF8AE08093C600E0960FB6F8944D
:10AAB000DEBF0FBECDBFCF91DF910895CF93DF935F
:10AAC000C7ECD9E0FE01949108C08091C00085FFD9
:10AAD000FCCF9093C600319694919923B1F7E1ECA5
:10AAE000FBE0949108C08091C00085FFFCCF90935B
:10AAF000C600319694919923B1F78091C00085FFEB
:10AB0000FCCF8AE08093C600FE019491E7ECF9E067
:10AB100008C08091C00085FFFCCF9093C60031969D
:10AB200094919923B1F740911505509116056091C4
:10AB300017057091180589EB9BE00E94D35D409149
:10AB4000190550911A0560911B0570911C0586EB43
:10AB50009BE00E94D35D40911D0550911E056091C0
:10AB60001F057091200583EB9BE00E94D35D40910F
:10AB7000210550912205609123057091240580EBF9
:10AB80009BE00E94D35DEFE1F2E007C08091C0003E
:10AB900085FFFCCF31969093C60090819923B1F741
:10ABA0008091C00085FFFCCF8AE08093C600FE0143
:10ABB0009491E7ECF9E008C08091C00085FFFCCFDC
:10ABC0009093C600319694919923B1F7E6E9FBE0A2
:10ABD000949108C08091C00085FFFCCF9093C6007F
:10ABE000319694919923B1F78091C00085FFFCCFF5
:10ABF0008AE08093C600FE019491E7ECF9E008C07A
:10AC00008091C00085FFFCCF9093C600319694914F
:10AC10009923B1F74091050550910605609107050C
:10AC2000709108058DE89BE0BED7409109055091D1
:10AC30000A0560910B0570910C058AE89BE0B3D77B
:10AC400040910D0550910E0560910F057091100512
:10AC500087E89BE0A8D740911105509112056091BB
:10AC600013057091140584E89BE09DD7EFE1F2E0B5
:10AC700007C08091C00085FFFCCF31969093C6003D
:10AC800090819923B1F78091C00085FFFCCF8AE0C5
:10AC90008093C600FE019491E7ECF9E008C0809132
:10ACA000C00085FFFCCF9093C60031969491992304
:10ACB000B1F7E6E6FBE0949108C08091C00085FF03
:10ACC000FCCF9093C600319694919923B1F780916F
:10ACD000C00085FFFCCF8AE08093C600FE019491FE
:10ACE000E7ECF9E008C08091C00085FFFCCF9093AD
:10ACF000C600319694919923B1F740912505509162
:10AD0000260560912705709128058DE59BE05ED7AB
:10AD10004091290550912A0560912B0570912C05D1
:10AD20008AE59BE053D740912D0550912E05609107
:10AD30002F057091300587E59BE048D7409131059C
:10AD400050913205609133057091340584E59BE0A4
:10AD50003DD7EFE1F2E007C08091C00085FFFCCF56
:10AD600031969093C60090819923B1F78091C000ED
:10AD700085FFFCCF8AE08093C600FE019491E7EC4A
:10AD8000F9E008C08091C00085FFFCCF9093C60019
:10AD9000319694919923B1F7EFE1FBE0949108C0CB
:10ADA0008091C00085FFFCCF9093C60031969491AE
:10ADB0009923B1F78091C00085FFFCCF8AE0809392
:10ADC000C600FE019491E7ECF9E008C08091C00054
:10ADD00085FFFCCF9093C600319694919923B1F7EB
:10ADE0004091390550913A0560913B0570913C05C1
:10ADF00086E19BE0D8D640913D0550913E0560919B
:10AE00003F057091400583E19BE0CDD6EFE1F2E094
:10AE100007C08091C00085FFFCCF31969093C6009B
:10AE200090819923B1F78091C00085FFFCCF8AE023
:10AE30008093C600FE019491E7ECF9E008C0809190
:10AE4000C00085FFFCCF9093C60031969491992362
:10AE5000B1F7E0E6FAE0949108C08091C00085FF68
:10AE6000FCCF9093C600319694919923B1F78091CD
:10AE7000C00085FFFCCF8AE08093C600FE0194915C
:10AE8000E7ECF9E008C08091C00085FFFCCF90930B
:10AE9000C600319694919923B1F7409135055091B0
:10AEA0003605609137057091380587E59AE07BD6C5
:10AEB00040914D0550914E0560914F0570915005A0
:10AEC00084E59AE070D640910105509102056091A9
:10AED00003057091040581E59AE078D6409141051B
:10AEE0005091420560914305709144058EE49AE0CB
:10AEF0005AD640914505509146056091470570919D
:10AF000048058BE49AE04FD64091490550914A0597
:10AF100060914B0570914C0588E49AE044D6EFE1CE
:10AF2000F2E007C08091C00085FFFCCF319690937E
:10AF3000C60090819923B1F78091C00085FFFCCFB6
:10AF40008AE08093C600FE019491E7ECF9E008C026
:10AF50008091C00085FFFCCF9093C60031969491FC
:10AF60009923B1F7E6E3FAE0949108C08091C0001C
:10AF700085FFFCCF9093C600319694919923B1F749
:10AF80008091C00085FFFCCF8AE08093C600FE015F
:10AF90009491E7ECF9E008C08091C00085FFFCCFF8
:10AFA0009093C600319694919923B1F74091AB0BE1
:10AFB0005091AC0B6091AD0B7091AE0B8DE29AE0AD
:10AFC000F2D54091AF0B5091B00B6091B10B7091E5
:10AFD000B20B8AE29AE0E7D54091B30B5091B40BE3
:10AFE0006091B50B7091B60B87E29AE0DCD5EFE18A
:10AFF000F2E007C08091C00085FFFCCF31969093AE
:10B00000C60090819923B1F78091C00085FFFCCFE5
:10B010008AE08093C600FE019491E7ECF9E008C055
:10B020008091C00085FFFCCF9093C600319694912B
:10B030009923B1F7E9E1FAE0949108C08091C0004A
:10B0400085FFFCCF9093C600319694919923B1F778
:10B050008091C00085FFFCCF8AE08093C600FE018E
:10B060009491E7ECF9E008C08091C00085FFFCCF27
:10B070009093C600319694919923B1F74091FE03C5
:10B080005091FF0360910004709101048FE09AE0F9
:10B090008AD5609102047091030480910404909118
:10B0A00005040E946E85AB01BC018CE09AE07BD563
:10B0B000609106047091070480910804909109043E
:10B0C0000E947A85AB01BC0189E09AE06CD5EFE182
:10B0D000F2E007C08091C00085FFFCCF31969093CD
:10B0E000C60090819923B1F78091C00085FFFCCF05
:10B0F0008AE08093C600DF91CF9108950F931F934C
:10B10000DF93CF93CDB7DEB766970FB6F894DEBF67
:10B110000FBECDBF80911B0290911C02A0911D0219
:10B12000B0911E028B8B9C8BAD8BBE8BFE013F962C
:10B1300004E610E0F999FECF12BD01BDF89A80B582
:10B1400080830F5F1F4F0836110511F03196F2CF43
:10B15000CE014396BE01615F7F4F43E050E00E9405
:10B16000BC0D009709F096C1E5E1F5E0F999FECF35
:10B1700012BD01BDF89A80B580830F5F1F4F08375D
:10B18000110511F03196F2CFE5E0F5E0F999FECF27
:10B1900012BD01BDF89A80B580830F5F1F4F08383C
:10B1A000110511F03196F2CFE5E2F5E0F999FECF05
:10B1B00012BD01BDF89A80B580830F5F1F4F08391B
:10B1C000110511F03196F2CF0E94031DE9E3F5E07D
:10B1D000F999FECF12BD01BDF89A80B580830F5F4B
:10B1E0001F4F0C39110511F03196F2CFEDE3F5E068
:10B1F000F999FECF12BD01BDF89A80B580830F5F2B
:10B200001F4F003A110511F03196F2CFE5E3F5E05A
:10B21000F999FECF12BD01BDF89A80B580830F5F0A
:10B220001F4F043A110511F03196F2CFEDE4F5E02D
:10B23000F999FECF12BD01BDF89A80B580830F5FEA
:10B240001F4F083A110511F03196F2CFE1E0F5E019
:10B25000F999FECF12BD01BDF89A80B580830F5FCA
:10B260001F4F0C3A110511F03196F2CFE1E4F5E0F1
:10B27000F999FECF12BD01BDF89A80B580830F5FAA
:10B280001F4F003B110511F03196F2CFE5E4F5E0D8
:10B29000F999FECF12BD01BDF89A80B580830F5F8A
:10B2A0001F4F043B110511F03196F2CFE9E4F5E0B0
:10B2B000F999FECF12BD01BDF89A80B580830F5F6A
:10B2C0001F4F083B110511F03196F2CFEBEAFBE07E
:10B2D000F999FECF12BD01BDF89A80B580830F5F4A
:10B2E0001F4F043C110511F03196F2CFFE0131964B
:10B2F000F999FECF12BD01BDF89A80B580830F5F2A
:10B300001F4F063C110599F7FE013396F999FECFC0
:10B3100012BD01BDF89A80B580830F5F1F4F083CB6
:10B32000110511F03196F2CFFE013596F999FECF55
:10B3300012BD01BDF89A80B580830F5F1F4F0A3C94
:10B34000110511F03196F2CFFE013796F999FECF33
:10B3500012BD01BDF89A80B580830F5F1F4F0C3C72
:10B36000110511F03196F2CFFE013996F999FECF11
:10B3700012BD01BDF89A80B580830F5F1F4F0E3C50
:10B38000110511F03196F2CFFE013B96F999FECFEF
:10B3900012BD01BDF89A80B580830F5F1F4F003D3D
:10B3A000110511F03196F2CFE6ECFBE0F999FECFF2
:10B3B00012BD01BDF89A80B580830F5F1F4F043D19
:10B3C000110511F03196F2CFEEEFF3E0F999FECFCF
:10B3D00012BD01BDF89A80B580830F5F1F4F083DF5
:10B3E000110511F03196F2CFE2E0F4E0F999FECFC9
:10B3F00012BD01BDF89A80B580830F5F1F4F0C3DD1
:10B40000110511F03196F2CFE6E0F4E0F999FECFA4
:10B4100012BD01BDF89A80B580830F5F1F4F003EBB
:10B42000110511F03196F2CFFE013D96F999FECF4C
:10B4300012BD01BDF89A80B58083013E110521F04F
:10B44000319601EE10E0F2CF0E946284E7ECF9E061
:10B45000949108C08091C00085FFFCCF9093C600F6
:10B46000319694919923B1F7EFEEF9E0949108C0E9
:10B470008091C00085FFFCCF9093C60031969491D7
:10B480009923B1F78091C00085FFFCCF8AE08093BB
:10B49000C60001C07AD912DB66960FB6F894DEBFFB
:10B4A0000FBECDBFCF91DF911F910F9108950895E9
:10B4B0008091D80B089567707070E82FF0E0E1512B
:10B4C000FB4E84918B3028F48830A0F4863090F1C4
:10B4D00006C08E30D0F08F50833060F521C080914F
:10B4E000B100887F8093B1008091B100862B80935A
:10B4F000B100089580919100887F809391008091A0
:10B500009100862B8093910008958091A100887FFF
:10B510008093A1008091A100862B8093A1000895C3
:10B5200080912101887F8093210180912101862BC8
:10B5300080932101089589ED9BE00C9493380E943B
:10B540004B858091D80B882309F036C081E0809329
:10B55000D80B8091DE0B9091DF0BA091E00BB091A6
:10B56000E10B8093E20B9093E30BA093E40BB09379
:10B57000E50BE7EEFBE0949108C08091C00085FFE9
:10B58000FCCF9093C600319694919923B1F7EEEEDB
:10B59000FBE0949108C08091C00085FFFCCF9093A0
:10B5A000C600319694919923B1F78091C00085FF30
:10B5B000FCCF8AE08093C6000895F8940E944B85E2
:10B5C000179A1092C30B169A1092C40B159A1092E8
:10B5D000C50B149A84E060E00E943393E7EEFBE031
:10B5E000949108C08091C00085FFFCCF9093C60065
:10B5F000319694919923B1F7E4E6FCE0949108C068
:10B600008091C00085FFFCCF9093C6003196949145
:10B610009923B1F78091C00085FFFCCF8AE0809329
:10B62000C600FFCF0E94A2966093E80B7093E90BCF
:10B630008093EA0B9093EB0BE3E8FCE0949108C055
:10B640008091C00085FFFCCF9093C6003196949105
:10B650009923B1F78091C00085FFFCCF8AE08093E9
:10B66000C60008956F927F928F929F92AF92BF9281
:10B67000CF92DF92EF92FF920F931F93F82E60917B
:10B68000F00B7091F10B8091F20B9091F30B2091E4
:10B69000F40B3091F50B4091F60B5091F70B0E9493
:10B6A000B59A3B014C0100D000D00DB71EB70F5F1B
:10B6B0001F4F6091CC037091CD03882777FD809553
:10B6C000982F0E943C992091F9033091FA03409100
:10B6D000FB035091FC030E947A9B20E030E040E79E
:10B6E00052E40E94A19820E030E048EC52E40E942D
:10B6F000A1985B016C01F801608271828282938261
:10B70000F4828091CA0B85838BE99BE06CEF7BE030
:10B7100040EF5BE020E001E032E0E32E0E94FA34EB
:10B720008091FC0B9091FD0BA091FE0BB091FF0B53
:10B7300080939B0B90939C0BA0939D0BB0939E0BBF
:10B740008091000C9091010CA091020CB091030C1F
:10B7500080939F0B9093A00BA093A10BB093A20B8F
:10B760008091040C9091050CA091060CB091070CEF
:10B770008093A30B9093A40BA093A50BB093A60B5F
:10B780008091080C9091090CA0910A0CB0910B0CBF
:10B790008093A70B9093A80BA093A90BB093AA0B2F
:10B7A0008DB79EB706960FB6F8949EBF0FBE8DBF9D
:10B7B0000E94A2966093E80B7093E90B8093EA0BCA
:10B7C0009093EB0B1F910F91FF90EF90DF90CF9034
:10B7D000BF90AF909F908F907F906F9008954F9201
:10B7E0005F926F927F928F929F92AF92BF92CF9211
:10B7F000DF92EF92FF920F931F93DF93CF9300D0CE
:10B800000F92CDB7DEB70E94A2966093E80B7093BB
:10B81000E90B8093EA0B9093EB0B8091FC0B9091DA
:10B82000FD0BA091FE0BB091FF0B89839A83AB8334
:10B83000BC8360919B0B70919C0B80919D0B9091B0
:10B840009E0B29813A814B815C810E949A988823C2
:10B8500009F09EC04090000C5090010C6090020CCA
:10B860007090030C60919F0B7091A00B8091A10BC5
:10B870009091A20BA30192010E949A98882309F04B
:10B8800087C00F920F92CDB6DEB60894C11CD11CB2
:10B89000E090040CF090050C0091060C1091070C40
:10B8A0006091F9037091FA038091FB039091FC037E
:10B8B00020E030E040E752E40E94A1984B015C0197
:10B8C0008AEC9BE0D6018D939C9369817A818B8170
:10B8D0009C81A3019201E8E0CE2EECE0DE2E0E94D6
:10B8E0005F230F900F908091FC0B9091FD0BA09126
:10B8F000FE0BB091FF0B80939B0B90939C0BA0933E
:10B900009D0BB0939E0B8091000C9091010CA09127
:10B91000020CB091030C80939F0B9093A00BA0930B
:10B92000A10BB093A20B8091040C9091050CA091F7
:10B93000060CB091070C8093A30B9093A40BA093DB
:10B94000A50BB093A60B8091080C9091090CA091C7
:10B950000A0CB0910B0C8093A70B9093A80BA093AB
:10B96000A90BB093AA0B0F900F900F900F90CF914F
:10B97000DF911F910F91FF90EF90DF90CF90BF90DC
:10B98000AF909F908F907F906F905F904F900895B1
:10B990000F920F92CDB6DEB60894C11CD11C409018
:10B9A000000C5090010C6090020C7090030CE09021
:10B9B000040CF090050C0091060C1091070C60919E
:10B9C000CC037091CD03882777FD8095982F0E9436
:10B9D0003C992091F9033091FA034091FB03509177
:10B9E000FC030E947A9B20E030E040E752E40E9492
:10B9F000A19820E030E048EC52E40E94A1984B016D
:10BA00005C018AEC9BE0F601918380835ECF84E940
:10BA10009BE00E94894FE6E8FCE0949108C0809189
:10BA2000C00085FFFCCF9093C60031969491992376
:10BA3000B1F74091DE0B5091DF0B6091E00B7091FC
:10BA4000E10B4F5F5F4F6F4F7F4F84E99BE02AE030
:10BA500030E00E9447508091C00085FFFCCF8AE013
:10BA60008093C600DFCD4F925F926F927F928F924C
:10BA70009F92AF92BF92CF92DF92EF92FF920F937D
:10BA80001F934090F9035090FA036090FB0370906D
:10BA9000FC030F2EF0E0AF2EF0EABF2EFCE8CF2E15
:10BAA000F6E4DF2EF02DA092F903B092FA03C092D3
:10BAB000FB03D092FC0360939B0B70939C0B8093D1
:10BAC0009D0B90939E0B20939F0B3093A00B409364
:10BAD000A10B5093A20BE092A30BF092A40B009346
:10BAE000A50B1093A60B0F920F92EAECFBE0ADB7FB
:10BAF000BEB71296FC93EE931197F7EACF2EFBE0B8
:10BB0000DF2E0F2EF0E08F2EF0E09F2EF6E9AF2E05
:10BB1000F3E4BF2EF02D0E945F230F900F900E9440
:10BB20002D134092F9035092FA036092FB03709236
:10BB3000FC031F910F91FF90EF90DF90CF90BF908B
:10BB4000AF909F908F907F906F905F904F900895EF
:10BB50008091F9039091FA03A091FB03B091FC034B
:10BB60008093110C9093120CA093130CB093140CAF
:10BB70008091CC039091CD0390939A0B8093990B75
:10BB800084E690E09093CD038093CC030E94A2962C
:10BB90006093E80B7093E90B8093EA0B9093EB0BA7
:10BBA00081E00C946410FC01949108C08091C00065
:10BBB00085FFFCCF9093C600319694919923B1F7FD
:10BBC00084E99BE022E030E00C944D51FC0194911B
:10BBD00008C08091C00085FFFCCF9093C6003196CD
:10BBE00094919923B1F784E99BE02AE030E00C942A
:10BBF0002B504091170C5091180C20E630E0B90101
:10BC0000469F9001479F300D569F300D1124682F9D
:10BC1000772767FD7095C901875E934F0E94A80D35
:10BC20009C019093160C8093150C80E0232B09F057
:10BC300081E008952F923F924F925F926F927F9290
:10BC40008F929F92AF92BF92CF92DF92EF92FF922C
:10BC50000F931F93DF93CF93CDB7DEB76C970FB6DB
:10BC6000F894DEBF0FBECDBF9E838D8383309105D8
:10BC700008F04AC2FC01E157F14FB4904C01880C26
:10BC8000991C880C991CF401E556F44F80E090E073
:10BC9000A0E0B0E080839183A283B38360919B0B8B
:10BCA00070919C0B80919D0B90919E0B20919F0B0E
:10BCB0003091A00B4091A10B5091A20BE090A30BEF
:10BCC000F090A40B0091A50B1091A60BE7EACE2EE5
:10BCD000EBE0DE2E0E944B1DED81FE81EE0FFF1F7B
:10BCE000EE51FC4F0190F081E02DF7FD10C0CF0127
:10BCF000880F991F8E0F9F1F28EE33E0820E931E30
:10BD0000D4016D917C918752944F0E945C392D80B3
:10BD10003E80220C331C220C331CF101EE56F14FF5
:10BD2000E590F590059114916B2D772767FD70953F
:10BD3000882777FD8095982F0E943C9969837A83A4
:10BD40008B839C83F101E450F44FFC8FEB8FC8018F
:10BD5000B70120E030E040EC5FE30E947A9B29814C
:10BD60003A814B815C810E947A9BAB8DBC8D6D9337
:10BD70007D938D939C931397F101E454FC4FF887C6
:10BD8000EF8360817181828193816093F903709365
:10BD9000FA038093FB039093FC030F920F92CDB6AE
:10BDA000DEB60894C11CD11C4090FC0B5090FD0BDA
:10BDB0006090FE0B7090FF0B2091000C3091010CF5
:10BDC0004091020C5091030C29873A874B875C877E
:10BDD000E090040CF090050C0091060C1091070CFB
:10BDE00020E030E040E752E40E94A1984B015C0162
:10BDF000EAECFBE0D601ED93FC93C301B201298587
:10BE00003A854B855C85B8E0CB2EBCE0DB2E0E94EA
:10BE10005F230F900F900E942D1391012556344FF0
:10BE20003E872D8780E090E0A0E0B0E0F9018083BC
:10BE30009183A283B38360919B0B70919C0B809143
:10BE40009D0B90919E0B20919F0B3091A00B4091E8
:10BE5000A10B5091A20BE090A30BF090A40B0091CA
:10BE6000A50B1091A60BA7EACA2EABE0DA2E0E9412
:10BE70004B1DF101EE53F14F459055906590749034
:10BE8000C301B201905829813A814B815C810E94A3
:10BE90007A9BAB8DBC8D6D937D938D939C93139703
:10BEA0000F920F92CDB6DEB60894C11CD11C209122
:10BEB000FC0B3091FD0B4091FE0B5091FF0B2F8737
:10BEC000388B498B5A8B8091000C9091010CA0917A
:10BED000020CB091030C8B8B9C8BAD8BBE8BE090D6
:10BEE000040CF090050C0091060C1091070C609169
:10BEF000F9037091FA038091FB039091FC0320E019
:10BF000030E040E752E40E94A1984B015C01EAEC6A
:10BF1000FBE0D601ED93FC936F85788989899A8936
:10BF20002B893C894D895E89F8E0CF2EFCE0DF2E1D
:10BF30000E945F230F900F900E942D13C301B20146
:10BF4000A30192010E94C19729813A814B815C81B2
:10BF50000E947A9BAB8DBC8D6D937D938D939C934A
:10BF60001397EF81F885608171818281938120E050
:10BF700030E040E05FE30E947A9B6093F9037093A6
:10BF8000FA038093FB039093FC030F920F92CDB6BC
:10BF9000DEB60894C11CD11C4090FC0B5090FD0BE8
:10BFA0006090FE0B7090FF0B2091000C3091010C03
:10BFB0004091020C5091030C2F8B388F498F5A8F70
:10BFC000E090040CF090050C0091060C1091070C09
:10BFD00020E030E040E752E40E94A1984B015C0170
:10BFE000EAECFBE0D601ED93FC93C301B2012F898B
:10BFF000388D498D5A8DE8E0CE2EECE0DE2E0E9481
:10C000005F230F900F900E942D13F101E256F14F24
:10C010006591759185919491F101E555F44FA0805A
:10C02000B180C280D380A60195010E94C1977B0197
:10C030008C01CB01D801ED85FE8580839183A2839D
:10C04000B383F101E655F14F659175918591949116
:10C0500027EB822E2BE0922E820C931CA6019501D9
:10C060000E94C197D4016D937D938D939C931397F8
:10C07000F101EA54F14F6591759185919491E6ED46
:10C08000F3E02E0E3F1EA60195010E94C197D1013B
:10C090006D937D938D939C931397C701D801EB8D7E
:10C0A000FC8D80839183A283B38320E030E040E065
:10C0B00050E02093F9033093FA034093FB0350932D
:10C0C000FC030E945D10ED81FE81ED53F44F81E091
:10C0D0008083AD81BE81AA0FBB1FFD01EE51FC4FD5
:10C0E0000190F081E02DF7FD0FC0CF01880F991F5F
:10C0F0008E0F9F1FAA0FBB1FA651BC4F6D917C9145
:10C100008752944F0E945C396C960FB6F894DEBF4C
:10C110000FBECDBFCF91DF911F910F91FF90EF9098
:10C12000DF90CF90BF90AF909F908F907F906F9057
:10C130005F904F903F902F9008950F931F93CF9350
:10C14000DF93C2EED3E00AEE13E02881398137FD98
:10C150000CC0C901880F991F820F931FF8016081DD
:10C1600071818752944F0E945C3922960C5F1F4F59
:10C17000F3E0C83EDF0749F7DF91CF911F910F91A0
:10C1800008952F923F924F925F926F927F928F927B
:10C190009F92AF92BF92CF92DF92EF92FF920F9356
:10C1A0001F93DF93CF93CDB7DEB72E970FB6F894DA
:10C1B000DEBF0FBECDBF88E893E00E94E9316091F9
:10C1C000C4037091C5038091C6039091C703609327
:10C1D000F9037093FA038093FB039093FC030F928F
:10C1E0000F92CDB6DEB60894C11CD11CE0909B0B1B
:10C1F000F0909C0B00919D0B10919E0B40909F0B1B
:10C200005090A00B6090A10B7090A20BB7EA2B2E60
:10C21000BBE03B2E20E030E040E752E40E94A198D2
:10C220004B015C01EAECFBE0D601ED93FC93C80105
:10C23000B701A30192010F2EF0E0EF2EF0E0FF2EE8
:10C24000F0E20F2FF1EC1F2FF02D61010E945F2310
:10C250000F900F900E942D1382E00E94CA104B0194
:10C260005C0160919B0B70919C0B80919D0B909158
:10C270009E0B20919F0B3091A00B4091A10B5091F0
:10C28000A20B850174010E944B1D2AEC3EE0F901CE
:10C2900085919591A591B49189839A83AB83BC8351
:10C2A000C501B40129813A814B815C810E94C1970B
:10C2B0006D837E838F8398870F920F92CDB6DEB603
:10C2C0000894C11CD11CE0909B0BF0909C0B00913A
:10C2D0009D0B10919E0B40909F0B5090A00B609077
:10C2E000A10B7090A20B6091F9037091FA038091F9
:10C2F000FB039091FC0320E030E040E752E40E9411
:10C30000A1984B015C01EAECFBE0D601ED93FC93B4
:10C31000C801B701A3019201ED80FE800F8118854D
:10C3200061010E945F230F900F900E942D13609176
:10C33000C4037091C5038091C6039091C70320E0A8
:10C3400030E040E252E40E94A1985B016C016093EE
:10C35000F9037093FA038093FB039093FC030F920D
:10C360000F928DB79EB701969E878D8740909B0B4D
:10C3700050909C0B60909D0B70909E0B80919F0B3A
:10C380009091A00BA091A10BB091A20B89879A87E5
:10C39000AB87BC8769817A818B819C8120E030E00A
:10C3A00040E050EC0E947A9B9B01AC016D817E8144
:10C3B0008F8198850E94C1977B018C01C601B501D0
:10C3C00020E030E040E752E40E94A1984B015C017C
:10C3D000EAECFBE0AD85BE85ED93FC93C301B201B1
:10C3E00029853A854B855C8561010E945F230F900A
:10C3F0000F900E942D1382E00E94CA107B018C01D5
:10C400006093A30B7093A40B8093A50B9093A60B42
:10C4100060919B0B70919C0B80919D0B90919E0B5A
:10C4200020919F0B3091A00B4091A10B5091A20B3A
:10C430000E944B1D2E960FB6F894DEBF0FBECDBFE7
:10C44000CF91DF911F910F91FF90EF90DF90CF90F0
:10C45000BF90AF909F908F907F906F905F904F9024
:10C460003F902F9008956F927F928F929F92AF92FC
:10C47000BF92CF92DF92EF92FF920F931F935B01D7
:10C480006C0139014A0160919B0B70919C0B80916A
:10C490009D0B90919E0B20919F0B3091A00B409192
:10C4A000A10B5091A20BDFDAE090A30BF090A40B4C
:10C4B0000091A50B1091A60BC601B501A401930133
:10C4C000D2DA2091E6033091E70337FD0DC0C901B0
:10C4D000880F991F820F931F6091F0037091F103F1
:10C4E0008752944F0E945C394CDE1091A30B00914F
:10C4F000A40BF090A50BE090A60B2091E6033091E1
:10C50000E70337FD0DC0C901880F991F820F931FE4
:10C510006091F2037091F3038752944F0E945C394B
:10C52000EFEDFEE0949108C08091C00085FFFCCF44
:10C530009093C600319694919923B1F7EAEDFEE00D
:10C54000949108C08091C00085FFFCCF9093C600F5
:10C55000319694919923B1F784E99BE0B601A50146
:10C5600022E030E00E944D51E5EDFEE0949108C0DC
:10C570008091C00085FFFCCF9093C60031969491C6
:10C580009923B1F784E99BE0B401A30122E030E0F4
:10C590000E944D51E0EDFEE0949108C08091C000F2
:10C5A00085FFFCCF9093C600319694919923B1F703
:10C5B00084E99BE0212F302FEF2DFE2DA901BF0133
:10C5C00022E030E00E944D51EEECFEE0949108C074
:10C5D0008091C00085FFFCCF9093C6003196949166
:10C5E0009923B1F7212F302F4F2D5E2DB901CA01AC
:10C5F0001F910F91FF90EF90DF90CF90BF90AF9081
:10C600009F908F907F906F9008958091150C9091DE
:10C61000160C019660E070E04AE050E00C94470C84
:10C620008091150C9091160C019660E070E00C94CE
:10C63000EA0ACF93DF93EC018091CA0B8093DD0B64
:10C6400084E5D7DA882309F481C0EADF0E940E99D5
:10C65000262F6093DD0B662309F478C0E1EEFBE042
:10C66000949108C08091C00085FFFCCF9093C600D4
:10C67000319694919923B1F7CD36D105C1F0CE36DC
:10C68000D10544F4C836D105C1F0C936D10509F049
:10C690004DC010C0CA3DD10539F0CD3DD10509F0DE
:10C6A00045C0E0E2F2E03FC0E7E3F2E031C0EEE493
:10C6B000F2E023C0E5E6F2E015C0ECE7F2E007C0E7
:10C6C0008091C00085FFFCCF31969093C600908189
:10C6D0009923B1F72BC08091C00085FFFCCF319624
:10C6E0009093C60090819923B1F720C08091C0003B
:10C6F00085FFFCCF31969093C60090819923B1F7C6
:10C7000015C08091C00085FFFCCF31969093C60084
:10C7100090819923B1F70AC08091C00085FFFCCFBA
:10C7200031969093C60090819923B1F784E99BE0FC
:10C73000622F40E050E00E9436508091C00085FF9B
:10C74000FCCF8AE08093C60081E001C080E0DF91E9
:10C75000CF910895AF92BF92CF92DF92EF92FF9266
:10C760000F931F93CF93DF936BE9E62E6BE0F62ECA
:10C77000CCEFDBE000E010E0F801E55AFB4F8081F0
:10C7800038DA882331F14CDF5B016C01F801EB569C
:10C79000F44F8081882311F061E002C060910C0C9D
:10C7A00070E0882777FD8095982F0E943C99F701CB
:10C7B00020813181428153810E947A9B9B01AC018F
:10C7C000C601B5010E94C197688379838A839B83E0
:10C7D00009C0F70180819181A281B3818883998307
:10C7E000AA83BB830F5F1F4F84E090E0E80EF91E21
:10C7F00024960430110509F0BFCF86E4FAD98823C6
:10C80000D9F00EDF7B018C0160930D0C70930E0C40
:10C8100080930F0C9093100C20E030E040E050E04B
:10C820000E94A89A181644F4E092F903F092FA03D1
:10C830000093FB031093FC03DF91CF911F910F91A5
:10C84000FF90EF90DF90CF90BF90AF90089582DF80
:10C8500089E4CFD9882351F0E3DE6093F00B709325
:10C86000F10B8093F20B9093F30B0CC080E090E0FF
:10C87000A0E0B0E08093F00B9093F10BA093F20B4B
:10C88000B093F30B8AE4B5D9882351F0C9DE6093E5
:10C89000F40B7093F50B8093F60B9093F70B0895C0
:10C8A00080E090E0A0E0B0E08093F40B9093F50B73
:10C8B000A093F60BB093F70B08958F929F92AF92CF
:10C8C000BF92CF92DF92EF92FF920F931F93CF937D
:10C8D000DF93E0E6CE2ED12CE3EEFEE0A4907AE0EA
:10C8E000972EE9E5FFE0B4908824839421C22D308F
:10C8F00071F02A3321F480919A0D882341F08091C0
:10C900009B0D90919C0D8F3591050CF4EDC1E0913C
:10C910009B0DF0919C0D309719F410929A0D41C225
:10C92000A0919D0DB0919E0DAC9D8001AD9D100D0F
:10C93000BC9D100D1124E00FF11FE75EF34F108234
:10C9400080919A0D882309F0CAC110929A0DA156C0
:10C95000B24F1C92E801C75ED34FCE016EE470E087
:10C960000E94A80D9C01009709F4F7C09093160C43
:10C970008093150C2F5F3F4F2C1B3D0B200F311F59
:10C98000C901875E934F60E070E04AE050E00E948A
:10C99000470C6093A30D7093A40D8093A50D909305
:10C9A000A60DE090DE0BF090DF0B0091E00B1091F4
:10C9B000E10BA80197012F5F3F4F4F4F5F4F621769
:10C9C00073078407950709F4D2C180919D0D90915A
:10C9D0009E0D9C012C9DC0012D9D900D3C9D900DA8
:10C9E0001124875E934F62E070E10E948E0D892BC7
:10C9F00009F0BDC1E7EEFBE0949108C08091C00052
:10CA000085FFFCCF9093C600319694919923B1F79E
:10CA1000EFECFFE0949108C08091C00085FFFCCF4F
:10CA20009093C600319694919923B1F784E99BE0E5
:10CA3000B801A7012AE030E00E9447508091C00071
:10CA400085FFFCCF73C01E274F5FFC01E40FF11D73
:10CA5000E75EF34FE081EA32B1F73093160C209392
:10CA6000150CC901019660E070E00E94EA0A0E947C
:10CA70000999212F30E02617370709F45DC0E7EE4A
:10CA8000FBE0949108C08091C00085FFFCCF90939B
:10CA9000C600319694919923B1F7E0EBFFE09491B1
:10CAA00008C08091C00085FFFCCF9093C6003196EE
:10CAB00094919923B1F74091DE0B5091DF0B609177
:10CAC000E00B7091E10B84E99BE02AE030E00E94EA
:10CAD00047508091C00085FFFCCF28C0E7EEFBE007
:10CAE000949108C08091C00085FFFCCF9093C60050
:10CAF000319694919923B1F7E6E8FFE0949108C04C
:10CB00008091C00085FFFCCF9093C6003196949130
:10CB10009923B1F784E99BE0B801A7012AE030E04E
:10CB20000E9447508091C00085FFFCCF8AE080932F
:10CB3000C6000E94075D4AC08091A30D9091A40D8C
:10CB4000A091A50DB091A60D8093DE0B9093DF0B05
:10CB5000A093E00BB093E10B3EC0CE016AE270E01F
:10CB60000E94A80D009709F436C0E7EEFBE094910F
:10CB700008C08091C00085FFFCCF9093C60031961D
:10CB800094919923B1F7ECE5FFE0949108C080916E
:10CB9000C00085FFFCCF9093C600319694919923F5
:10CBA000B1F74091DE0B5091DF0B6091E00B70917B
:10CBB000E10B84E99BE02AE030E00E94475080913D
:10CBC000C00085FFFCCF8AE08093C60010929C0DC8
:10CBD00010929B0DE6C080919D0D90919E0D8C9DB5
:10CBE00080018D9D100D9C9D100D1124E801C75EE4
:10CBF000D34FCE0167E470E00E94A80D9C0100971E
:10CC000009F441C09093160C8093150C2F5F3F4F91
:10CC10002C1B3D0B200F311FC901875E934F60E035
:10CC200070E00E94EA0A0E9409996430710558F583
:10CC30008091D80B882399F49B2DE9E5FFE008C08B
:10CC40008091C00085FFFCCF9093C60031969491EF
:10CC50009923B1F78091C00085FFFCCF12C09A2DB7
:10CC6000E3EEFEE008C08091C00085FFFCCF90930A
:10CC7000C600319694919923B1F78091C00085FF49
:10CC8000FCCF9092C60080919D0D90919E0D9C01CD
:10CC90002C9DC0012D9D900D3C9D900D1124875E13
:10CCA000934F63E972E00E94B30D009711F40E9464
:10CCB000DD5A80919D0D90919E0D019664E070E08B
:10CCC0000E947F9C90939E0D80939D0D8091E60B1A
:10CCD0009091E70B01969093E70B8093E60B1092EF
:10CCE0009C0D10929B0D24C02B3311F480929A0D51
:10CCF00080919A0D8823E1F420919B0D30919C0D39
:10CD000080919D0D90919E0D8C9DF0018D9DF00D5B
:10CD10009C9DF00D1124E20FF31FE75EF34F80910D
:10CD2000990D80832F5F3F4F30939C0D20939B0D77
:10CD30008091900B9091910B2091920B3091930BDD
:10CD4000821B930B8F779070892B59F18091E60BA2
:10CD50009091E70B04972CF584E99BE00E946B4FC0
:10CD6000282F8093990D8A3009F0C1CDD0CD8091C4
:10CD70009D0D90919E0D8C9DE0018D9DD00D9C9DF3
:10CD8000D00D1124CE01875E934F6AE270E00E94BD
:10CD9000A80D9C01009709F4A1CE10E040E0CE015F
:10CDA00054CEDF91CF911F910F91FF90EF90DF90C4
:10CDB000CF90BF90AF909F908F900895EF92FF9289
:10CDC0000F931F938091E60B9091E70B03970CF460
:10CDD00074DD0E94A296E090EC0BF090ED0B0091B8
:10CDE000EE0B1091EF0B2091E80B3091E90B409185
:10CDF000EA0B5091EB0B621B730B840B950BE61641
:10CE0000F7060807190738F4E114F10401051105C4
:10CE100011F00E94DD5A8091F5039091F603A091E4
:10CE2000F703B091F8030097A105B10559F10E94ED
:10CE3000A2962091E80B3091E90B4091EA0B5091BA
:10CE4000EB0B621B730B840B950B2091F503309158
:10CE5000F6034091F7035091F80326173707480768
:10CE6000590780F49091820A8091830A981751F4AF
:10CE7000179A1092C30B169A1092C40B159A10921F
:10CE8000C50B149A0E943C201F910F91FF90EF90C8
:10CE900008952F923F924F925F926F927F928F925E
:10CEA0009F92AF92BF92CF92DF92EF92FF920F9339
:10CEB0001F93DF93CF93CDB7DEB7CB5CD0400FB6D7
:10CEC000F894DEBF0FBECDBF87E40E94F95D8823D2
:10CED00011F40C94B570A4DB0E9409996C317105B2
:10CEE00009F493C06D3171059CF462307105C9F18C
:10CEF0006330710524F477234CF50C94348263304D
:10CF00007105C1F16430710511F00C9434823EC09A
:10CF10006A35710511F40C9446706B35710554F443
:10CF20006D31710509F485C46E31710511F00C94F1
:10CF30003482DAC76B35710511F40C944A706C3584
:10CF4000710511F00C9434820C944F708091D80BC1
:10CF5000882311F00C943482FDDB0E94EF5B0C946B
:10CF600057828091D80B882311F00C9434826FDCA7
:10CF700081E008C08091D80B882311F00C94348292
:10CF800066DC80E00E94325B0C94578280E50E9450
:10CF9000F95D882321F4EE24FF24870105C040DBDE
:10CFA0000E940E997B018C0183E50E94F95D882324
:10CFB00059F036DB20E030E04AE754E40E947A9BE7
:10CFC0000E940E997B018C010E942D130E94A29653
:10CFD0005B016C01AE0CBF1CC01ED11E0E94A2964C
:10CFE0006093E80B7093E90B8093EA0B9093EB0B43
:10CFF00003C00E949F89E2DE0E94A2966A157B050B
:10D000008C059D05B0F30C94348288E893E00E946F
:10D01000E93184E190E090938203809381038091D1
:10D02000F9039091FA03A091FB03B091FC03809364
:10D03000110C9093120CA093130CB093140C8091CC
:10D04000CC039091CD0390939A0B8093990B84E637
:10D0500090E09093CD038093CC030E94A2966093BE
:10D06000E80B7093E90B8093EA0B9093EB0B81E054
:10D070000E94641080919B0B90919C0BA0919D0B42
:10D08000B0919E0B8093FC0B9093FD0BA093FE0B35
:10D09000B093FF0B80919F0B9091A00BA091A10BDF
:10D0A000B091A20B8093000C9093010CA093020C02
:10D0B000B093030C8091A30B9091A40BA091A50BAE
:10D0C000B091A60B8093040C9093050CA093060CD2
:10D0D000B093070C8091A70B9091A80BA091A90B7E
:10D0E000B091AA0B8093080C9093090CA0930A0CA2
:10D0F000B0930B0C80E090E0A0E0B0E08093F903E7
:10D100009093FA03A093FB03B093FC0388E50E947D
:10D11000F95D882361F489E50E94F95D882339F47B
:10D120008AE50E94F95D882311F481E001C080E066
:10D130008093FD03882329F48AE50E94F95D882302
:10D1400021F082E090E00E941A5E8091FD03882326
:10D1500061F488E50E94F95D882309F483C289E5BA
:10D160000E94F95D882309F47DC280E090E0A0E090
:10D17000B0E080939B0B90939C0BA0939D0BB0937E
:10D180009E0B80939F0B9093A00BA093A10BB09349
:10D19000A20BFFE86F2EFEE07F2EF3018490E0905B
:10D1A000A30BF090A40B0091A50B1091A60BBC0152
:10D1B000CD019B01AC01E7EACE2EEBE0DE2E0E9412
:10D1C0004B1DB2E94B2EBEE05B2EF20165917591CD
:10D1D0008591949120E030E040EC5FE30E947A9BDF
:10D1E0007B018C01992487FC9094AA2497FCA0943D
:10D1F000BA2CC501B4010E943C999B01AC01C80145
:10D20000B7010E947A9B6093FC0B7093FD0B809397
:10D21000FE0B9093FF0BA4E08A2E912C840C951C9E
:10D22000F40165917591859194910894611C711C2C
:10D23000F301D49020E030E040EC5FE30E947A9B61
:10D240007B018C016D2D772767FD7095872F972FB8
:10D250000E943C999B01AC01C801B7010E947A9BD6
:10D260006093000C7093010C8093020C9093030C5C
:10D270002091BC033091BD034091BE035091BF0388
:10D280002093F9033093FA034093FB035093FC037C
:10D29000E090C003F090C1030091C2031091C3035A
:10D2A000C801B7010E949A98882344F4E092F903D8
:10D2B000F092FA030093FB031093FC03F201A59094
:10D2C000B590C590D490F401E590F5900591149136
:10D2D000C601B501A80197010E94A89A18162CF45E
:10D2E000C801B701A601950104C0C601B501A80196
:10D2F00097010E94A1989B01AC010E947A9B9B011F
:10D30000AC01CA0120E030E040E85FE30E94C19731
:10D310000E94E79B9B01AC016091F9037091FA03B5
:10D320008091FB039091FC030E947A9B6093F90328
:10D330007093FA038093FB039093FC030F920F9278
:10D34000CDB6DEB60894C11CD11C4090FC0B5090A9
:10D35000FD0B6090FE0B7090FF0B8091000C909184
:10D36000010CA091020CB091030CC054DF4F8883D4
:10D370009983AA83BB83C05CD040E090040CF090FA
:10D38000050C0091060C1091070C6091F903709147
:10D39000FA038091FB039091FC0320E030E040E72A
:10D3A00052E40E94A1984B015C01FAEC2F2EFBE0A5
:10D3B0003F2ED6012D923C92C301B201C054DF4FE3
:10D3C000288139814A815B81C05CD040E8E0CE2E63
:10D3D000ECE0DE2E0E945F230F900F900E942D1331
:10D3E000EEE9FEE065917591859194912091AB0BEA
:10D3F0003091AC0B4091AD0B5091AE0B0E94C19798
:10D400003B014C0160939B0B70939C0B80939D0B95
:10D4100090939E0BEAEAFEE0659175918591949157
:10D420002091AB0B3091AC0B4091AD0B5091AE0BFA
:10D430000E94C1976093B70B7093B80B8093B90BA0
:10D440009093BA0BE6EBFEE065917591859194910E
:10D450002091AB0B3091AC0B4091AD0B5091AE0BCA
:10D460000E94C1976093D6037093D7038093D8032B
:10D470009093D903E2EAFEE06591759185919491CC
:10D480002091AF0B3091B00B4091B10B5091B20B8A
:10D490000E94C1975B016C0160939F0B7093A00B7E
:10D4A0008093A10B9093A20BEEEAFEE0659175913B
:10D4B000859194912091AF0B3091B00B4091B10BBD
:10D4C0005091B20B0E94C1976093BB0B7093BC0B41
:10D4D0008093BD0B9093BE0BEAEBFEE065917591D6
:10D4E000859194912091AF0B3091B00B4091B10B8D
:10D4F0005091B20B0E94C1976093DA037093DB03E3
:10D500008093DC039093DD03E090A30BF090A40BD9
:10D510000091A50B1091A60BC401B301A6019501C2
:10D52000B7EACB2EBBE0DB2E0E944B1D80919B0BFC
:10D5300090919C0BA0919D0BB0919E0BCC53DF4F13
:10D5400088839983AA83BB83C45CD0408093FC0BFF
:10D550009093FD0BA093FE0BB093FF0B40909F0B9D
:10D560005090A00B6090A10B7090A20B4092000C09
:10D570005092010C6092020C7092030C0F920F9269
:10D58000CDB6DEB60894C11CD11CE090040CF0901E
:10D59000050C0091060C1091070C6091F903709135
:10D5A000FA038091FB039091FC0320E030E040E718
:10D5B00052E40E94A1984B015C01D6012D923C924D
:10D5C000CC53DF4F688179818A819B81C45CD040D4
:10D5D000A3019201A8E0CA2EACE0DA2E0E945F23DC
:10D5E00080E090E0A0E0B0E08093F9039093FA032C
:10D5F000A093FB03B093FC030F900F900E942D1398
:10D600000E945D108091FC0B9091FD0BA091FE0B90
:10D61000B091FF0B80939B0B90939C0BA0939D0B61
:10D62000B0939E0B8091000C9091010CA091020C84
:10D63000B091030C80939F0B9093A00BA093A10B30
:10D64000B093A20B8091040C9091050CA091060C54
:10D65000B091070C8093A30B9093A40BA093A50B00
:10D66000B093A60B8091FD03882329F488E50E94DE
:10D67000F95D882321F080E090E00E941A5E80919D
:10D68000FD03882329F489E50E94F95D882321F0B0
:10D6900081E090E00E941A5E88E50E94F95D88238F
:10D6A000D9F00E9405636115710581059105A1F00E
:10D6B0000E9410632091AB0B3091AC0B4091AD0BED
:10D6C0005091AE0B0E94C19760939B0B70939C0B83
:10D6D00080939D0B90939E0B89E50E94F95D8823B2
:10D6E000D9F00E9405636115710581059105A1F0CE
:10D6F0000E9410632091AF0B3091B00B4091B10BA1
:10D700005091B20B0E94C19760939F0B7093A00B36
:10D710008093A10B9093A20B8AE50E94F95D882368
:10D72000D9F00E9405636115710581059105A1F08D
:10D730000E9410632091B30B3091B40B4091B50B54
:10D740005091B60B0E94C1976093A30B7093A40BEA
:10D750008093A50B9093A60B8091FD03882329F459
:10D760008AE50E94F95D8823D1F06091A30B709146
:10D77000A40B8091A50B9091A60B2091C60B309124
:10D78000C70B4091C80B5091C90B0E94C197609381
:10D79000A30B7093A40B8093A50B9093A60B6091A1
:10D7A0009B0B70919C0B80919D0B90919E0B2091F7
:10D7B0009F0B3091A00B4091A10B5091A20BE090D8
:10D7C000A30BF090A40B0091A50B1091A60BF7EA08
:10D7D000CF2EFBE0DF2E0E944B1D8091110C90910B
:10D7E000120CA091130CB091140C8093F903909338
:10D7F000FA03A093FB03B093FC038091990B9091E3
:10D800009A0B9093CD038093CC030E94A2966093D1
:10D81000E80B7093E90B8093EA0B9093EB0B0E945B
:10D820005D1082E390E090938203809381030C94D7
:10D83000348284E190E0909382038093810380910D
:10D84000C30B882321F08091C40B882329F5E1EED6
:10D85000FBE0949108C08091C00085FFFCCF9093BD
:10D86000C600319694919923B1F7EDE7FEE09491CB
:10D8700008C08091C00085FFFCCF9093C600319610
:10D8800094919923B1F78091C00085FFFCCF8AE085
:10D890008093C6000C9434820E942D1388E893E094
:10D8A0000E94E931CE010D960E94471E6D857E854E
:10D8B0008F85988960939B0B70939C0B80939D0B35
:10D8C00090939E0B29893A894B895C8920939F0B01
:10D8D0003093A00B4093A10B5093A20BED88FE88D0
:10D8E0000F89188DE092A30BF092A40B0093A50B67
:10D8F0001093A60BE7EACE2EEBE0DE2E0E944B1D26
:10D900000E94A85D8091C4039091C503A091C603B5
:10D91000B091C7038093F9039093FA03A093FB039C
:10D92000B093FC03C354DF4F1882CD5BD040222458
:10D930003324E0EAF0E0C754DF4FF983E883C95BA2
:10D94000D040C554DF4F19821882CB5BD040C254FF
:10D95000DF4F19821882CE5BD04028C0C354DF4FFE
:10D96000F881CD5BD040FF2391F421E0C354DF4F19
:10D970002883CD5BD04080EA282E312C80E69FEFB3
:10D98000C754DF4F99838883C95BD0400FC0C3540D
:10D99000DF4F1882CD5BD04022243324A0EAB0E0D0
:10D9A000C754DF4FB983A883C95BD040C254DF4F4F
:10D9B00088819981CE5BD040880F991F880F991F6D
:10D9C000E1E3F0E0EC0FFD1FE80FF91FCB54DF4F50
:10D9D000F983E883C55BD0401FE5412E512C4C0EE6
:10D9E0005D1E480E591EC254DF4F28813981CE5B1F
:10D9F000D040CD54DF4F39832883C35BD040C95416
:10DA0000DF4F19821882C75BD040C554DF4F888131
:10DA10009981CB5BD040AA2797FDA095BA2FC85318
:10DA2000DF4F88839983AA83BB83C85CD040CD54E1
:10DA3000DF4FA881B981C35BD040AB2B29F4EE2422
:10DA4000FF2400EA10E410C06091A30B7091A40BB6
:10DA50008091A50B9091A60B20E030E040EA50E4C5
:10DA60000E94C1977B018C01B101882777FD8095C9
:10DA7000982F0E943C993B014C01C853DF4F6881AD
:10DA800079818A819B81C85CD0400E943C995B016E
:10DA90006C01C401B301A60195010E943362CB540D
:10DAA000DF4FE881F981C55BD04061937193819329
:10DAB0009193CB54DF4FF983E883C55BD040D2010B
:10DAC0006D927D928D929C921397F201A08AB18AF9
:10DAD000C28AD38A80E090E0A0E8BFE380A391A34C
:10DAE000A2A3B3A3CD54DF4F28813981C35BD040BB
:10DAF0002F5F3F4FCD54DF4F39832883C35BD04026
:10DB0000C954DF4F88819981C75BD0400196C954C1
:10DB1000DF4F99838883C75BD040A4E0B0E04A0E12
:10DB20005B1E029749F0C754DF4FE881F981C95B5A
:10DB3000D0402E0E3F1E7BCFC254DF4F288139814B
:10DB4000CE5BD0402E5F3F4FC254DF4F39832883D6
:10DB5000CE5BD040C554DF4F88819981CB5BD040EC
:10DB600080569F4FC554DF4F99838883CB5BD0404D
:10DB70002430310509F0F2CE8091110C9091120CF5
:10DB8000A091130CB091140C8093F9039093FA03B5
:10DB9000A093FB03B093FC038091990B90919A0B97
:10DBA0009093CD038093CC030E94A2966093E80BE0
:10DBB0007093E90B8093EA0B9093EB0B84E090E079
:10DBC00063E070E0AE01415A5F4F9E012F5C3F4F12
:10DBD0000E944F4E4C01E7E6FEE0949108C0809110
:10DBE000C00085FFFCCF9093C60031969491992395
:10DBF000B1F7D4014D915D916D917C9184E99BE0E9
:10DC000022E030E00E944D51E2E6FEE0949108C02F
:10DC10008091C00085FFFCCF9093C600319694910F
:10DC20009923B1F7F401448155816681778184E9B4
:10DC30009BE022E030E00E944D51EDE5FEE0949142
:10DC400008C08091C00085FFFCCF9093C60031963C
:10DC500094919923B1F7D40118964D915D916D91EE
:10DC60007C911B9784E99BE022E030E00E944D51BB
:10DC70008091C00085FFFCCF8AE08093C600B9E1A7
:10DC8000AB2EB12CAC0EBD1EF401408151816281DE
:10DC90007381705804811581268137813058C50100
:10DCA0000F2EF0E0CF2EF0E0DF2EF0E8EF2EFFE3B6
:10DCB000FF2EF02D0E946E30C50168E972E00E94CF
:10DCC000B032AFE8AA2EB12CAC0EBD1EC501C98C76
:10DCD000DA8CEB8CFC8C0D8D1E8D2F8D38A149A11B
:10DCE0005AA16BA17CA10E94C433A8E8B3E0F5015E
:10DCF00084E201900D928150E1F7CE0185960E9459
:10DD0000471E6DA17EA18FA198A560939B0B709378
:10DD10009C0B80939D0B90939E0B29A53AA54BA538
:10DD20005CA520939F0B3093A00B4093A10B5093C5
:10DD3000A20BE090C60BF090C70B0091C80B10919E
:10DD4000C90BE092A30BF092A40B0093A50B1093C8
:10DD5000A60BF7EACF2EFBE0DF2E0E944B1DC4017D
:10DD60000E94E4940E942D1382E00E94B8100E9449
:10DD70003C9920911D0530911E0540911F05509141
:10DD800020050E94A1987B018C0160919B0B7091F2
:10DD90009C0B80919D0B90919E0B20E030E040E029
:10DDA00050E00E94C19769837A838B839C83609142
:10DDB0009F0B7091A00B8091A10B9091A20B20E082
:10DDC00030E040E050E00E94C1976D837E838F83F6
:10DDD00098878091A30B9091A40BA091A50BB09173
:10DDE000A60B89879A87AB87BC872DB73EB72A5287
:10DDF00030400FB6F8943EBF0FBE2DBFEDB7FEB753
:10DE000031969F0148E853E084E2DA010D90AD01BC
:10DE1000D9010D929D018150C1F7CE01019695A3C4
:10DE200084A3CE01059697A386A3CE01099691A758
:10DE300080A70E94753169857A858B859C85A801AC
:10DE400097010E94C0972091A30B3091A40B4091A1
:10DE5000A50B5091A60B0E94C1977B018C01CB01B1
:10DE6000D8018093A30B9093A40BA093A50BB09320
:10DE7000A60BEDB7FEB7BA960FB6F894FEBF0FBE6D
:10DE8000EDBF60919B0B70919C0B80919D0B9091CD
:10DE90009E0B20919F0B3091A00B4091A10B5091B4
:10DEA000A20BE7EACE2EEBE0DE2E0E944B1D82E3B2
:10DEB00090E09093820380938103EFE4FEE09491DD
:10DEC00008C08091C00085FFFCCF9093C6003196BA
:10DED00094919923B1F78091C00085FFFCCF8AE02F
:10DEE0008093C6000C9434822091E6033091E703BE
:10DEF00037FD0DC0C901880F991F820F931F6091D4
:10DF0000F0037091F1038752944F0E945C390E9494
:10DF10002D130E94A85D8091C4039091C503A09128
:10DF2000C603B091C7038093F9039093FA03A093BB
:10DF3000FB03B093FC030E94C160EBE4FEE094910C
:10DF400008C08091C00085FFFCCF9093C600319639
:10DF500094919923B1F7E6E4FEE0949108C0809192
:10DF6000C00085FFFCCF9093C60031969491992311
:10DF7000B1F740919B0B50919C0B60919D0B709160
:10DF80009E0B84E99BE022E030E00E944D51E1E4E9
:10DF9000FEE0949108C08091C00085FFFCCF909373
:10DFA000C600319694919923B1F740919F0B5091FF
:10DFB000A00B6091A10B7091A20B84E99BE022E081
:10DFC00030E00E944D51ECE3FEE0949108C0809156
:10DFD000C00085FFFCCF9093C600319694919923A1
:10DFE000B1F74091A30B5091A40B6091A50B7091D8
:10DFF000A60B84E99BE022E030E00E944D51EAE369
:10E00000FEE0949108C08091C00085FFFCCF909302
:10E01000C600319694919923B1F78091110C90919B
:10E02000120CA091130CB091140C8093F9039093EF
:10E03000FA03A093FB03B093FC038091990B90919A
:10E040009A0B9093CD038093CC030E94A296609389
:10E05000E80B7093E90B8093EA0B9093EB0B209104
:10E06000E6033091E70337FF02C00C943482C90104
:10E07000880F991F820F931F6091F2037091F30331
:10E080008752944F0E945C390C94348210920C0C8D
:10E090000C94348281E080930C0C0C94348285E4DF
:10E0A0000E94F95D882311F40E942D13ABE98A2E9A
:10E0B000ABE09A2EFBEA6F2EFBE07F2EAA24BB2456
:10E0C000F501E55AFB4F80810E94F95D8823E9F153
:10E0D000F3E0AF1669F40E941063D4016D937D9351
:10E0E0008D939C93139787EA9BE00E942E1D2DC071
:10E0F0000E941063F30120813181428153810E948B
:10E10000C197D4016D937D938D939C9313976091E8
:10E110009B0B70919C0B80919D0B90919E0B20917D
:10E120009F0B3091A00B4091A10B5091A20BE0905E
:10E13000A30BF090A40B0091A50B1091A60BE7EA9E
:10E14000CE2EEBE0DE2E0E944B1D0894A11CB11CCC
:10E15000E4E0F0E08E0E9F1E6E0E7F1EF4E0AF1620
:10E16000B10409F0ADCF0C9434828DE40E94F95DC6
:10E17000882311F40C9456810E9410630E9409991F
:10E18000683C710511F40C94CE7A693C71050CF071
:10E190008CC06936710509F472C26A3671050CF0DB
:10E1A00041C06135710509F4C1C662357105DCF401
:10E1B0006F31710509F436C16032710554F4613173
:10E1C000710509F429C16231710511F00C94348292
:10E1D000CBC66A32710509F4D3C16035710511F0FF
:10E1E0000C9434829FC66435710509F4BDC665354B
:10E1F000710554F46235710509F4ADC663357105D6
:10E2000011F00C943482ABC66C35710509F420C74B
:10E210006836710509F4FEC16535710511F00C947D
:10E220003482FBC66337710509F49BC764377105F7
:10E23000DCF46D36710509F446C36E36710554F48D
:10E240006A36710509F431C66B36710511F00C940C
:10E2500034825CC66037710509F4FCC16237710510
:10E2600011F00C9434829FC76837710511F40C9437
:10E27000C8796937710554F46537710509F481C7A8
:10E280006737710511F00C943482C3C06C38710586
:10E2900009F4E4C16E3B710509F4FEC469377105E8
:10E2A00011F00C9434820C94CD7921E06033720724
:10E2B00011F40C94327E31E0613373070CF051C0DD
:10E2C0006C3D710511F40C94257C6D3D710504F5D0
:10E2D0006C3C710511F40C94897B6D3C710564F400
:10E2E000693C710511F40C94487B6B3C710511F08D
:10E2F0000C9434820C946B7B6D3C710511F40C947E
:10E30000A97B6E3C710511F00C9434820C94077C4F
:10E3100081E06831780711F40C94B17C91E06931A7
:10E32000790764F46D3D710511F40C94347C623E00
:10E33000710511F00C9434820C945B7CA1E06E3278
:10E340007A0711F40C94DB7EB1E06F327B0714F096
:10E350000C94EA7E6D52714011F00C9434820C944E
:10E360005F7DF1E0643F7F0711F40C94557F21E05D
:10E37000653F720724F531E06039730711F40C949E
:10E380002A7F81E0613978076CF491E06E35790776
:10E3900011F40C9499806F55714011F00C943482F3
:10E3A0000C94D980B1E061397B0711F40C942D7F76
:10E3B0006259714011F00C9434820C94417FF1E069
:10E3C000673F7F0711F40C945E7F21E0683F72077E
:10E3D0006CF431E0653F730711F40C94587F665F6D
:10E3E000714011F00C9434820C945B7F93E06B3895
:10E3F000790711F40C946A80A3E0673E7A0711F460
:10E400000C9441816355734011F00C9434820C9448
:10E41000617FE4EAF2E0CDC7179816981598149832
:10E420000C9434820E94A2966093D40B7093D50B07
:10E430008093D60B9093D70B2091D00B3091D10BBA
:10E440004091D20B5091D30B621B730B840B950B35
:10E4500028EE33E040E050E00E94929CF22EE32E42
:10E46000D42EC52EEDB7FEB738970FB6F894FEBF81
:10E470000FBEEDBF0DB71EB70F5F1F4FCE018F5BF5
:10E480009F4F928381838BE29EE0D80113969C93E9
:10E490008E931297622F732F842F952F2CE330E0E9
:10E4A00040E050E00E94929CF801358324836F2D58
:10E4B0007E2D8D2D9C2D2CE330E040E050E00E941D
:10E4C000929CD80117967C936E9316970E94CA0D62
:10E4D000E1EEFBE094912DB73EB7285F3F4F0FB6BA
:10E4E000F8943EBF0FBE2DBF08C08091C00085FFCD
:10E4F000FCCF9093C600319694919923B1F7FE0119
:10E50000EF5BFF4F07C08091C00085FFFCCF3196C5
:10E510009093C60090819923B1F78091C00085FF48
:10E52000FCCF8AE08093C60080917105882311F4A6
:10E530000C943482109271058091CA0B082F10E060
:10E54000000F111F0955124FD8016D917C9188273A
:10E5500077FD8095982F0E943C992091B0033091CF
:10E56000B1034091B2035091B3030E94A89A1816C8
:10E5700014F00C943482F801118210820C943482CD
:10E5800083E50E94F95D882311F40C9434820E9483
:10E5900010630E9409997B018C016B0180E50E9448
:10E5A000F95D882369F0F7FC0BC0FFEFEF16F1046B
:10E5B00009F034F40E9410630E9409998B0102C093
:10E5C0000DE010E0EFE5F4E0808191818017910784
:10E5D00011F40C943482329624E0E739F207A1F763
:10E5E0000830110529F4D092CD0BC092CC0B04C099
:10E5F00017FF02C00C943482802F61E00E94339395
:10E60000802F6C2D0E94E693802FB6010E947C958E
:10E610000C94348288E690E00E941963882311F0FC
:10E620000C94348283E50E94F95D882379F00E947E
:10E6300010632091DD0B022F10E0000F111F095510
:10E64000124F0E940999D8016D937C930E944A85CC
:10E650000C9434820E94DD5A0C94348283E50E942B
:10E66000F95D882311F40C9434820E9410630E9497
:10E6700009997093AA0D6093A90D0C94348289E6D0
:10E6800090E00E941963882311F00C943482E5E233
:10E69000FEE0949108C08091C00085FFFCCF90936C
:10E6A000C600319694919923B1F7E091DD0BF0E02B
:10E6B000EE0FFF1FEE0FFF1FE355F24F4081518118
:10E6C0006281738184E99BE021E030E00E944D513A
:10E6D000E2E2FEE0949108C08091C00085FFFCCF8B
:10E6E0009093C600319694919923B1F7E091DD0B98
:10E6F000F0E0EE0FFF1FE955F24F6081718188272E
:10E7000077FD8095982F0E943C99AB01BC0184E96C
:10E710009BE021E030E00E944D51EEE1FEE094915B
:10E7200008C08091C00085FFFCCF9093C600319651
:10E7300094919923B1F74091B30D5091B40D60912C
:10E74000B50D7091B60D84E99BE021E030E00E94A8
:10E750004D51EBE1FEE0949108C08091C00085FF2F
:10E76000FCCF9093C600319694919923B1F76091B4
:10E77000A90D7091AA0D882777FD8095982F0E948A
:10E780003C99AB01BC0184E99BE021E030E00E94B0
:10E790004D51E8E1FEE0949108C08091C00085FFF2
:10E7A000FCCF9093C600319694919923B1F784E9F8
:10E7B0009BE060E070E04AE050E00E947A50E6E1C1
:10E7C000FEE0949108C08091C00085FFFCCF90933B
:10E7D000C600319694919923B1F74091AD0D5091B7
:10E7E000AE0D6091AF0D7091B00D84E99BE021E01A
:10E7F00030E00E944D51E3E1FEE0949108C0809129
:10E80000C00085FFFCCF9093C60031969491992368
:10E81000B1F76091A70D7091A80D882777FD8095BD
:10E82000982F0E943C99AB01BC0184E99BE021E058
:10E8300030E00E944D51EFE0FEE0949108C08091DD
:10E84000C00085FFFCCF9093C60031969491992328
:10E85000B1F78091DD0B0E948F84BC0184E99BE0BD
:10E860004AE050E00E947A50EAE0FEE0949108C04D
:10E870008091C00085FFFCCF9093C60031969491A3
:10E880009923B1F78FEF9FEF0E948F84BC0184E939
:10E890009BE04AE050E00E947A50EDEBF2E007C0C6
:10E8A0008091C00085FFFCCF31969093C600908187
:10E8B0009923B1F78091C00085FFFCCF8AE0809357
:10E8C000C6000C9457828DE690E00E94196388235D
:10E8D00011F00C9434821092710583E50E94F95D69
:10E8E000882399F00E9410632091DD0B022F10E025
:10E8F000000F111F0955124F0E940999F8017183E9
:10E90000608381E08093F40316C082E50E94F95D84
:10E91000882389F00E9410632091DD0B022F10E004
:10E92000000F111F0955124F0E940999D8016D93CC
:10E930007C931092F40383E50E94F95D882351F0E3
:10E940000E9410636093B0037093B1038093B2038D
:10E950009093B30382E40E94F95D882351F00E94F2
:10E9600010636093AC037093AD038093AE039093F8
:10E97000AF0386E40E94F95D882369F00E9410636A
:10E980006093B4037093B5038093B6039093B70379
:10E9900081E0809371050E944A850E94A2964B01F6
:10E9A0005C012091DD0B022F10E01092DC0B000FB8
:10E9B000111FF801E955F24F60817181882777FDB9
:10E9C0008095982F0E943C99000F111F0355124FFC
:10E9D000F80120813181428153810E94A89A181642
:10E9E0001CF481E08093DC0BCC24CA94DC2C7601EF
:10E9F000E7E0FEE05490E3E0FEE06490EFEFFDE03E
:10EA000074906AE0462E3BC1952DE7E0FEE008C019
:10EA10008091C00085FFFCCF9093C6003196949101
:10EA20009923B1F7E091DD0BF0E0EE0FFF1FEE0F41
:10EA3000FF1FE355F24F408151816281738184E968
:10EA40009BE021E030E00E944D51962DE3E0FEE096
:10EA500008C08091C00085FFFCCF9093C60031961E
:10EA600094919923B1F76091DD0B84E99BE070E00C
:10EA70004AE050E00E947A50972DEFEFFDE008C089
:10EA80008091C00085FFFCCF9093C6003196949191
:10EA90009923B1F7F7FE03C0EEEBF2E02CC00E9421
:10EAA000A2966C197D098E099F090E943A999B01D3
:10EAB000AC0160E070E08AEF93E40E94C09720E030
:10EAC00030E04AE754E40E94A1980E940E99AB01FD
:10EAD000BC0184E99BE02AE030E00E942B50809149
:10EAE000C00085FFFCCF0EC08091C00085FFFCCF29
:10EAF00031969093C60090819923B1F78091C00020
:10EB000085FFFCCF4092C6000E94A2964B015C019B
:10EB10000E949F890E94DE66FFEFCF16FFEFDF069F
:10EB2000FFEFEF06FFEFFF0609F052C08091DC0B0C
:10EB3000E091DD0B882331F1F0E08F01000F111F10
:10EB4000000F111F0355124FEE0FFF1FE955F24F33
:10EB500060817181882777FD8095982F0E943C996C
:10EB600020E030E040E251E40E94C0979B01AC01FC
:10EB7000D8016D917D918D919C910E94A89A87FFFB
:10EB800058C05EC0F0E08F01000F111F000F111F71
:10EB90000355124FEE0FFF1FE955F24F608171814F
:10EBA000882777FD8095982F0E943C9920E030E0DF
:10EBB00040E251E40E94C1979B01AC01F8016081E1
:10EBC0007181828193810E949A98181694F538C0B9
:10EBD000F7FC36C0E091DD0BF0E08F01000F111F54
:10EBE000000F111F0355124FEE0FFF1FE955F24F93
:10EBF00060817181882777FD8095982F0E943C99CC
:10EC00009B01AC01D8016D917D918D919C910E94E9
:10EC1000C0970E94099997FF07C0909580957095BD
:10EC200061957F4F8F4F9F4F6B3071058105910527
:10EC30003CF00E94A296AC01CB01DA016C017D018F
:10EC4000BFEFCB16BFEFDB06BFEFEB06BFEFFB0658
:10EC5000B1F0F7FE02C00C9437820E94A2966C19A4
:10EC60007D0980E090E00E943A9920E030E04AEF90
:10EC700053E40E949A98882314F00C9437820E94DF
:10EC8000A296681979098A099B09695E73408040D8
:10EC9000904008F0B9CE3CCF83E50E94F95D88230F
:10ECA00061F00E9410630E9409997093AA0D60930D
:10ECB000A90D81E08093F4030FC082E50E94F95D05
:10ECC000882351F00E9410630E9409997093AA0D45
:10ECD0006093A90D1092F4030E94A2967B018C010F
:10ECE0001092DC0B6091A90D7091AA0D882777FD19
:10ECF0008095982F0E943C992091B30D3091B40DCE
:10ED00004091B50D5091B60D0E94A89A18160CF0BE
:10ED100080C081E08093DC0B7CC00E94A2966E19BB
:10ED20007F09800B910B695E73408040904008F42E
:10ED30006BC0E091CA0BF0E0EE0FFF1FEE0FFF1F5C
:10ED4000E355F24F40815181628173819B2DECEF3D
:10ED5000FDE008C08091C00085FFFCCF9093C60005
:10ED6000319694919923B1F784E99BE022E030E059
:10ED70000E944D519C2DE8EFFDE008C08091C0003D
:10ED800085FFFCCF9093C600319694919923B1F7FB
:10ED90006091CA0B84E99BE070E04AE050E00E9479
:10EDA0007A509D2DE4EFFDE008C08091C00085FF02
:10EDB000FCCF9093C600319694919923B1F740917E
:10EDC000B30D5091B40D6091B50D7091B60D84E9FD
:10EDD0009BE021E030E00E944D51EDEBF2E007C0F6
:10EDE0008091C00085FFFCCF31969093C600908142
:10EDF0009923B1F78091C00085FFFCCFA092C60097
:10EE00000E94A2967B018C010E949F890E94DE666F
:10EE10000BC0ECEFFDE0B490E8EFFDE0C490E4EF50
:10EE2000FDE0D4907AE0A72E8091DC0B2091A90D13
:10EE30003091AA0D8823A9F0B901882777FD809524
:10EE4000982F0E943C992091B30D3091B40D4091C0
:10EE5000B50D5091B60D0E94A89A18160CF45DCF0E
:10EE600018C0B901882777FD8095982F0E943C999A
:10EE70002091B30D3091B40D4091B50D5091B60D68
:10EE80000E949A9888232CF48091F403882309F433
:10EE900044CF0E94A2966093E80B7093E90B809395
:10EEA000EA0B9093EB0B0C94348283E50E94F95D9E
:10EEB000882321F10E94106320E030E040E050E020
:10EEC0000E949A9888231CF460E070E011C00E94B0
:10EED000106320E030E04FE753E40E94A89A181630
:10EEE0001CF46FEF70E004C00E9410630E94099947
:10EEF0007093CD0B6093CC0B0C9434828FEF90E029
:10EF00009093CD0B8093CC0B0C9434821092CB0B4E
:10EF10001092CD0B1092CC0B1092CF0B1092CE0B07
:10EF20000C9434829D9AA5980C9434820E944B854F
:10EF30000E942D13149A0E9439131092CD0B109237
:10EF4000CC0B68EE73E080E090E00E94B0969D9A52
:10EF5000A59A0C9434821092980B0C94348281E020
:10EF60008093980B0C94348283E50E94F95D88238A
:10EF7000A1F00E94106320E030E04AE754E40E94D0
:10EF80007A9B0E940E996093F5037093F603809329
:10EF9000F7039093F8030C94348288E50E94F95D9E
:10EFA000882311F00C944C8289E50E94F95D882336
:10EFB00011F00C944C828AE50E94F95D882311F0CF
:10EFC0000C944C8285E40E94F95D882311F00C9426
:10EFD0004C820E942D13149A0E9439130C9434828F
:10EFE000179A1092C30B89E50E94F95D882319F0E6
:10EFF000169A1092C40B8AE50E94F95D882319F0D5
:10F00000159A1092C50B85E40E94F95D882311F4CE
:10F010000C943482149A0C94348283E50E94F95D36
:10F02000882311F40C9434820E94106320E030E0B5
:10F030004AE754E40E947A9B0E940E996093EC0B7D
:10F040007093ED0B8093EE0B9093EF0B0C94348246
:10F0500065E1662E65E0762E55E0252E55E0352ECD
:10F0600041E5442E45E0542E88249924F401E55AC4
:10F07000FB4F80810E94F95D882309F460C023E082
:10F08000821609F054C00E9410635B016C0120E0FD
:10F0900030E040EA51E40E949A9888230CF041C085
:10F0A000D3016D917D918D919C91A60195010E9456
:10F0B000A1987B018C016091490570914A0580916E
:10F0C0004B0590914C05A80197010E947A9B609393
:10F0D000490570934A0580934B0590934C05F101C7
:10F0E0006081718182819381A80197010E947A9B3E
:10F0F000D1016D937D938D939C931397F201608161
:10F100007181828193810E943A99A80197010E949E
:10F110007A9B0E940E99D2016D937D938D939C935F
:10F120001397F301A082B182C282D38208C00E94E9
:10F130001063D3016D937D938D939C9313970894E3
:10F14000811C911CE4E0F0E06E0E7F1E2E0E3F1E2F
:10F150004E0E5F1EF4E08F16910409F087CF0C94D9
:10F160003482E7E2FDE0949108C08091C00085FF01
:10F17000FCCF9093C600319694919923B1F70C94EB
:10F1800034828091150C9091160C05966AE270E01D
:10F190000E94A80DFC01009711F40C943482319761
:10F1A00010820C943482E4E2FDE0949108C08091D6
:10F1B000C00085FFFCCF9093C600319694919923AF
:10F1C000B1F740919B0B50919C0B60919D0B7091FE
:10F1D0009E0B84E99BE022E030E00E944D51E0E28A
:10F1E000FDE0949108C08091C00085FFFCCF909312
:10F1F000C600319694919923B1F740919F0B50919D
:10F20000A00B6091A10B7091A20B84E99BE022E01E
:10F2100030E00E944D51ECE1FDE0949108C08091F6
:10F22000C00085FFFCCF9093C6003196949199233E
:10F23000B1F74091A30B5091A40B6091A50B709175
:10F24000A60B84E99BE022E030E00E944D51E8E10A
:10F25000FDE0949108C08091C00085FFFCCF9093A1
:10F26000C600319694919923B1F74091A70B509124
:10F27000A80B6091A90B7091AA0B84E99BE022E096
:10F2800030E00E944D51EDE0FDE0949108C0809186
:10F29000C00085FFFCCF9093C600319694919923CE
:10F2A000B1F780E00E94B8100E943C9920911505AA
:10F2B0003091160540911705509118050E94A198AC
:10F2C000AB01BC0184E99BE022E030E00E944D519B
:10F2D000E9E0FDE0949108C08091C00085FFFCCF7B
:10F2E0009093C600319694919923B1F781E00E94E2
:10F2F000B8100E943C992091190530911A0540914F
:10F300001B0550911C050E94A198AB01BC0184E92A
:10F310009BE022E030E00E944D51E5E0FDE0949159
:10F3200008C08091C00085FFFCCF9093C600319645
:10F3300094919923B1F782E00E94B8100E943C9901
:10F3400020911D0530911E0540911F05509120050B
:10F350000E94A198AB01BC0184E99BE022E030E06F
:10F360000E944D51EDEBF2E007C08091C00085FF97
:10F37000FCCF31969093C60090819923B1F780918C
:10F38000C00085FFFCCF8AE08093C6000C943482D5
:10F3900080E00E9464100C94348281E00E9464102A
:10F3A0000C9434828091C00085FFFCCF31969093FD
:10F3B000C60090819923B1F78091C00085FFFCCFF2
:10F3C0008AE08093C600EDEFFCE0949108C0809144
:10F3D000C00085FFFCCF9093C6003196949199238D
:10F3E000B1F71E9B03C0E0ECF2E00AC0E5ECF2E0EE
:10F3F00007C08091C00085FFFCCF31969093C60076
:10F4000090819923B1F78091C00085FFFCCF8AE0FD
:10F410008093C600E5EFFCE0949108C08091C000A5
:10F4200085FFFCCF9093C600319694919923B1F754
:10F43000379B03C0E0ECF2E00AC0E5ECF2E007C065
:10F440008091C00085FFFCCF31969093C6009081DB
:10F450009923B1F78091C00085FFFCCF8AE08093AB
:10F46000C600EDEEFCE0949108C08091C00085FFDD
:10F47000FCCF9093C600319694919923B1F71D9BD0
:10F4800003C0E0ECF2E00AC0E5ECF2E007C08091D6
:10F49000C00085FFFCCF31969093C60090819923E0
:10F4A000B1F78091C00085FFFCCF8AE08093C60051
:10F4B000E5EEFCE0949108C08091C00085FFFCCF90
:10F4C0009093C600319694919923B1F7029B03C0A3
:10F4D000E0ECF2E00AC0E5ECF2E007C08091C00089
:10F4E00085FFFCCF31969093C60090819923B1F7A8
:10F4F0008091C00085FFFCCF8AE08093C600EDEDCF
:10F50000FCE0949108C08091C00085FFFCCF9093EF
:10F51000C600319694919923B1F71C9B03C0E0EC8F
:10F52000F2E00AC0E5ECF2E007C08091C00085FF80
:10F53000FCCF31969093C60090819923B1F78091CA
:10F54000C00085FFFCCF8AE08093C600E5EDFCE0BB
:10F55000949108C08091C00085FFFCCF9093C600B5
:10F56000319694919923B1F7019B03C0E0ECF2E04E
:10F570000AC0E5ECF2E007C08091C00085FFFCCF37
:10F5800031969093C60090819923B1F78091C00085
:10F5900085FFFCCF8AE08093C60066C784E40E94A2
:10F5A000F95D882309F460C70E94106320E030E011
:10F5B00040E05FE30E947A9B7B018C0120E030E019
:10F5C00040E050E00E949A98882359F40F2EF0E012
:10F5D000CF2EF0E0DF2EF0E8EF2EFFE3FF2EF02D30
:10F5E00011C0C801B701A80197010E947A9B9B0135
:10F5F000AC01CA012BED3FE049E450E40E947A9B44
:10F600006B017C018091CA0B8093DD0B84E50E9425
:10F61000F95D882321F10E9410630E940E99609386
:10F62000DD0B6623E1F0E1EEFBE0949108C08091F0
:10F63000C00085FFFCCF9093C6003196949199232A
:10F64000B1F7EFECF2E007C08091C00085FFFCCF7E
:10F6500031969093C60090819923B1F705C78091A8
:10F66000DD0B082F10E0000F111F000F111F0E52AD
:10F670001C4F60E070E080E89FE3A70196010E94C4
:10F68000A198D8016D937D938D939C931397ECC6AD
:10F690000BE514E025E2E22E25E0F22EF801808150
:10F6A0000E94F95D882351F00E9410630E940E9918
:10F6B000D7016D937D938D939C9313970F5F1F4F8D
:10F6C000E4E0F0E0EE0EFF1EF4E00F351F0731F727
:10F6D0000E94031DC9C60BE514E095E0E92E95E0F4
:10F6E000F92ED8018C910E94F95D882339F00E948F
:10F6F0001063F70160837183828393830F5F1F4FD1
:10F7000024E030E0E20EF31E34E00F35130749F732
:10F71000ABC683E50E94F95D882351F00E94106317
:10F720006093390570933A0580933B0590933C05AF
:10F7300084E50E94F95D882309F496C60E9410634F
:10F7400060933D0570933E0580933F05909340057F
:10F750008BC683E50E94F95D882351F00E941063F7
:10F76000609335057093360580933705909338057F
:10F7700084E50E94F95D882351F00E941063609334
:10F780004D0570934E0580934F059093500582E48C
:10F790000E94F95D882361F00E9410630E940E9917
:10F7A000609301057093020580930305909304050F
:10F7B00088E50E94F95D882351F00E9410636093F0
:10F7C00041057093420580934305909344058AE573
:10F7D0000E94F95D882351F00E94106360934505F3
:10F7E00070934605809347059093480585E40E94F1
:10F7F000F95D882309F438C60E94106360934905B7
:10F8000070934A0580934B0590934C052DC60BE5EC
:10F8100014E08BEAE82E8BE0F82ED8018C910E9440
:10F82000F95D882339F00E941063F70160837183CA
:10F83000828393830F5F1F4F24E030E0E20EF31EBC
:10F8400034E00E35130749F70FC683E50E94F95DD2
:10F85000882309F409C60E9410630E9409997093D5
:10F86000CD036093CC0300C683E50E94F95D882335
:10F8700009F4FAC50E9410630E9409997B018C016A
:10F8800084E50E94F95D882389F08DED90E00E9467
:10F890001963882309F0E8C5E091DD0BF0E0EE0F75
:10F8A000FF1FE053FC4FF182E082DEC5F092CF03F0
:10F8B000E092CE03D9C580E50E94F95D882309F462
:10F8C000D3C50E9410630E9409997B0183E50E94C1
:10F8D000F95D882319F40FEF1FEF05C00E94106334
:10F8E0000E9409998B01C8010196039708F0BCC5D5
:10F8F000EFE5F4E0808191818E159F0509F4B4C590
:10F90000329684E0E739F807A9F7F7FCADC50E9405
:10F910002D13DE2C8E2D60E00E943393011511050E
:10F9200041F00130110579F09FEF0F3F190791F475
:10F9300003C000E010E00EC08E2D0E94189400E07D
:10F9400010E0892B39F401E010E004C00E949F8987
:10F950000E94DE668D2D0E94189480179107B1F7E2
:10F9600083C580E50E94F95D882319F40FEF1FEF2E
:10F9700005C00E9410630E9409998B0183E50E94D3
:10F98000F95D882309F446C00E9410630115110532
:10F9900051F40E9409999B01AC0189ED9BE0B901EA
:10F9A0000E945C3961C5E1EEFBE0949108C0809152
:10F9B000C00085FFFCCF9093C600319694919923A7
:10F9C000B1F7E6EEF2E007C08091C00085FFFCCF02
:10F9D00031969093C60090819923B1F784E99BE01A
:10F9E000B8014AE050E00E947A50EDEEF2E007C024
:10F9F0008091C00085FFFCCF31969093C600908126
:10FA00009923B1F78091C00085FFFCCF8AE08093F5
:10FA1000C6002AC517FD28C5EBEFF2E007C08091AC
:10FA2000C00085FFFCCF31969093C600908199234A
:10FA3000B1F7EEEFF2E007C08091C00085FFFCCF88
:10FA400031969093C60090819923B1F784E99BE0A9
:10FA5000B8014AE050E00E947A50E6E0F3E007C0C7
:10FA60008091C00085FFFCCF31969093C6009081B5
:10FA70009923B1F7C801880F991F800F911F8752F2
:10FA8000944F0E940839BC0184E99BE04AE050E0B1
:10FA90000E947A50EDEBF2E007C08091C00085FF34
:10FAA000FCCF31969093C60090819923B1F7809155
:10FAB000C00085FFFCCF8AE08093C600D5C480E5F6
:10FAC0000E94F95D882351F00E9410636093FE0349
:10FAD0007093FF03809300049093010489E40E94D3
:10FAE000F95D882359F00E941063F2D760930204F5
:10FAF00070930304809304049093050484E40E94AB
:10FB0000F95D882359F00E941063EED760930604D4
:10FB100070930704809308049093090483E40E947F
:10FB2000F95D882351F00E94106360930A0470937A
:10FB30000B0480930C0490930D04C4D6EBEFF2E019
:10FB400007C08091C00085FFFCCF31969093C6001E
:10FB500090819923B1F7E9E0F3E007C08091C000FC
:10FB600085FFFCCF31969093C60090819923B1F721
:10FB70004091FE035091FF036091000470910104D5
:10FB800084E99BE022E030E00E944D51EDE0F3E09B
:10FB900007C08091C00085FFFCCF31969093C600CE
:10FBA00090819923B1F760910204709103048091D0
:10FBB00004049091050492D7AB01BC0184E99BE059
:10FBC00022E030E00E944D51E1E1F3E007C0809176
:10FBD000C00085FFFCCF31969093C6009081992399
:10FBE000B1F7609106047091070480910804909128
:10FBF000090480D7AB01BC0184E99BE022E030E03E
:10FC00000E944D51E5E1F3E007C08091C00085FFFF
:10FC1000FCCF31969093C60090819923B1F7409123
:10FC20000A0450910B0460910C0470910D0484E956
:10FC30009BE022E030E00E944D51EDEBF2E007C086
:10FC40008091C00085FFFCCF31969093C6009081D3
:10FC50009923B1F78091C00085FFFCCF8AE08093A3
:10FC6000C60002C480E50E94F95D882351F00E941D
:10FC7000106360930E0470930F04809310049093AC
:10FC8000110489E40E94F95D882359F00E941063F1
:10FC90001FD76093120470931304809314049093FD
:10FCA000150484E40E94F95D882359F00E941063D2
:10FCB0001BD76093160470931704809318049093D5
:10FCC000190400D6EBEFF2E007C08091C00085FF79
:10FCD000FCCF31969093C60090819923B1F7E9E06B
:10FCE000F3E007C08091C00085FFFCCF3196909370
:10FCF000C60090819923B1F740910E0450910F04F2
:10FD0000609110047091110484E99BE022E030E0DE
:10FD10000E944D51EDE0F3E007C08091C00085FFE7
:10FD2000FCCF31969093C60090819923B1F76091F2
:10FD30001204709113048091140490911504CED68E
:10FD4000AB01BC0184E99BE022E030E00E944D5110
:10FD5000E1E1F3E007C08091C00085FFFCCF319660
:10FD60009093C60090819923B1F760911604709129
:10FD700017048091180490911904BCD6AB01BC0102
:10FD800084E99BE022E030E00E944D51EDEBF2E08F
:10FD900007C08091C00085FFFCCF31969093C600CC
:10FDA00090819923B1F78091C00085FFFCCF8AE054
:10FDB0008093C60059C383E50E94F95D882329F426
:10FDC00060E070E080E090E002C00E9410630E945A
:10FDD000FA1C4AC385E40E94F95D882319F4CC24F7
:10FDE000DD2412C00E9410630E9409996B0177FF05
:10FDF0000BC00F2EF0E0EF2EF0E0FF2EFCE80F2FEF
:10FE0000F2E41F2FF02D0AC00F2EF0E0EF2EF0E0ED
:10FE1000FF2EF6E10F2FF3E41F2FF02D83E50E9454
:10FE2000F95D882321F00E9410637B018C0183E43B
:10FE30000E94F95D882319F425E030E005C00E9496
:10FE400010630E9409999B01C801B701A6010E9495
:10FE50003D8C0AC30E942D1307C32091E603309105
:10FE6000E70337FD01C3C901880F991F820F931F54
:10FE70006091F0037091F1038752944F0E945C39B6
:10FE8000F3C22091E6033091E70337FDEDC2C901CB
:10FE9000880F991F820F931F6091F2037091F303F3
:10FEA0008752944F0E945C39DFC20E944F51DCC2DE
:10FEB0000E947E58D9C20E94C553D6C20E945E5588
:10FEC000D3C28AE50E94F95D882309F4BCC00E9470
:10FED00010637B018C0120E030E040E050EC0E9498
:10FEE000A89A88230CF44EC0C801B70120E030E086
:10FEF00040EA50E40E949A9818160CF443C0D801C6
:10FF0000C701B0588093C60B9093C70BA093C80B42
:10FF1000B093C90BE1EEFBE0949108C08091C00062
:10FF200085FFFCCF9093C600319694919923B1F749
:10FF3000E9ECFCE0949108C08091C00085FFFCCF03
:10FF40009093C600319694919923B1F78091C000A7
:10FF500085FFFCCF8AE08093C600EDEBF2E007C09E
:10FF60008091C00085FFFCCF31969093C6009081B0
:10FF70009923B1F78091C00085FFFCCF8AE0809380
:10FF8000C60072C2E1EEFBE0949108C08091C0000F
:10FF900085FFFCCF9093C600319694919923B1F7D9
:10FFA000E0ECFCE0949108C08091C00085FFFCCF9C
:10FFB0009093C600319694919923B1F7E8EBFCE059
:10FFC000949108C08091C00085FFFCCF9093C6003B
:10FFD000319694919923B1F784E99BE040E050E099
:10FFE00060E070EC22E030E00E944D51E0EBFCE07C
:10FFF000949108C08091C00085FFFCCF9093C6000B
:020000021000EC
:10000000319694919923B1F784E99BE040E050E068
:1000100060EA70E422E030E00E944D51EDEBF2E046
:1000200007C08091C00085FFFCCF31969093C60039
:1000300090819923B1F78091C00085FFFCCF8AE0C1
:100040008093C60011C2E1EEFBE0949108C080915C
:10005000C00085FFFCCF9093C60031969491992300
:10006000B1F7E4EAFCE0949108C08091C00085FFFC
:10007000FCCF9093C600319694919923B1F780916B
:10008000C00085FFFCCF8AE08093C6004091C60B7C
:100090005091C70B6091C80B7091C90B705884E9DF
:1000A0009BE022E030E00E944D51EDEBF2E007C012
:1000B0008091C00085FFFCCF31969093C60090815F
:1000C0009923B1F78091C00085FFFCCF8AE080932F
:1000D000C600CAC188E50E94F95D882351F00E94DC
:1000E00010630E9409999B01AC0180E0B9010E9454
:1000F00058128AE50E94F95D882351F00E9410632E
:100100000E9409999B01AC0181E0B9010E9458123B
:1001100085E40E94F95D882309F4A6C10E9410635A
:100120000E9409999B01AC0182E0B9010E9458121A
:100130009BC183E50E94F95D882319F400E010E07B
:100140000FC010E00E9410630E940E999B01AC0149
:10015000812F622F0E9403121F5F153099F7EECF97
:10016000F801E55AFB4F80810E94F95D882351F028
:100170000E9410630E940E999B01AC01802F622F98
:100180000E9403120F5F1F4F0430110549F782E4EC
:100190000E94F95D882351F00E9410630E940E991D
:1001A0009B01AC0184E0622F0E9403120E94E910BF
:1001B0005BC183E50E94F95D882309F45FC00E945A
:1001C00010630E9409996130710529F06230710550
:1001D00009F054C029C000E010E0F801E55AFB4FD7
:1001E00080810E94F95D882359F00E9410630E946B
:1001F00009999B01AC01802F622F4FEF0E94C5111E
:100200000F5F1F4F0430110541F782E40E94F95D32
:100210008823A1F10E9410630E9409999B01AC01FF
:1002200084E0622F4FEF28C000E010E0F801E55AAB
:10023000FB4F80810E94F95D882359F00E94106372
:100240000E9409999B01AC01802F6FEF422F0E9401
:10025000C5110F5F1F4F0430110541F782E40E9462
:10026000F95D882359F00E9410630E9409999B014F
:10027000AC0184E06FEF422F0E94C5110E94E9108B
:10028000F3C01092D80B8091E20B9091E30BA091F8
:10029000E40BB091E50B8093DE0B9093DF0BA09302
:1002A000E00BB093E10B0E94075DDEC084E50E9485
:1002B000F95D882309F48DC00E9410630E940E9995
:1002C000262F6093DD0B6623B9F1E1EEFBE09491FC
:1002D00008C08091C00085FFFCCF9093C600319686
:1002E00094919923B1F7E9E1F3E007C08091C00050
:1002F00085FFFCCF31969093C60090819923B1F78A
:1003000084E99BE0622F40E050E00E943650EBE130
:10031000F3E007C08091C00085FFFCCF3196909339
:10032000C60090819923B1F78091C00085FFFCCF72
:100330008AE08093C60098C086E40E94F95D882315
:10034000E1F00E9410637B018C0160930D0C7093AF
:100350000E0C80930F0C9093100C20E030E040E0E6
:1003600050E00E94A89A181644F4E092F903F09223
:10037000FA030093FB031093FC03E1EEFBE094917E
:1003800008C08091C00085FFFCCF9093C6003196D5
:1003900094919923B1F7ECE2F3E007C08091C0009B
:1003A00085FFFCCF31969093C60090819923B1F7D9
:1003B0006091CA0B84E99BE070E04AE050E00E9443
:1003C0007A508091C00085FFFCCF8AE08093C60000
:1003D0004BC0E1EEFBE0949108C08091C00085FF26
:1003E000FCCF9093C600319694919923B1F7E1E93F
:1003F000FCE0949108C08091C00085FFFCCF9093F1
:10040000C600319694919923B1F72091170C309141
:10041000180C80E690E0289FF001299FF00D389F8E
:10042000F00D1124E75EF34F07C08091C00085FFF7
:10043000FCCF31969093C60090819923B1F7EFE8F5
:10044000FCE0949108C08091C00085FFFCCF9093A0
:10045000C600319694919923B1F78091C00085FF31
:10046000FCCF8AE08093C6000E94125B20C00E94ED
:10047000A2966093D00B7093D10B8093D20B909384
:10048000D30B0E94A2966093E80B7093E90B8093C4
:10049000EA0B9093EB0BE8CF0E942D1388E50E94A6
:1004A000F95D882311F00C94F0770C94F377C55321
:1004B000DF4F0FB6F894DEBF0FBECDBFCF91DF91F7
:1004C0001F910F91FF90EF90DF90CF90BF90AF9072
:1004D0009F908F907F906F905F904F903F902F9064
:1004E00008958091E60B9091E70B039714F40E9416
:1004F0005D648091E60B9091E70B892BC1F00E941F
:1005000049678091E60B9091E70B01979093E70B79
:100510008093E60B8091170C9091180C019664E083
:1005200070E00E947F9C9093180C8093170C07D763
:100530000E94DE660C943E1BDF93CF930F920F92C6
:10054000CDB7DEB79D9AA59884E99BE040E052ECD8
:1005500061E070E00E94334FECEEF0E1949108C04E
:100560008091C00085FFFCCF9093C6003196949196
:100570009923B1F78091C00085FFFCCF8AE080937A
:10058000C60041EE5BE0FA01949108C08091C00082
:1005900085FFFCCF9093C600319694919923B1F7D3
:1005A00084B7282F80FF15C0E4EEF0E1949108C0D5
:1005B0008091C00085FFFCCF9093C6003196949146
:1005C0009923B1F78091C00085FFFCCF8AE080932A
:1005D000C60021FF15C0E4EDF0E1949108C08091C0
:1005E000C00085FFFCCF9093C6003196949199236B
:1005F000B1F78091C00085FFFCCF8AE08093C600F0
:1006000022FF15C0E3ECF0E1949108C08091C00096
:1006100085FFFCCF9093C600319694919923B1F752
:100620008091C00085FFFCCF8AE08093C60023FF45
:1006300015C0E3EBF0E1949108C08091C00085FF04
:10064000FCCF9093C600319694919923B1F7809195
:10065000C00085FFFCCF8AE08093C60025FF15C04F
:10066000E3EAF0E1949108C08091C00085FFFCCFDF
:100670009093C600319694919923B1F78091C00070
:1006800085FFFCCF8AE08093C60014BEECE9F0E160
:10069000949108C08091C00085FFFCCF9093C60064
:1006A000319694919923B1F7E6E9F0E1949108C06D
:1006B0008091C00085FFFCCF9093C6003196949145
:1006C0009923B1F78091C00085FFFCCF8AE0809329
:1006D000C600FA019491E1EEFBE008C08091C000F1
:1006E00085FFFCCF9093C600319694919923B1F782
:1006F000E6E8F0E1949108C08091C00085FFFCCF4E
:100700009093C600319694919923B1F7E1E7F0E117
:10071000949108C08091C00085FFFCCF9093C600E3
:10072000319694919923B1F7E5E6F0E1949108C0F0
:100730008091C00085FFFCCF9093C60031969491C4
:100740009923B1F7E4E4F0E1949108C08091C000EE
:1007500085FFFCCF9093C600319694919923B1F711
:100760008091C00085FFFCCF8AE08093C600E9E35A
:10077000F0E1949108C08091C00085FFFCCF909378
:10078000C600319694919923B1F7EDE2F0E194918E
:1007900008C08091C00085FFFCCF9093C6003196C1
:1007A00094919923B1F78091C00085FFFCCF8AE036
:1007B0008093C600FA019491E1EEFBE008C08091BD
:1007C000C00085FFFCCF9093C60031969491992389
:1007D000B1F7EEE1F0E1949108C08091C00085FF8F
:1007E000FCCF9093C600319694919923B1F7209154
:1007F000DC0E3091DD0ECE0101962115310519F484
:10080000825E9E4002C0821B930B9A83898369811A
:100810007A8184E99BE04AE050E00E947A50E7E068
:10082000F0E1949108C08091C00085FFFCCF9093C7
:10083000C600319694919923B1F784E99BE060E179
:1008400075E04AE050E00E947A508091C00085FF38
:10085000FCCF8AE08093C60010929F0D1092A00DED
:100860001092A10D1092A20D0E947E586FD40E948A
:10087000A2200E94C2120E949D60809101018860A6
:100880008093010186E06FEF0E94E69386E06FEFB0
:1008900070E00E947C9580E197E220E931E0F90167
:1008A0003197F1F70197D9F786E062E80E94E69365
:1008B00086E062E870E00E947C950F900F90CF91E7
:1008C000DF91089560E070E08CE593E420910204EC
:1008D0003091030440910404509105040E94A198B2
:1008E0006093D50D7093D60D8093D70D9093D80D4E
:1008F00060E070E08CE593E42091120430911304E1
:1009000040911404509115040E94A1986093DD0D4C
:100910007093DE0D8093DF0D9093E00D0895FC0140
:1009200097FF03C08091B70D03C0E854F24F808158
:1009300090E008952F923F924F925F926F927F9234
:100940008F929F92AF92BF92CF92DF92EF92FF92DF
:100950000F931F93CF93DF93EC0121E030E0A901C7
:10096000440F551F440F551FFA01EC53FE4E85915D
:100970009491C817D9070CF059C0B9016150704063
:10098000660F771F660F771FCB018A539E4EFC01BF
:10099000059114916C537E4EFB01C590D490FA01E1
:1009A000EA53FE4EE590F490FA01EC53FE4EA5900A
:1009B000B490B801882777FD8095982F0E943C99C4
:1009C0001B012C01CC19DD09BE01882777FD80951C
:1009D000982F0E943C993B014C01E01AF10A002734
:1009E000F7FC0095102FC801B7010E943C999B01AC
:1009F000AC01C401B3010E947A9B7B018C01AC184D
:100A0000BD08CC24B7FCC094DC2CC601B5010E9403
:100A10003C999B01AC01C801B7010E94A1989B01C0
:100A2000AC01C201B1010E94C19719C0822F8F5F32
:100A30002F5F3F4F2A33310509F091CF8A3329F0D8
:100A4000E0E070E080E060E00CC0EAEAF2E165918D
:100A50007491882777FD8095982F0E943C99E62F06
:100A6000692F2E2F372F482F562FB901CA01DF913A
:100A7000CF911F910F91FF90EF90DF90CF90BF909B
:100A8000AF909F908F907F906F905F904F903F902E
:100A90002F90089508951092A80D1092A70D10920E
:100AA000B80D75981092AA0D1092A90D1092B90D5B
:100AB0009FB7F894E2E0F1E080818F7E80839FBF52
:100AC0001092AA0D1092A90D1092B70DA598089535
:100AD0002DEB37E346E05EE30C947A9B2DEB37E396
:100AE00046E05EE30C94A1982DEB37E346E05EE32D
:100AF0000C94A1982DEB37E346E05EE30C947A9BCF
:100B0000A5980E94585A882319F5ECE0F1E19491D8
:100B100008C08091C00085FFFCCF9093C60031963D
:100B200094919923B1F7E3E1F1E1949108C08091A8
:100B3000C00085FFFCCF9093C60031969491992315
:100B4000B1F78091C00085FFFCCF8AE08093C6009A
:100B50000C949F5A1F93182F9EDF0E94585A882387
:100B600091F5ECE0F1E1949108C08091C00085FF1F
:100B7000FCCF9093C600319694919923B1F784E904
:100B80009BE0612F70E04AE050E00E947A50809133
:100B9000C00085FFFCCF8AE08093C600EDE4F1E160
:100BA000949108C08091C00085FFFCCF9093C6004F
:100BB000319694919923B1F78091C00085FFFCCFC5
:100BC0008AE08093C6000E949F5A1F9108951F9348
:100BD000182F61DF0E94585A882391F5ECE0F1E16B
:100BE000949108C08091C00085FFFCCF9093C6000F
:100BF000319694919923B1F784E99BE0612F70E0DD
:100C00004AE050E00E947A508091C00085FFFCCFFE
:100C10008AE08093C600EAE7F1E1949108C08091F0
:100C2000C00085FFFCCF9093C60031969491992324
:100C3000B1F78091C00085FFFCCF8AE08093C600A9
:100C40000E949F5A1F9108951F920F920FB60F9204
:100C50000BB60F9211242F933F934F935F936F9393
:100C60007F938F939F93AF93BF93EF93FF93909155
:100C70001C04992391F48091B80D8093BF0D8823B3
:100C800011F0759A01C075988091B70D8093BE0DD3
:100C9000882311F0A59A01C0A5988091BF0D8917EE
:100CA00008F475988091BE0D891708F4A5989F5F88
:100CB0009F7790931C0480911D04843009F46BC0CD
:100CC000853050F4813009F1813098F08230D9F1CB
:100CD000833009F094C043C0863009F484C0863064
:100CE00008F465C0873009F480C0883009F087C0F7
:100CF00084C010927B0080E480937C0080917A0015
:100D0000806480937A0081E01BC08091780090918C
:100D10007900A0E0B0E02091CC0D3091CD0D409154
:100D2000CE0D5091CF0D280F391F4A1F5B1F209306
:100D3000CC0D3093CD0D4093CE0D5093CF0D82E06E
:100D400080931D045CC010927B0082E480937C0041
:100D500080917A00806480937A0083E0F1CF809163
:100D6000780090917900A0E0B0E02091C00D309122
:100D7000C10D4091C20D5091C30D280F391F4A1F5C
:100D80005B1F2093C00D3093C10D4093C20D509353
:100D9000C30D84E0D5CF10927B0081E480937C006A
:100DA00080917A00806480937A0085E0C9CF809139
:100DB000780090917900A0E0B0E02091C80D3091CA
:100DC000C90D4091CA0D5091CB0D280F391F4A1FF4
:100DD0005B1F2093C80D3093C90D4093CA0D5093EB
:100DE000CB0D86E0ADCF87E0ABCF10921D04809194
:100DF000D00D8F5F8093D00D02C010921D048091A2
:100E0000D00D803108F463C08091B90D882381F43E
:100E10008091CC0D9091CD0D9093AC0D8093AB0D46
:100E20008091C00D9091C10D9093B20D8093B10D42
:100E300081E08093B90D1092D00D1092CC0D1092DC
:100E4000CD0D1092CE0D1092CF0D1092C80D1092B4
:100E5000C90D1092CA0D1092CB0D1092C40D1092B4
:100E6000C50D1092C60D1092C70D1092C00D1092B4
:100E7000C10D1092C20D1092C30D2091AB0D309197
:100E8000AC0D8091BA0D9091BB0D8217930714F0B1
:100E900080E09DDE2091AB0D3091AC0D80911A0465
:100EA00090911B042817390714F080E053DE20913D
:100EB000B10D3091B20D8091BC0D9091BD0D821796
:100EC00093072CF01092AA0D1092A90D19DEFF9134
:100ED000EF91BF91AF919F918F917F916F915F91B2
:100EE0004F913F912F910F900BBE0F900FBE0F901F
:100EF0001F9018952F926F927F928F929F92AF9230
:100F0000BF92CF92DF92EF92FF920F931F93DF93E6
:100F1000CF93CDB7DEB729970FB6F894DEBF0FBEDB
:100F2000CDBF8C01E62E662369F1ECE0F1E19491EE
:100F300008C08091C00085FFFCCF9093C600319619
:100F400094919923B1F784E99BE06E2D70E04AE01B
:100F500050E00E947A50E7EAF1E1949108C0809154
:100F6000C00085FFFCCF9093C600319694919923E1
:100F7000B1F78091C00085FFFCCF8AE08093C60066
:100F80000E94DD5AAE2DB0E0FD01EE0FFF1FE956C5
:100F9000FB4F6081718179876887672B09F49FC057
:100FA000A756BB4F7C917B832224239479C0222DAA
:100FB00030E0A901440F551F440F551FE885F985FE
:100FC000E40FF51F85919491081719070CF067C07D
:100FD000C9010197880F991F880F991FFC0132964C
:100FE000A885B985EA0FFB1FC590D4908A0F9B1F77
:100FF000FC01659174917A836983FA013296EA0F54
:10100000FB1FE590F490FD01E40FF51FA590B4904F
:10101000B601882777FD8095982F0E943C996C83B4
:101020007D838E839F8389819A81081B190BB80168
:10103000882777FD8095982F0E943C993B014C01B1
:10104000EC18FD080027F7FC0095102FC801B70128
:101050000E943C999B01AC01C401B3010E947A9BA0
:101060007B018C01A981BA81AA1ABB0ACC24B7FCE6
:10107000C094DC2CC601B5010E943C999B01AC01D7
:10108000C801B7010E94A1989B01AC016C817D81D0
:101090008E819F810E94C197E62F692F09C02394FA
:1010A000BB812B1608F483CFE0E070E080E060E0C5
:1010B000FB812F1679F5E22DF0E0EE0FFF1FEE0F0A
:1010C000FF1F329768857985E60FF71F6591749148
:1010D000882777FD8095982F0E943C9919C0B80108
:1010E000882777FD8095982F0E943C9920E030E07A
:1010F0004AEF5EE30E947A9B20E030E040E85DE347
:101100000E947A9B20E030E040E050E00E94C197CE
:10111000E62F692F2E2F372F482F562FB901CA01DE
:1011200029960FB6F894DEBF0FBECDBFCF91DF91E9
:101130001F910F91FF90EF90DF90CF90BF90AF90F5
:101140009F908F907F906F902F900895EF92FF92D5
:101150000F931F93CF93DF930F2EF0E0EF2EF0E06D
:10116000FF2EF0E00F2FF0E01F2FF02DE092D10DB9
:10117000F092D20D0093D30D1093D40D60E070E087
:101180008CE593E42091020430910304409104041F
:10119000509105040E94A1986093D50D7093D60DCF
:1011A0008093D70D9093D80DE092D90DF092DA0D7F
:1011B0000093DB0D1093DC0D60E070E08CE593E4B0
:1011C000209112043091130440911404509115049D
:1011D0000E94A1986093DD0D7093DE0D8093DF0D6A
:1011E0009093E00D6D9A80910101806180930101DF
:1011F0009D9A8091010180628093010188E061E005
:1012000070E00E945B5A87ED80937A0010927E0016
:1012100010927D0080917E00816080937E0080919D
:101220007E00826080937E0080917E008460809347
:101230007E0080E888BD80916E00846080936E009F
:101240006AEF70E080E090E00E94B09685E090E068
:101250009093E20D8093E10D09C080911A04909162
:101260001B04409790931B0480931A0480911A04E6
:1012700090911B0460E03EDE20E030E040EA50E464
:101280000E949A9887FDE9CF81E391E090931F0433
:1012900080931E0409C08091BA0D9091BB0D4096B9
:1012A0009093BB0D8093BA0D8091BA0D9091BB0DB8
:1012B00060E020DE20E030E848E953E40E94A89A8C
:1012C00018164CF3C091BC0DD091BD0DEC2E1D2F06
:1012D000CE0130DB609620E030E046E153E40E942E
:1012E000A89A18169CF3E092BC0D1093BD0DDF91E7
:1012F000CF911F910F91FF90EF9008958091AB0DCA
:101300009091AC0D60E0F6DD6093AD0D7093AE0D85
:101310008093AF0D9093B00D8091B10D9091B20D6F
:1013200009DB6093B30D7093B40D8093B50D90936A
:10133000B60D8FB7F8941092B90D8FBF08952F9204
:101340003F924F925F926F927F928F929F92AF9255
:10135000BF92CF92DF92EF92FF920F931F938091F3
:10136000B90D882309F478C2C9DF6090AD0D709083
:10137000AE0D8090AF0D9090B00DC090A70DD090A5
:10138000A80DB601882777FD8095982F0E943C997B
:10139000A40193010E94C0977B018C016093E30D2F
:1013A0007093E40D8093E50D9093E60D20E030E01E
:1013B00040E851E40E94A89A181674F481E08093E2
:1013C000E70D0F2EF0E0EF2EF0E0FF2EFCE50F2FE3
:1013D000F3E41F2FF02DF3C0C801B70120E030E087
:1013E00040E851EC0E949A9887FD02C0CD2821F474
:1013F00081E08093E70DC4C08091E70D882371F0F0
:1014000080E090E0A0E0B0E08093E80D9093E90DDB
:10141000A093EA0DB093EB0D1092E70DC801B70150
:101420002091FE033091FF0340910004509101048C
:101430000E947A9B1B012C016093EC0D7093ED0DC3
:101440008093EE0D9093EF0DC801B7012091E80D48
:101450003091E90D4091EA0D5091EB0D0E94C1973A
:101460005B016C01E090D10DF090D20D0091D30D95
:101470001091D40DA80197010E949A9887FD12C07F
:10148000E090D50DF090D60D0091D70D1091D80DAC
:10149000C601B501A80197010E94A89A181614F078
:1014A00086017501E092E80DF092E90D0093EA0DD6
:1014B0001093EB0DC801B701209102043091030491
:1014C00040910404509105040E947A9B5B016C01D9
:1014D0006093F00D7093F10D8093F20D9093F30DE6
:1014E000C401B3012091F40D3091F50D4091F60D3A
:1014F0005091F70D0E94C097209106043091070487
:1015000040910804509109040E947A9B20ED3CEC24
:101510004CE45DE30E947A9B7B018C016091F80DA5
:101520007091F90D8091FA0D9091FB0D23E333E357
:1015300043E75FE30E947A9B9B01AC01C801B701BE
:101540000E94C1977B018C016093F80D7093F90D97
:101550008093FA0D9093FB0DC201B101A601950194
:101560000E94C197A80197010E94C0977B018C013E
:1015700020E030E040E050E00E949A9888235CF43C
:101580000F2EF0E0EF2EF0E0FF2EF0E00F2FF0E056
:101590001F2FF02D14C0C801B70120E030E041E654
:1015A00053E40E94A89A181654F40F2EF0E0EF2E80
:1015B000F0E0FF2EF1E60F2FF3E41F2FF02D6092E5
:1015C000F40D7092F50D8092F60D9092F70D6091EA
:1015D000E10D7091E20D882777FD8095982F0E948C
:1015E0003C999B01AC01C401B3010E94A89A181652
:1015F000DCF460911E0470911F04882777FD8095AC
:10160000982F0E943C999B01AC01C401B3010E9438
:101610009A9888234CF4C801B7010E9409997595DE
:1016200067956093B80D02C01092B80D6090B30D2D
:101630007090B40D8090B50D9090B60D6091A90D8D
:101640007091AA0D882777FD8095982F0E943C996C
:10165000A40193010E94C0977B018C016093FC0D53
:101660007093FD0D8093FE0D9093FF0D20910E045D
:1016700030910F0440911004509111040E947A9B04
:101680001B012C016093000E7093010E8093020EDB
:101690009093030EC801B7012091040E3091050EFE
:1016A0004091060E5091070E0E94C1975B016C019C
:1016B000E090D90DF090DA0D0091DB0D1091DC0D6A
:1016C000A80197010E949A9887FD12C0E090DD0D55
:1016D000F090DE0D0091DF0D1091E00DC601B50117
:1016E000A80197010E94A89A181614F086017501A6
:1016F000E092040EF092050E0093060E1093070E72
:10170000C801B701209112043091130440911404D0
:10171000509115040E947A9B5B016C016093080E46
:101720007093090E80930A0E90930B0EC401B301BF
:1017300020910C0E30910D0E40910E0E50910F0E17
:101740000E94C0972091160430911704409118040C
:10175000509119040E947A9B20ED3CEC4CE45DE32F
:101760000E947A9B7B018C016091100E7091110E8A
:101770008091120E9091130E23E333E343E75FE36E
:101780000E947A9B9B01AC01C801B7010E94C197DE
:101790007B018C016093100E7093110E8093120EDA
:1017A0009093130E60920C0E70920D0E80920E0E9E
:1017B00090920F0EC201B101A60195010E94C1973E
:1017C000A80197010E94C0977B018C0120E030E0C6
:1017D00040E050E00E949A9888235CF40F2EF0E0DD
:1017E000EF2EF0E0FF2EF0E00F2FF0E01F2FF02D96
:1017F00014C0C801B70120E030E04FE753E40E9475
:10180000A89A181654F40F2EF0E0EF2EF0E0FF2EF9
:10181000FFE70F2FF3E41F2FF02DC401B30120E0E9
:1018200030E040EA50E40E94A89A18169CF4C401E3
:10183000B30120E030E046E153E40E949A98882307
:101840004CF4C801B7010E9409997595679560939A
:10185000B70D02C01092B70D1F910F91FF90EF903E
:10186000DF90CF90BF90AF909F908F907F906F90C0
:101870005F904F903F902F9008952F923F924F92FC
:101880005F926F927F928F929F92AF92BF92CF9210
:10189000DF92EF92FF920F931F93DF93CF93CDB719
:1018A000DEB7E6970FB6F894DEBF0FBECDBF6C8FE4
:1018B0007D8F8E8F9F8F5EAB4DAB39A328A30E9487
:1018C000A296698B7A8B8B8B9C8B2DA93EA922309B
:1018D00031051CF4EEE3F3E019C0E1E5F3E007C0E5
:1018E0008091C00085FFFCCF31969093C600908117
:1018F0009923B1F78091C00085FFFCCF42C480914D
:10190000C00085FFFCCF31969093C600908199234B
:10191000B1F78091C00085FFFCCF8AE08093C600BC
:10192000BAD84DA95EA957FF0EC08FE78093B70DB7
:101930002FE7A22EB12CC12CD12C9FE7292E312CC0
:10194000412C512C10C0EDA9FEA9E854F24F80E7BC
:10195000808380E7A82EB12CC12CD12C00E7202E4B
:10196000312C412C512C89899A89AB89BC898D876E
:101970009E87AF87B88B89879A87AB87BC8719AA60
:101980001AAA1BAA1CAA1F8A1E8A91E09D8B1D827F
:101990001E821F82188620E030E040E050E029835C
:1019A0003A834B835C830F2EF0E06F2EF0E47F2EA2
:1019B000FCE18F2EF6E49F2EF02D4DA95EA9485430
:1019C000524F5BA34AA3EDE8F3E154915CA3E8E82E
:1019D000F3E184918DA3E1E8F3E194919EA3EAE71A
:1019E000F3E1A491AFA3E4E7F3E1B491B8A7EEE685
:1019F000F3E1249129A7E1E6F3E134913AA7EBE57D
:101A0000F3E144914BA7E5E5F3E154915CA7EFE4E2
:101A1000F3E184918DA7ADA9BEA9AA0FBB1FAA0FA0
:101A2000BB1FA355B24FBFA7AEA7E5E1F3E1B49149
:101A3000B8AB8091B90D882309F4CDC25FDCEDA964
:101A4000FEA9F7FF0DC0F091B30DF9AB2091B40DD5
:101A50002AAB3091B50D3BAB4091B60D4CAB11C0EC
:101A6000AEA5BFA5BC91B9ABEEA5FFA5F181FAABC0
:101A7000AEA5BFA51296BC91BBABEEA5FFA5F381A9
:101A8000FCAB69817A818B819C8129A93AA94BA9F8
:101A90005CA90E94A89A181644F089A99AA9ABA932
:101AA000BCA989839A83AB83BC83C401B30129A9F0
:101AB0003AA94BA95CA90E949A9887FD06C089A9FA
:101AC0009AA9ABA9BCA93C014D012D89222309F497
:101AD00051C069A97AA98BA99CA92C8D3D8D4E8DE9
:101AE0005F8D0E94A89A18160CF075C20E94A296EB
:101AF00029853A854B855C85621B730B840B950B9E
:101B0000695873418040904008F465C2D601C50110
:101B100082199309A409B5094DA95EA957FF07C009
:101B2000B595A795979587958093B70D07C0B595FF
:101B3000A79597958795EAA1FBA180830E94A2961D
:101B40006D877E878F87988B9B01AC0189859A85ED
:101B5000AB85BC85281B390B4A0B5B0B2D833E8361
:101B60004F8358872C8D3D8D4E8D5F8D29833A8311
:101B70004B835C8369A97AA98BA99CA92C8D3D8D87
:101B80004E8D5F8D0E949A9888230CF023C20E948C
:101B9000A2962D853E854F855889621B730B840B59
:101BA000950B695873418040904008F413C20E941D
:101BB000A29669877A878B879C874E895F89452B98
:101BC00009F4E3C1DC01CB012D853E854F855889A1
:101BD000821B930BA40BB50B2D813E814F81588541
:101BE000280F391F4A1F5B1F288F398F4A8F5B8F41
:101BF0002D813E814F815885281B390B4A0B5B0B89
:101C0000CA01B901A20191010E944C9C288D398D15
